:020000040800F2
:1000000000A00020EDD60008B9AD000831C80008F6
:10001000B7AD0008B5AD0008B3AD000800000000A2
:10002000000000000000000000000000B1AD00086A
:10003000AFAD000800000000ADAD0008D3A100087E
:1000400055D7000855D7000855D7000855D70008E0
:1000500055D7000855D7000855D7000855D70008D0
:1000600055D7000855D7000855D7000855D70008C0
:1000700055D70008A5AA00086F95000855D70008B5
:1000800055D7000855D7000855D7000855D70008A0
:1000900019AE000855D7000855D7000855D70008F5
:1000A00091840008BD84000881840008CD84000884
:1000B000B1840008A184000855D7000855D700086E
:1000C00055D7000855D7000855D7000855D7000860
:1000D00055D70008898600087D86000871860008CB
:1000E000E1A1000855D7000899C7000855D70008B6
:1000F00055D7000855D7000855D7000855D7000830
:1001000000000000000000000000000055D70008BB
:1001100055D7000855D7000855D7000855D700080F
:1001200055D7000855D7000855D7000855D70008FF
:1001300055D7000855D70008000000000000000057
:1001400055D7000855D7000855D700080000000013
:10015000000000000000000000000000000000009F
:10016000000000000000000055D7000855D7000827
:1001700055D700080000000000000000000000004B
:080180000000000055D7000843
:100188002DE9F04F2DED028B924D934B2B60A9B0CA
:1001980000236B6007F043FE18B907F063FE05F013
:1001A80025FE05F0E1FE8D4B8D4C1A7842F00102D8
:1001B8001A708C4A4FF47001C2F888100022099214
:1001C8000A92226842F4803222600493236803F47E
:1001D80000330A93099B013309930A9B1BB9099BB6
:1001E800B3F5A04FF2D1236813F4003318BF0123ED
:1001F8000A930A9B012B6FD07A4F7B4BFB60636A93
:10020800AB60636ADFF814A2DFF81482DFF8149297
:1002180043F080736362636943F4FC0328AE63614F
:1002280003238DF8523041F6FF7326F8503D4FF006
:10023800904031460AF04AFC4FF6FF73504631466B
:10024800ADF850300AF042FC684831460AF03EFCEE
:10025800674831460AF03AFC664831460AF036FCEF
:10026800314665480AF032FC304604F02DFF149BF5
:10027800624AB3FBF2F3624A62491360624B00229E
:100288001A60624B5960F02187F823109A60604F1A
:1002980007221A60BB68C8F8003099E80F0086E8A2
:1002A8000F006369149843F480236361636943F41E
:1002B800802363611023CAF818302023CAF8183045
:1002C80015A90AF003FC169817A90AF0FFFBD8F83D
:1002D8000030180729D4A7E04E4B12221A60636831
:1002E800636063686360636843F480636360636842
:1002F80023F47C136360636843F4E8136360236842
:1003080043F0807323602268354B9101FBD55A680E
:1003180022F003025A605A6842F002025A60636887
:1003280003F00C03082BFAD166E797F89231012BFA
:100338007AD8D9F8100030603146504697F893B112
:100348000AF0C4FB0A2009F02BFFBAF8103003F4B6
:1003580080539BB2002B67D11E4A9268D20040F1AD
:100368008784DB0760D52C4BDFF8B0A018684FF006
:10037800200BAAF828B0314614904FF090400AF0AC
:10038800A5FB4FF0904308229A613C2009F013FF27
:10039800CAF818B04FF0000A97F893319A4543DA33
:1003A8001E4A4FF0904B1021082391617820069146
:1003B8000592ABF82830039309F0F2FE059A0699E6
:1003C800039B11857820CBF8183009F0E9FE0AF173
:1003D800010AE1E770010020A9560008CA2200209E
:1003E8000010024000ED00E00005FA050008004892
:1003F800000C0048001000480014004840420F005C
:10040800D81700203F190100DC17002010E000E099
:10041800CC1A0020002002407007010800040048A0
:10042800082200205C070108642009F0C4FEC822E5
:10043800CB4800210EF035FDE369CA4A43F00303B7
:10044800E361A36943F4A123A361636943F4C0236F
:10045800636102F1B00C937B506892F80FE003F0EF
:100468000701DB0800EB83038900186A4FF00F0AC5
:100478000EFA01FE0AFA01F120EA01011962196A6D
:1004880010324EEA010162451962E4D10023DFF817
:100498000CA30AF10C020021995401330B2BF6D15D
:1004A800FF23B14A8AF817308AF818308AF81930C9
:1004B8008AF81A308AF81B30AC4BDFF8E4B21360C4
:1004C800AB4A039304201070584630220EF0E9FC22
:1004D800142202218BF800208BF824100122A54950
:1004E800039B8BF8182097F805B081F800B0A3F5A6
:1004F800EE71CAF81C10A049D8F80080A3F58E73D5
:100508000B609E4B03EBCB0318F0200F5B78CAF807
:10051800203018BFCAF820200023994A40F2DC5145
:1005280022F813100133082BF7D10DA800211C2243
:100538000EF0B7FCBBF10E0F03D00BF0EF03082B46
:1005480002D101238DF84430022007F0B7F818B122
:100558004088003018BF0120C8F340038DF83A30B6
:10056800C8F380138DF83C30C8F340338DF834302D
:10057800C8F3C03300F001008DF8373018F4006379
:100588008DF8390007D097F8863103F1FF3EDEF188
:10059800000343EB0E038DF83830C8F300438DF8A1
:1005A8003D302B6AB7F84801ADF84800003318BF52
:1005B80001238DF83E30C8F300538DF83F30B7F86B
:1005C8004A31ADF8423018F4805FB7F8563118BF99
:1005D8006C48ADF84030C8F380438DF83B30B7F82D
:1005E80054311CBFB0F85001ADF84800B3F5FA7F9C
:1005F800ADF8463084BF0023ADF84830624897F81C
:10060800D63185F82430002385F8253043709DF8CD
:10061800443008F00101002BC8F3C0028DF83510F2
:100628008DF836200CBF0023022301B902B1013333
:1006380009EB83094FF0000AD9F818309A1E1433D1
:1006480003920593039A32F8023F03924FF6FF7222
:10065800934200F04581DAB2190A9DF839307BB12E
:10066800404B4A4F03EB02135868B84208D11B8924
:10067800B3F5806F00F02F81B3F5006F00F02B8188
:100688009DF83A3053B1374B03EB02135868B0F179
:10069800904F03D11B89102B00F01D81022902D134
:1006A8009DF8343003E0012904D19DF83530002B42
:1006B80000F011812B4F9DF83F304FEA02194F444B
:1006C80033B19DF844301BB9043A032A40F2EC8058
:1006D8000129CBB266D1FF2385F86C3085F86D30DF
:1006E800204BEF6703EB09024FF00008517B50687D
:1006F8008DF8521002F1080B1289ADF8502014A998
:10070800022285F8708006938DF8532085F828809A
:10071800C5F82C80C5F83080C5F83480C5F86880E5
:1007280085F86E8085F86F800AF0D0F9069B9BF8F3
:10073800021053F8090042460AF0FAF838460AF05F
:10074800EBFF134B1349C5F88030134BC5F88430C1
:10075800C5F8888038460A1D07F02CFFBBE000BFAB
:100768002818002068200108640F0020BC1C002005
:10077800060400206C0600206C190020B022010835
:10078800F6030020CC1A0020950100200004004840
:10079800F1A60008F0010020D1A700087001002090
:1007A8002C0F0020022B46D15FFA8AF21C2101FB94
:1007B80002FC05EB0C089B4A88F871A0012188F817
:1007C800701002EB09014FF0000B91F80DE048683A
:1007D80088F872B001F108020989ADF8501088F85C
:1007E8007AB014A9C8F87C70CDF81CC08DF852E016
:1007F80006928DF853300AF069F98A4B069A53F835
:10080800090091785A460AF093F838460AF084FFAE
:10081800DDF81CC08449854AC8F880206144844AB0
:10082800C8F88420C8F888B038460A1D07F0C2FE08
:100838000AF1010A4FE0032B34D19DF83B30DFF871
:100848002C823BB195F82690384608214FF6FF7266
:1008580000231BE0BDF846207649BDF8483091F8E2
:100868002690B2F5FA7F0BD97349B1FBF2F23846FC
:10087800082192B20AF053F9704B48F829000AE0AF
:100888006F49B1FBF2F23846012192B20AF047F9FA
:100898006C4B48F82900C36095F82630013385F879
:1008A800263018E0042B16D195F82580BDF8402095
:1008B800634B93FBF2F23846BDF84230012192B205
:1008C8000AF02DF995F8253005EB88080133C8F8AA
:1008D800500185F82530039B059A93427FF4B2AE08
:1008E80095F8252085F87021574A584B92F800E072
:1008F800AEF117020027022A1F709C461AD8EB692E
:100908003B44D3ED007AF5EE407AF1EE10FA02D1CD
:100918002B6A73BB26E04E4A07EB02080FCB88E828
:100928000F009CF8003010370133C02F8CF80030CE
:10093800E5D1EDE7474B13F83E908CF8009003EBB8
:10094800CE03D3F804A0BAF1000FE1D04F45DFDAA7
:100958003F4A3B0103EB020853440FCB013788E8B9
:100968000F00F3E73C4B03931A6812F4805F24D11D
:100978001DE03A4B3A4A13F83E00107003EBCE03E1
:100988005D68002DEED000238342EBDAC3EBC30190
:100998006A18DFF8DC80D2F8009041F8089001EB83
:1009A80008079188B9809279BA710133ECE70EF0A3
:1009B800EF03082B2B4B20D122E09CF80020012AC2
:1009C800F5D9294B03EB0212103210339342EED0C3
:1009D80053ED047AB6EE007A67EE877A43ED047A2F
:1009E80053ED057A67EE877A43ED057A53ED037A7E
:1009F80067EE877A43ED037AE7E7BEF10E0F09D178
:100A08001A7842F010021A70BEF1180F32D109F0AC
:100A180093FD2FE01A7822F010021A70BEF1190F18
:100A2800F4E700BF68200108F001002035AA00089B
:100A3800C9A600087001002000127A00F1A700087A
:100A480040420F00E1A700086C060020D6170020DE
:100A5800A8050020B022010808220020B40B0108D4
:100A6800F81800209A0B0020B0050020F817002085
:100A7800F918002009F044FD039B1B685D0358BF6B
:100A8800AE4BAF4D5CBF01221A70049B049A1B78D1
:100A980043F0040313702023ADF8503011238DF870
:100AA800523063694FF0020843F4003331468DF841
:100AB80053804FF0904063610AF008F8A14BA24AB6
:100AC8001A60002009F090FBA04B1D60636943F495
:100AD80000336361E36943F48003E361236B23F02C
:100AE80020032363236B43F080534FF0904743F078
:100AF800200323637B6A23F0F0037B627B6A43F065
:100B080040037B627B6A23F470637B627B6A43F4F5
:100B180080634FF000097B6231464FF400734FF059
:100B2800030A384614938DF856908DF857908DF82F
:100B380054808DF855A004F035FC4FF4806331469D
:100B48003846149304F02EFC2B68814E23F00103E1
:100B58002B602A687F4B13402B607F4B2B612B68DF
:100B680043F001032B60C5F80890C5F80C90C5F850
:100B78000890AB6843F40043AB602B682B606B684C
:100B880023F0784323F400436B602B6843F00103A0
:100B98002B60039B4FF0100B1D68304649465A46A0
:100BA8000EF07FF905EA08054FF6FF730B938DF8F1
:100BB80031808DF832908DF833908DF830A065B182
:100BC80028A9384641F874BD04F0ECFB0125072339
:100BD800357086F80190F370B570E36A23F4F87302
:100BE800E362E36A43F4D873E362636943F08053D2
:100BF80043F002036361594C204604F0D9F90023FD
:100C0800169318931E9319934FF480731A934FF405
:100C18008063534A1B932023204614921C93514A05
:100C280015924FF4005314A91D93ADF85C5004F0CD
:100C3800A1F9236843F0010323604B4CA36823F018
:100C48004053A360A36843F08053A3600A2009F0CF
:100C5800B2FAA36823F08043A360A368A360A368E3
:100C680043F00043A360A3683F4A002B08DAFAE781
:100C78000BF1FF33092B8CBF00230123FFF771BB56
:100C880093683A4923F040539360936843F00053C4
:100C980093608868364B034043F468338B60D168AF
:100CA800344B0B4043F40053D360136B013D23F0E6
:100CB8000F031D431563002401233219917800297D
:100CC80000F08B805D1C042B375DD078DFF898E04E
:100CD800EDB20ED803EB43035A00DEF830101F23A1
:100CE800934021EA030107FA02F30B43CEF83030B0
:100CF80050E0092B0ED8053B06225A43DEF8341083
:100D08001F23934021EA030107FA02F30B43CEF8AD
:100D180034303FE00E2B4FF006012DD8A3F10A0224
:100D28004A43DEF838C01F2393402CEA030107FA30
:100D380002F30B43CEF838302CE000BFD80A00206D
:100D480000580040D4220020E9990008901A002099
:100D5800EC0D0020FFE0CF007A25E00008040240F7
:100D680040010050FC0D002000010050000300501D
:100D7800E010FCFF07C0FFFD0F3B01FB03F2DEF8AC
:100D88003CC01F2393402CEA030107FA02F30B43EC
:100D9800CEF83C30092FA34A0FD99369A7F10A036B
:100DA80003EB430397690721994027EA0101916101
:100DB80091699840084390610EE053697B1E03EBEC
:100DC800430357693821994027EA01015161516964
:100DD80003339840084350612B460434102C7FF4A9
:100DE8006CAF904B9A6842F001029A601A461168FB
:100DF8008C4BC807FBD5DA688B4C22F00202DA600C
:100E0800DA6842F00202DA60DA6842F00102DA6077
:100E18009A6842F004029A60B4F85C31002B40F002
:100E28007384B4F95E21002A40F06E84B4F960211D
:100E3800002A40F069847D4B7D4E1B687D48B3F8DD
:100E48005630049300210C22B4F8647194F863B10D
:100E5800B4F80C9094F80FA0DFF80C82764D0EF0E1
:100E680020F83046002114220EF01BF8002388F8E1
:100E78000030C5F8743107F0EBFA002833D06F4B17
:100E880033606F4B73606F4BF360B7F5807F6E4BC9
:100E980033616E4B01D1002216E0BB2F01D901222C
:100EA80012E0612F01D902220EE0292F01D9032275
:100EB8000AE0132F01D9042206E0092F01D90522DF
:100EC80002E0002FE7D006221A706149614A0591B5
:100ED800042388F8003002230B70136843F00103E1
:100EE80013605A460EE0012006F0BEFDF8E04FF010
:100EF800010B0BFA02F140F2B2330B4043B1012A65
:100F08005BD9002254490023092A0B70F9D8EEE76F
:100F180011F04D0FF3D00692C5F8743107F098FA26
:100F2800069A0028EBD00620014614AA0AF070FBA6
:100F38009DF8551001EA0B029DF8531001EA0B01C8
:100F480001FA0BF343EA82019DF8512002EA0B03F0
:100F58000B430AD05BB25B4501D1002302E0022BB0
:100F68000DD1012385F8783110E00C2059460BAAE1
:100F78000AF04EFB9DF82C3013F00F0303D1032029
:100F880006F072FD02E0042BEBD1E6E7294B334A69
:100F98001A60334A5A6095F87821002A0CBF6F22EC
:100FA8006E221A722C4B04221A70059A032353706E
:100FB800284A136843F002031360264B1A6812F09C
:100FC800020F9B4602D01B4B1B689847254ABAF173
:100FD800000F4BD017F0FF0F0BD1DBF8003013F0E8
:100FE800020F4FF07D0140F2712308BF4FF4FA73EE
:100FF80002E04FF47A731946994505DBB9F57A6F23
:10100800A8BF4FF47A6900E099464B1E4B44B3FBE6
:10101800F1F3013BDBB203FB011185F87931116073
:1010280028E000BF00010050CC1A0020F40E002078
:10103800F010002054220020700100201D7D0008BF
:10104800517C0008B17B000890C1793D0000002068
:10105800FC00002050220020EB220020797D0008AF
:10106800917C0008080500202804002085F879A153
:10107800C2F8009033689847BF4B00221A7094F862
:1010880058210AB188F8002094F859210AB1BB49BF
:101098000A7094F85A2102B11A70DBF80030B84986
:1010A80013F0080F1AD0BDF91000DFEDB66A6422FC
:1010B80090FBF2F302FB130212B207EE902AB8EE8D
:1010C800E77A07EE903AF8EEE77AE7EE267AB2EE9C
:1010D800047A67EE877AC1ED007A01E000230B609D
:1010E800A94B1A7842F002021A70A84A20211185E9
:1010F800102191610A279946DFF89082B8F81430D8
:101108009BB283F02003A8F81430B8F814309BB2CF
:1011180083F01003A8F81430192009F04CF80120C6
:1011280009F062F8192009F046F8013F002009F09B
:101138005BF817F0FF07DFD11023C8F81830202319
:10114800C8F81830924B9FED938A1B689FED920A5E
:101158001B7BDFF8708207EE903AF8EEE77AA7EE8D
:10116800880A04F0E6FCB8F8003007EE903AF8EE8A
:10117800E77A27EE800A0EF0A3F8884B9FED887A6D
:101188001880B8F8003007EE903AF8EEE77A854B09
:10119800C7EE277AFF211B229FED837AC7EE877A55
:1011A8009FED827AC5ED5F7AD6ED047A804E67EEC0
:1011B800887A304667EE877AC3ED007A0DF071FEC3
:1011C8007C4A7D4B12683770012112F0020F18BF5C
:1011D800717019701FBF032119700221B170510776
:1011E80048BF1978304641BF4E1C1E70032646542E
:1011F80012F00A0F0CD01A7804218154511CC9B27C
:1012080005264654D11C0232D2B2197006218154E7
:10121800039A11688A0641BF1A78561C1E70072661
:1012280048BF86546679082E01D00E2E04D11A784C
:10123800571C1F700B2787541A7811F0040F4FF0B2
:101248000C0E00F802E002F101071CBFDFF868E1AC
:101258000232FFB21F701FBF8EF80020544A4FF0B1
:10126800100E02F807E01A78571CFFB24FF0120E62
:1012780011F4806F1F7000F802E00ED094F814E2A9
:10128800BEF1000F09D0DFF830E102328EF80020FD
:10129800474A4FF0130E02F807E01A7811F4007F5E
:1012A8004FF0140E00F802E002F101071CBFDFF84E
:1012B80008E10232FFB21F701FBF8EF800203C4ABF
:1012C8004FF0150E02F807E0182E0DD11A781627E0
:1012D8008754571CFFB24FF0170E00F807E0D71CD1
:1012E8000232D2B21F708654CE0541BF1A78511C03
:1012F80019701A2348BF8354002198222F480DF0F3
:10130800D0FD012006F0AEFA002600285CD0012EA0
:101318005AD82A4B4FF04C0A0AFB06F803EB080B85
:101328000BF148039F78049317B10136F6B2ECE746
:1013380090F9003090F804E01846214B03228DE81C
:10134800840001213A4653F82E3006F073F80590D0
:1013580068B15246584639460DF0A3FD174A059B19
:1013680042F808300123049A1E449370F6B2012013
:1013780006F05EFAC9E700BFEA220020EB2200204F
:10138800781900208988883CCA2200200004004877
:10139800B404002035FA8E3CDB0FC93FD00400208E
:1013A8000AE81C41B004002000401C46BD378635C1
:1013B800D503002050220020D40300203803002049
:1013C8002812010802000020A14BA24A1A60A24B71
:1013D800B4F852111980A14900230B808B70A049E1
:1013E8000A60B4F8982190B29E4921F8130001339D
:1013F800122BF9D1039B1B68D8045CBFB4F89E017B
:1014080008801F0740F1C18094F89231062B00F242
:10141800B680DFE803F004070E3C5674740045F20A
:10142800F05201E042F6F8228F4B1A800AF03BFB9B
:10143800A4E007EE902ADFED8D6A8B4BB8EEE77AD1
:10144800DFED8B7AE7EE267A42F6F8211980002341
:10145800FCEEE77A874A17EE901A42F82310013318
:10146800122BF7D1844A85491160854A40201370B0
:1014780006F0F8F9002800F082800123072690F989
:101488000000804A8DE8480040217F4B71E0764B90
:1014980042F6F8221A80784B7C4A1A60784B102260
:1014A80040201A7006F0DEF9002868D001230025D4
:1014B80090F90000764A8DE8280040214FF4E13386
:1014C80057E0694B42F6F8221A806B4B714A1A6052
:1014D8006B4B082240201A7006F0C4F900284ED041
:1014E8000121002390F900006B4A8DE80A00402191
:1014F8004FF4E13305F09EFFC5F880013BE05A4AFE
:10150800DFF8F8C1DFF8F8E1644F654E654D6648CD
:1015180042F6F82111805A490C22062B0A700DD088
:1015280000238CF800308EF800303B701B2333709A
:1015380005232A7003704FF4E1350AE000218CF886
:1015480000108EF8001039702A702121574D317023
:101558000370494B564A1A60402006F083F970B16F
:101568000122002390F900008DE80C00514A402127
:101578002B4605F05FFF003018BF012028B908206E
:1015880004F0FAFB3C4B4C4A1A604C4D3C4A2B6821
:1015980013F4804F1FBF082111703749484818BFFE
:1015A800086042F20101194003F0010003F40056FB
:1015B80079B12D4B44F62061198026B108231370A8
:1015C8002D4B4049196020B10C2313702A4B3E491A
:1015D80019601378043B537008F0C6FD3B4B186044
:1015E8006379052B02BF3A4B4FF4C8721A80394B06
:1015F8004FF47A721A80384A137843F0080313704C
:10160800364A137823F0020313702A6840F602035F
:1016180013406BB1324B334A1A60334B03221A70B2
:10162800324B01221A70324A00231380314A138048
:10163800A3682B60304B01221A7099F8003063F0D0
:101648007F0389F8003029B0BDEC028BBDE8F08F2C
:10165800940B0020561C0020980B00201422002018
:1016680004220020E80C002024050020CDCCCC3F2B
:101678000000B0C4A00C002074000020714A0008CB
:10168800C0210020DD4C0008A08601005D4A00084A
:10169800314C0008454A0008E54B00082C0D002095
:1016A8002E0D00202B0C00202F0D002090D00300C1
:1016B80061490008C54A000881BB000808220020CB
:1016C800A54A000875BB0008B54A000800050020B7
:1016D800AA0B0020E82200209A0B0020ED2200200F
:1016E800E80D0020481C00204C22002000010020AA
:1016F8001003002012030020D80A00202C0C002020
:101708002D0D002035FA8E3C1BB207EE903A5FEDA6
:10171800036AB4F95E31104AF8EEE77A07EE103A38
:1017280067EEA67AB4F96031CDED147A07EE903AF7
:10173800B8EEC77AF8EEE77A002127EE267A67EE48
:10174800A67A117014A805498DED157ACDED167A93
:1017580004F052FAFFF76FBB46000020C40D0020CA
:101768002DE9F04FC14BB3F90610C14B2DED028B9B
:101778001E68728989B09142039311DBB1F5FA6F43
:1017880096F807B0BDBF8B1A03FB0BF3A2F5FA6BF3
:10179800CBF1640BBCBF93FBFBFB0BF1640B01E0CB
:1017A8004FF0640BB34DB44B2A68059293F962214C
:1017B800B3F898A1059C029392B2079200225300B5
:1017C8000693AA4B33F912300493CAEB030303F2CE
:1017D800F31740F2E630874203D8002BB8BF5B42CC
:1017E80001E04FF4FA73022A01934FF06400059B5D
:1017F800A24F34D093F811E1BEF1000F06D0019B3F
:101808007345CCBFCEEB030300230193019BDFF8A4
:10181800B8E293FBF0FC6FF063093EF81C8009FB0B
:101828000C390CF1010C069B3EF91CE00FFA88FC00
:10183800CCEB0E0E0EFB09FE9EFBF0FEC64427F80D
:1018480003E0B718019B3F797B438D4F93FBF7F378
:1018580064339BB20BFB03F393FBF0F031E093F896
:1018680012E1BEF1000F06D0019B7345CCBFCEEB51
:10187800030300230193019BDFF8388293FBF0F008
:101888006FF0630C38F910E00CFB00390130BDF83B
:101898001C3038F91000CEEB000000FB09F999FB69
:1018A800FCF9CEEB090919FB03F9019BA7F8049091
:1018B800B079002BB8BF5B424343714893FBF0F00B
:1018C800643063786F4F4FF0640E434393FBFEF32D
:1018D800BB546D4FE37A434393FBFEF3BB54637DE4
:1018E800664F5843694B90FBFEF0022A9854684BA8
:1018F8000FD183F802E0049B53450FDB5E4CB4F82C
:101908009A21914216DBB1F5FA6FA8BF4FF4FA613C
:1019180011E003F802B0049B534504DA069B0698CD
:10192800FB5A5B423B520132032A04F101047FF463
:1019380046AFE3E71146891A4FF47A735943554B7A
:101948004E4E6FF0630CC2F5FA624FF0640EB1FBB5
:10195800F2F191FBFEF233F812000CFB0211013296
:1019680033F9122003B2D21A514391FBFEF3034418
:10197800FB80494B1B88580637D5484B484A1B887B
:101988001288DFED487A9FED480A9B1A1BB208EED1
:10199800103AB8EEC88A28EE278A38EE000A04F012
:1019A800C8F8F0EE408AB0EE480A04F0C2F8B6F97A
:1019B800023006EE903AB6F90030F8EEE66A07EE25
:1019C800903A20EE667AF8EEE77AA7EEA87A67EE04
:1019D800807ABDEEC77AE6EEA87A17EE103AFDEEE9
:1019E800E77A338017EE903A7380304E3368990760
:1019F80040F1AA802E4B2F491A684B6945F20720FF
:101A0800D31A8342884640F39F804A6103F0B8FDA9
:101A1800294BDFF8B8A01A78032A9946BAF800309B
:101A280056D10A2B60D90023282089F8003008F005
:101A3800C2FB03F0A5FD214B188803F08BFD204B5A
:101A48001A68D37890FBF3F0013008281D4BA8BF23
:101A580008201870537980B213FB00F3A8F81830E7
:101A6800137913FB00F0A8F81A003DE0E80C0020F9
:101A7800E8210020F40E0020CC1A00202E170020A8
:101A88000CFEFFFFD017002006030020D31700200C
:101A98003C1700206A0F00202C170020A40B002000
:101AA800C822002035FA8E3CDB0FC93F08220020EF
:101AB800D0220020F80200204C220020040E002032
:101AC800E80D002000010020820F0020900E002069
:101AD8000A2B09D80323A64A89F80030002313707B
:101AE800A8F81830A8F81A3099F80030A14A012B44
:101AF8000DD002D3022B1DD026E0B8F81820BAF872
:101B080000309A4220DD012389F8003010E0BAF84D
:101B18000010B8F81A308B4202DD0223137010E06F
:101B2800954B1B8B0133994202DD002313700BE0A8
:101B3800082007E0B8F81A30BAF8002001339A42B2
:101B4800E1DC072005F052FFD6F800B08B4E1BF4FD
:101B5800006F7ED08A4B88491A68CB69C3EB0209AB
:101B680045F207239945884673DD864BB7F9067019
:101B7800D3F800A0CA619AF80A30B4F85211012BC0
:101B88004FF47A72A7F57A7799FBF2F903D045D327
:101B9800022B23D045E07C4BD8F82000597B7B4BA7
:101BA80033F81110082789B290FBF7F3C01A4318CD
:101BB800A8F82410C8F8203040F6E44193FBF7F366
:101BC8009BB24B43BAF80810C1EB13335A43BAF926
:101BD800063092FBF3F2C8F8282022E03278BAF8EF
:101BE8000830C8F8283052071BD56948019305F01A
:101BF800CBFE019B18B91BF0100F18BF002707FB7D
:101C080007F2322192FBF1F21744BAF90620574342
:101C18004FF47A7297FBF2F73B4400E00023C8F8D0
:101C28002830D8E90C01D8F828305A4A03FB09F3C0
:101C38004FF47A7993FBF9F310EB030A41EBE37B5A
:101C4800C8E90CAB5046594600230AF007FEC8F80D
:101C58003800514B1A6812F4805F984602D00A2067
:101C680005F0C4FE4D4F3B68002B52D0DFF854E11D
:101C78004B4ADEF8000011688142F246914648D886
:101C8800484ADFF828B110785968D8B90123137089
:101C9800BBF800208A5C22B31846019308F0A4FA26
:101CA800414A019B13700AF0C5F8BBF80030C3B96C
:101CB8003B681B78053B012B13D808F055FA2E4BCF
:101CC800D8630EE000231370BBF800208A5C42B191
:101CD8001846019308F088FA334A019B13700AF0FA
:101CE800A9F83A68BBF8003052683048D25CFE2A3E
:101CF80001D100230CE0FF2A02D105F05FFE08E0C5
:101D0800DAF800700A2111FB0272C9F800200133C9
:101D1800038033785F0703D5254B10221A8561E0CD
:101D2800D8F80020D0075EBF144943F001030B70B8
:101D3800204B1B7819075EBF337823F001033370FB
:101D4800D30242BF337823F0010333701A4B1A8849
:101D5800154B1AB1194A1268970702D4184A128803
:101D680092B302221A70337823F00103337030E003
:101D7800000100204C220020F8020020ED22002063
:101D8800D0220020E80D0020EC0D0020FC0D0020E2
:101D9800561C0020407E0500740B00209C0F00207C
:101DA800940F0020900F002038220020980F002068
:101DB800000400489A0B0020AA0B002050220020A3
:101DC800E8220020C41A00203178C80758BF022230
:101DD8001A7008F0C9F9B44B1B68C01A002801DB57
:101DE8000AF028F8B14F3E78002E00F0D080B04BB2
:101DF8001A689846002A01F01C80D8F80000036889
:101E08005B689847002801F01480A94BA94C186812
:101E180003689B689847092801D03F2852D14FF0A2
:101E2800000A2668DFF8CC92554636B1A248D9F8A0
:101E3800001032460DF082F810B9CA4605B94D4671
:101E48009E4B09F110099945EFD3EDB1D5F800C0C3
:101E5800DAF8009023681CF803E019F803007045CD
:101E680012D15A1C944958B92D2B09D8DFF844E2ED
:101E7800CEF800204FF0200E01F803E0885403E06C
:101E880001F803E02260E5E723680BB1554510D05F
:101E98008B480AF0C5F8554507D855F8100B0AF0D5
:101EA800BFF809200AF0B4F8F5E786480AF0B8F850
:101EB800002623689E42A0D27F4B985D0AF0A8F8BE
:101EC8000136F6E72368002B40F09487042841F098
:101ED8006C84794804F028FB00F0ABBFD8F8000008
:101EE800DFF8F0B103685B689847002845D0DBF855
:101EF800000003689B689847D9F8003093F8482099
:101F08008246002A51D1242840F08880012283F893
:101F18004820D9F8002092F848000628DED192F827
:101F280049304B2B00F0DB8600F28781322B00F022
:101F3800088700F22181222B00F06C8500F2DC80FA
:101F4800032B00F01D8200F2A480012B40F090804A
:101F5800032009F0DDFF002009F0ADFF012009F0A2
:101F6800AAFF0D2009F0A7FF574F3B68987909F0A1
:101F7800A2FF3B68002283F84820544B93F81331A2
:101F8800002B40F025874C36982E00F05287504A97
:101F9800931993F84A100129F5D14B4FB2583B6079
:101FA8004C4BB9461A60984698E7012A04D14D2847
:101FB80014BF00220222AAE7022A04D13C2814BF37
:101FC80000220322A3E7032A0AD140284FF0000287
:101FD8009FBF1A71DA715871987198BF042296E7F9
:101FE800042A08D19A7983F8490080EA020A83F81A
:101FF80006A005228BE7052A8BD159791A799142D7
:10200800997906D941409971511C19711344187274
:102018007FE781420CBF0622002278E72E4B1A7810
:1020280052073FF576AF2328DBF8002013D11F496C
:102038000193012008701E4928480A602349C1F805
:10204800D82009F0EDFF1F4809F0EAFF019B1A7834
:1020580042F002021A70224B1B681B78534501BFDD
:10206800204B214A1A60214B04BF214ADA6050E70D
:10207800022B40F00187042009F04AFF432009F0B1
:102088001AFF4C2009F017FF462009F014FF4C20D6
:1020980068E7042B00F07F81052B40F0ED861A20BD
:1020A80009F036FF002787E13C220020EC220020BF
:1020B80048220020F00E0020C00E0020F40A01087B
:1020C800182101081D21010840220020F8020020E3
:1020D8003803002044220020ED2200204D21010871
:1020E800640F0020FC9F0020EFBEADDE00ED00E095
:1020F8000400FA0574090108282B00F0D68515D8C4
:10210800242B00F0B885262B40F0B686B64F062063
:1021180009F0FEFEB7F85C0109F0FDFEB7F85E01B4
:1021280009F0F9FEB7F8600100F022BE2A2B00F092
:10213800CF852C2B40F0A086AB4F0C2009F0E8FE91
:1021480097F8920109F0B7FEB7F89C0109F0E3FE91
:10215800B7F8980109F0DFFEB7F89A0109F0DBFE3D
:1021680097F8930109F0A7FEB7F89E0109F0D3FE8E
:10217800B7F8A00100F0FCBD3D2B00F01D8323D86B
:10218800382B00F07E8512D8342B00F06684362B6D
:1021980040F07286954B944F93F80E01C0EBC00047
:1021A800C0B209F0B5FE07F1200800F0F0BD3A2BE7
:1021B80000F0A8823B2B40F05F86012009F0A8FEC2
:1021C8008B4B1B681878CDE6452B00F0EE8527D899
:1021D800402B00F0BE85422B40F04E86824F1020E7
:1021E80009F096FE787909F066FEB86809F09CFE59
:1021F80097F8920109F05FFEB7F85C0109F08BFED1
:10220800B7F85E0109F087FEB7F8600109F083FEB0
:10221800B7F8820109F07FFEB7F8840100F0A8BD85
:10222800462B00F0B885492B40F02686022009F09D
:102238006FFE6D4B988900F09BBD702B00F0E88213
:1022480056D8682B00F0368224D8652B00F0E4803D
:1022580015D84D2B00F05285642B40F00D860720D1
:1022680009F056FEE72009F026FE5F4B587909F081
:1022780022FE002009F01FFE042000F0A5BD662BF9
:1022880000F08B81672B40F0F785102009F040FEA5
:102298000027A3E16D2B00F02F8213D8692B00F0E3
:1022A80015826C2B40F0E885524F062009F030FE6D
:1022B800388809F030FE788809F02DFE4E4B1888D2
:1022C80000F056BD6E2B00F021826F2B40F0D485B4
:1022D8004A4F0B2009F01CFE3B68187809F0EBFD0B
:1022E8003B68587809F0E7FD4FF00009B8466FE2FF
:1022F800782B00F07B811ED8742B00F0D7830BD885
:10230800722B00F04984732B40F0B685082009F041
:10231800FFFD012700F090BC752B00F06F83772B31
:1023280040F0AA85DFF8C48098F8DC0009F0F0FDD9
:10233800002700F027BCF02B00F0908414D87B2BEA
:1023480000F0F882A02B40F097850C2009F0E0FD02
:102358002B4B186809F0E8FD2A4B186809F0E4FDD2
:10236800294B186800F030BDF12B00F07D81FE2B61
:1023780040F08285082009F0CBFD002000F064BC05
:10238800184609F0C5FD012009F095FD0A2009F05D
:1023980092FD0020E6E5062009F0BAFD412009F08B
:1023A8008AFD572009F087FD462009F084FD332077
:1023B80009F081FD00F050BC144BD85D013709F0DD
:1023C8007AFD0B2FF8D10027114BD85D013709F0A2
:1023D80072FD082FF8D100270E4BD85D013709F0A0
:1023E8006AFD072FF8D1BFE5CC1A0020F8020020BB
:1023F800F40E00209A1A0020A40B0020E8210020E7
:10240800ACF7FF1FB0F7FF1FB4F7FF1F85210108C6
:10241800912101089A2101080B2009F079FDCF4B81
:10242800188809F078FDCE4B1A68CE4B9A420CBF3B
:10243800CD4BCE4B188880B209F06DFDCC4B1B6894
:10244800C3F3C000C3F38002800040EA4200C3F334
:1024580040021043C3F3401240EAC20003F01003E5
:10246800184309F058FDC34B1A88C34B12F0010FEB
:1024780014BF4FF002084FF0000812F0020F14BF0B
:102488004FF0040C4FF0000C12F0040F14BF4FF083
:10249800100E4FF0000E12F0400F14BF2027002737
:1024A80012F0100F14BF4FF40070002012F0200F2C
:1024B8001B6814BF4FF4806B4FF0000B12F4807F41
:1024C80014BF4FF400610021019102F0080903F4E0
:1024D800475141EA090903F4804149EA010903F433
:1024E800004149EA010903F4803149EA010903F48A
:1024F800003149EA010903F4802A49EA0A0903F488
:10250800002149EA010103F4801941EA090903F0AD
:10251800007349EA0303DFF8909299F80090C9F331
:10252800800943EA090343EA080343EA0C0C4CEA2E
:102538000E0E4EEA07073843019B12F4007F40EA6B
:102548000B0B4BEA030B14BF4FF4001100218B4B0C
:1025580012F4806F4BEA01014FF0000014BF4FF0F6
:10256800806B4FF0000B93F8DC7041EA0B010346D7
:10257800BB420CD2824A13F802E0012202FA0EFE94
:102588001EEA010F1CBF9A4010430133F0E709F01F
:10259800CBFC7C4B93F8C806E4E4122009F0B8FCA5
:1025A800794B1B88B3F5806F8CBF4FF008084FF04C
:1025B80001080027754B33F9170090FBF8F0013735
:1025C80080B209F0A8FC032FF4D1714F388809F0C4
:1025D800A2FC788809F09FFCB88835E36D4BD85D7C
:1025E800013709F068FC102FF8D1BDE4702009F01C
:1025F8008FFC4FF000082B680E2707FB08F73B44B9
:1026080008F10108B3F8190109F085FC2B683B446F
:10261800B3F81B0109F07FFC2B683B44B3F81D019C
:1026280009F079FC2B683B4493F81F0109F043FC3F
:102638002B683B4493F8200109F03DFC2B683B4490
:1026480093F8210109F037FC2B683B4493F82201E9
:1026580009F031FC2B681F44D7F8230109F064FC0A
:10266800B8F1080FC7D17FE47020464F09F050FC3D
:1026780007F1700897F8D40009F01DFC97F8D50009
:1026880009F019FC97F8D60009F015FC97F8D7005F
:1026980009F011FC97F8D80009F00DFC97F8D9005B
:1026A80009F009FC073797F8D30009F004FC4745FF
:1026B800E0D159E4102009F02BFC0027364BD85DF7
:1026C800013709F0F8FB102FF8D14DE4DFF8DC8072
:1026D80098F80000400000F0FE0009F019FC0027FF
:1026E80098F800309F42BFF43FAC2C4B33F81700EA
:1026F80009F011FC0137F3E709F00AFC002009F0A2
:1027080013FCA9E2042009F003FC5CE3072009F0AC
:10271800FFFB234B194F1888FF28A8BFFF20C0B222
:1027280009F0C9FBB86B4FF6FF784045A8BF404693
:1027380020EAE07080B209F0EEFB1A4B188809F025
:10274800EAFB104BB86A93F887318BB30A235843D6
:102758004045A8BF404620EAE0702BE064220020F4
:10276800901A0020005400406022002062220020BD
:10277800502200202C170020740B0020F8020020A3
:10278800D5030020CC1A002002000020F00300200E
:1027980036170020F6030020E0170020E80C002080
:1027A800900E0020780B0020ED220020C021002090
:1027B80000F30F0080B2DBE2D24F022009F0A8FB41
:1027C80097F8E20109F077FB97F8E101FFF7CABB38
:1027D800D8F80030CC4F4B4409F10109187909F0B9
:1027E8006AFBB9F1030FF3D13B68D87909F063FBB1
:1027F8003B68987809F05FFB3B68D87809F05BFB89
:102808003B68588909F087FB3B68187AFFF7AABB31
:10281800BE4F1E2009F07CFB3B681B78022B4FF053
:10282800000871D13B6803EB880393ED080AB2EE08
:10283800048A20EE080A0CF043FD80F30800C0B2B9
:1028480009F039FB3B68DFEDB27A03EB880393EDBF
:102858000B0A20EE270A0CF033FD80F30800C0B203
:1028680009F029FB3B68DFEDAB7A03EB880393EDB6
:102878000E0A20EE270A0CF023FD80F30800C0B2F0
:1028880008F1010809F017FBB8F1030FCAD1B8F134
:10289800070F3B6823D193ED110A20EE080A0CF0CC
:1028A8000FFD80F30800C0B209F005FB3B6893ED0B
:1028B800120A20EE080A0CF003FD80F30800C0B2EB
:1028C80009F0F9FA3B6893F84C3000EE103AB8EE8C
:1028D800400A0CF0F5FC80F30800C0B20BE043445A
:1028E800587809F0E8FA3B684344D87A09F0E3FAE3
:1028F8003B684344587D08F1010809F0DCFAB8F157
:102908000A0FC4D1FFF730BB3B684344587809F03D
:10291800D2FA3B684344D87A09F0CDFA3B6843447D
:1029280008F10108587D09F0C6FAB8F10A0FEBD191
:10293800FFF71ABB3C2009F0EBFA0027DFF8CC813F
:102948009FED748AD8F8003003EB870393ED080AEB
:1029580020EE080A0CF0B4FC80B209F0DCFAD8F8D2
:10296800003003EB870393ED0B0A20EE080A0CF006
:10297800A7FC80B209F0CFFAD8F8003003EB870340
:1029880093ED0E0A20EE080A0CF09AFC013780B28B
:1029980009F0C1FA032FD1D1072FD8F8003018D188
:1029A80093ED110A20EE080A0CF08AFC80B209F0B7
:1029B800B2FAD8F8003093ED120A20EE080A0CF0AB
:1029C8007FFC80B209F0A7FAD8F8003093F84C00E1
:1029D8000DE03B44587809F09EFAD8F800303B44A3
:1029E800D87A09F098FAD8F800303B44587D013776
:1029F80009F091FA0A2FCFD1FFF7B6BA2F2009F0C4
:102A080087FA454F17F8010F00283FF4ADAA09F0DF
:102A180052FAF7E7502009F07BFA00273B4B1B6876
:102A280003EB87083D4B98F879200C2101FB023312
:102A3800013793F8380009F03EFA98F87A0009F05F
:102A48003AFA98F87B0009F036FA98F87C0009F011
:102A580032FA142FE2D1FFF787BA482009F058FA62
:102A68004FF00008294B1F68062303FB087708F17D
:102A7800010897F8CE0009F01EFA97F8C90009F086
:102A88001AFA97F8CA0009F016FA97F8CB0009F075
:102A980012FA97F8CC0009F00EFA97F8CD0009F071
:102AA8000AFAB8F10C0FDDD1FFF75EBA4FF0000853
:102AB8004FF001094FF0000A194B93F8DC209245BA
:102AC80042DADD334FF0000B1AF80320134F0C23C2
:102AD80007F1300103FB0BF3595C914209D13B44E8
:102AE800586B0CF022FA0246B9F1000F07D14B4699
:102AF80018E00BF1010BBBF11C0FE7D121E080447A
:102B08001FE000BFCC1A0020E8210020F40E0020AE
:102B18000000C84200007A44B7070108B807010856
:102B2800F802002093420CDA0C2101FB0B7104928D
:102B3800496B0193C85C09F0BEF9019B049A013303
:102B4800F0E70AF1010AB7E7B9F1000F3FF40CAA60
:102B58005FFA88F009F0DCF94FF00009AAE70131C3
:102B68001C290ED0CC480C2200F1300C02FB01F3DA
:102B780013F80C207245F2D1034493F8380009F099
:102B88009AF9013798F8DC309F42BFF4EDA9C34B9E
:102B9800002117F803E0E5E7162009F0B9F9029BD0
:102BA800B3F8980109F0B7F9029BB3F8440109F0AA
:102BB800B2F9029BB3F8460109F0ADF9029BB3F8EC
:102BC800480109F0A8F9029BB3F8DA0109F0A3F962
:102BD800002009F070F9002009F06DF9002009F0D3
:102BE8006AF9029B93F8870109F065F9029B93F84B
:102BF800940109F060F9002009F05DF9A84B1B6801
:102C08000A20B3F9563093FBF0F080B209F083F94B
:102C1800029B93F87C0109F04EF9029B93F880011E
:102C280009F049F9029B93F87F0109F044F9029BE6
:102C380093F88101FFF796B9F8B2013709F03BF92B
:102C4800092FF9D1FFF790B909F065F9002009F0CB
:102C580062F9002009F05FF9002089E0904F042014
:102C680009F056F93B68B3F85A0009F054F93B6883
:102C7800B3F858007CE0042009F04AF9894B9868B9
:102C8800A2E0884F042009F043F997F87C0109F085
:102C980012F997F8800109F00EF997F87F0109F009
:102CA8000AF997F88101FFF75DB97E4F072009F00F
:102CB8002FF9B7F8820109F02EF9B7F8840109F065
:102CC8002AF997F8860109F0F6F8B7F888014FE075
:102CD800012009F01DF9734B5879FFF743B9714F7B
:102CE800042009F015F997F8D80109F0E4F897F8E5
:102CF800D90109F0E0F8B7F8DA0139E06A4FDFF8EE
:102D0800D081387800EB4000C0B209F001F94FF0EB
:102D180000093B78994508F10208BFF425A918F87D
:102D2800020C09F0C8F818F8010C00EB800000EB61
:102D3800800000F2EE2080B209F0EDF809F10109F7
:102D4800E7E7012009F0E4F8564B93F89401FFF700
:102D580009B9082009F0DCF80027524B3B44013739
:102D680093F88A0109F0A7F8082FF6D1FFF7FCB805
:102D780009F0D1F8FFF7F8B84C4AD25C904264D019
:102D88000C33302BF8D1083747453FF4EDA897F8B6
:102D9800F2010023F0E70D2009F0BAF8002009F04D
:102DA8008AF8002009F0C0F80AE0132009F0B0F80A
:102DB80000273F4BD85D013709F07DF80B2FF8D17C
:102DC800002009F0B1F8002009F0AEF8FFF7CCB800
:102DD800384BF05807F00EFA18B9322007F0EBF923
:102DE800F6E707F069FB02F0D7FF334B334ADA60A6
:102DF800FFF7C9B80C2800F0DA840A2840F0DB8411
:102E08002F4D304809F00CF9284623210CF07FF8A3
:102E180008B1401B20602368002B40F0D08428486C
:102E28002360002130220CF03CF83B78002B40F066
:102E3800FB84254B9B68002B00F01D85234809B0B7
:102E4800BDEC028BBDE8F04F184709F034F8B7F82D
:102E5800F40109F060F897F8F60109F02CF897F8F2
:102E6800F70109F028F897F8F90109F024F897F81C
:102E7800F80109F020F886E74C2B3BD108F0FEFF5B
:102E8800084F87F8D80108F0F9FF87F8D90108F04A
:102E9800FFFFA7F8DA0128E0B8070108D5030020EA
:102EA800F40E0020CC1A0020C02100202C0F002096
:102EB800852101083803002000ED00E00400FA0530
:102EC800C00E0020F12C0108F01000200C04002096
:102ED8006E1C0020D42B00F05183D22B40F061846B
:102EE800CA4B1B785B0740F19083002009F010F86B
:102EF800FFF73AB800F27B81352B27D108F0BEFFE7
:102F08000B28804602D908F00FFEEEE7C04B1F6879
:102F180008F0B4FF0328F6D8062303FB087787F8E0
:102F2800CE0008F0ABFF87F8C90008F0A7FF87F8C4
:102F3800CA0008F0A3FF87F8CB0008F09FFF87F8C6
:102F4800CC0008F09BFF87F8CD00CEE700F2A58003
:102F5800292B11D108F09CFFAE4FA7F8820108F089
:102F680097FFA7F8840108F089FF87F8860108F021
:102F78008FFFA7F88801B8E759D8252B07D1A54BAB
:102F880000229A6008F08EFF02F0FEFEADE7272BC4
:102F98000DD108F07DFF9F4FA7F85C0108F078FF7E
:102FA800A7F85E0108F074FFA7F860019DE7232BDE
:102FB80040F0F78308F062FF13288146A3D8DFF8B2
:102FC8005082D8F8007008F059FF002292490C236B
:102FD800534301EB030E9EF838E0864523D10B449A
:102FE8000FFA89F907EB890793F8303087F87930B9
:102FF80008F044FF87F87A0008F040FF87F87B0064
:1030080008F03CFF854B864A1A6087F87C00854BA0
:10301800D8F800001860793008F0F6FC824B80F090
:103028000100187061E701321C2ACFD16BE72D2B04
:1030380023D108F023FFDFF8DC8188F8920108F03B
:1030480027FFA8F89C0108F023FFA8F8980108F0CA
:103058001FFFA8F89A0108F011FF3B6888F8930150
:103068005B79082B7FF641AF08F012FFA8F89E01A4
:1030780008F00EFFA8F8A00137E7332B05D108F0B8
:10308800FDFE644B83F894012FE72B2B40F08983D6
:1030980008F0F4FE5F4B587127E73E2B09D108F082
:1030A800EDFE5C4F87F8E20108F0E8FE87F8E101E1
:1030B8001BE759D8392B11D108F0E0FE554F87F896
:1030C8007C0108F0DBFE87F8800108F0D7FE87F85E
:1030D8007F0108F0D3FE87F8810106E73C2B0BD16E
:1030E8004B4FD7F8008008F0C9FE88F800003B680D
:1030F800187807F0C1FAF8E6372B40F05283537975
:103108000727B3FBF7F2C2EBC2029A1A12F0FF0FBD
:103118007FF4F9AEB3FBF7F7013FFFB2FF2F3FF49F
:10312800E4AE08F0ABFE5FFA80F94FFA89F004F0DC
:10313800C5FA804600283FF4E6AE80F8009008F013
:10314800A7FEA8F8020008F099FE88F8040008F025
:1031580095FE88F8050008F091FE88F8070008F049
:103168008DFE88F80600D7E7432B22D108F086FEAB
:10317800284F0023BB60787108F094FE02F004FE2B
:1031880008F07CFE87F8920108F082FEA7F85C013F
:1031980008F07EFEA7F85E0108F07AFEA7F8600145
:1031A80008F076FEA7F8820108F072FEA7F88401FD
:1031B8009BE60DD8412B40F0F482002708F05EFE14
:1031C800144B3B440137082F83F88A01F6D18CE66B
:1031D800442B04D1154B012283F8132185E64A2B91
:1031E80040F0DF8208F054FE0A4B98817DE6D02B30
:1031F8001ED1064B1B7858073FF577AE04F032FE18
:1032080002F0F4FD02F0B0FE6FE600BFED220020F0
:10321800F40E0020CC1A0020B8070108E40B0020A7
:10322800101C0020E80B002014000020F8020020E9
:1032380000F28E81CC2B50D15379092B7FF663AEE7
:10324800039BD3F8008008F019FE039B88F8000060
:10325800D3F8008008F012FE88F8010008F00EFE8E
:10326800039B64281B68A8BF6420187108F006FE39
:10327800039B64281B68A8BF6420587108F0FEFDF2
:10328800039BFF281B68A8BFFF20987108F0F6FD74
:10329800039B6428D3F8008028BF642088F80700BF
:1032A80008F0ECFD039B88F80200D3F8008008F0D2
:1032B800E5FD039B88F80300D3F8008008F0E8FDDB
:1032C8003B68A8F80A005B790A2B7FF60EAEDC4B48
:1032D8001F6808F0D3FD387207E600F2DC80C82BBF
:1032E80015D157797F08122F3FF60DAE4FF0000821
:1032F800B84507D208F0CCFDD24B23F8180008F1E6
:103308000108F5E7D04B012283F81221EDE5CA2B1D
:1033180040F09280CD4F3B681B78022B4FF000089D
:103328006FD1D7F8009008F0A9FD07EE900AF8EEE3
:10333800677AB2EE048AC7EE887A09EB8809C9ED84
:10334800087AD7F8009008F099FD07EE900A9FEDEB
:10335800C07AF8EE677A09EB8809C7EE877AC9ED73
:103368000B7AD7F8009008F089FD07EE900A9FEDD8
:10337800B97AF8EE677A09EB8809C7EE877A08F117
:103388000108B8F1030FC9ED0E7ACAD1B8F1070FD9
:10339800D7F800901CD108F071FD07EE900AF8EEFE
:1033A800677AC7EE887AC9ED117AD7F8009008F0E5
:1033B80065FD07EE900AF8EE677AC7EE887AC9EDE0
:1033C800127AD7F8009008F059FD89F84C0012E0FD
:1033D80008F054FDC14489F80100D7F8009008F0BE
:1033E8004DFDC14489F80B00D7F8009008F046FD60
:1033F800C14489F8150008F10108B8F10A0FC5D1D0
:1034080073E5D7F8009008F039FDC14489F8010048
:10341800D7F8009008F032FDC14489F80B00D7F8BE
:10342800009008F02BFDC14408F10108B8F10A0F1B
:1034380089F81500E5D158E54E2B40F0B28157794F
:103448000323B7FBF3F7122F3FF65DADDFF81082C9
:103458004FF00009B945BFF448AD08F00FFD88F8F2
:10346800A20108F015FD40F2ED23984205DD40F673
:10347800CA039842A8BF184601E040F2EE20A0F225
:10348800EE20192309F1010990FBF3F008F1020875
:1034980088F8A101DEE7CE2B0AD16F4B1B785A07BB
:1034A8003FF523AD6D4A137843F0040313701CE510
:1034B80044D908F0EDFC6FF4AF67C3199BB2C62B73
:1034C8009CBF674BA3F8980108F0E2FCA4F84401FC
:1034D80008F0DEFCA4F8460108F0DAFCA4F848017C
:1034E80008F0D6FCA4F8DA0108F0C8FC08F0C6FC1D
:1034F80008F0C4FC08F0C2FC84F8870108F0BEFCA0
:1035080084F8940108F0BAFC504B1F6808F0C0FC1E
:1035180000EB80004000A7F8560008F0AFFC84F8E4
:103528007C0108F0ABFC84F8800108F0A7FC84F863
:103538007F0108F0A3FC84F88101D6E4464B1B7890
:1035480059073FF5D2AC474B4FF4C8721A80CCE408
:10355800D62B09D1002708F09BFC434B23F8170012
:103568000137082FF7D1C0E45BD8D32B7FF4B2AC76
:1035780008F08EFC344BA3F81001B6E453790F2BF6
:103588007FF4C1AC08F07AFC072807463FF6BBACCD
:10359800DFF8B880D8F8009008F07AFC0E235F4373
:1035A800B944A9F81901D8F8009008F071FCB94499
:1035B800A9F81B01D8F8009008F06AFCB944A9F8EA
:1035C8001D01D8F8009008F059FCB94489F81F018A
:1035D800D8F8009008F052FCB94489F82001D8F8CE
:1035E800009008F04BFCB94489F82101D8F8009004
:1035F80008F044FCB944D8F8008089F8220108F0A2
:1036080051FC4744C7F823016FE408F037FC144B1A
:10361800022883F8C8067FF6F3AD002283F8C8268F
:10362800EEE5EF2B22D1094FD7F8008008F030FCE7
:10363800A8F85A003F6808F02BFCA7F8580054E493
:10364800E8210020E80C0020F8020020F40E0020F9
:103658000000C84200007A44ED2200209A0B0020A6
:10366800CC1A0020AA0B0020EC2100206DD8D82B02
:1036780040F097800027DFF834829FED818AD8F8E0
:10368800009008F005FC07EE900AF8EE677A09EB5F
:103698008709C7EE887AC9ED087AD8F8009008F04B
:1036A800F7FB07EE900AF8EE677A09EB8709C7EE91
:1036B800887AC9ED0B7AD8F8009008F0E9FB07EE94
:1036C800900AF8EE677A09EB8709C7EE887A01371E
:1036D800032FC9ED0E7ACED1072FD8F800901CD150
:1036E80008F0D6FB07EE900AF8EE677AC7EE887AFC
:1036F800C9ED117AD8F8009008F0CAFB07EE900AD5
:10370800F8EE677AC7EE887AC9ED127AD8F8009091
:1037180008F0BEFB89F84C0012E008F0B9FBB94488
:1037280089F80100D8F8009008F0B2FBB94489F88C
:103738000B00D8F8009008F0ABFBB94489F81500E5
:1037480001370A2FC8D1FFF7D0BBF22B22D108F0DE
:1037580095FB0F2807463FF6D6AB08F08FFB494B81
:10376800C7EBC7071F44387108F088FB787108F069
:1037780085FBB87108F082FBF87108F07FFB38729E
:1037880008F07CFB787208F079FBB87206F0D4FE7A
:10379800FFF7ABBBFA2B04D13B4B1B785B077FF5DC
:1037A8002FAD08F0C1F9FEF7DFBB0C284AD1374826
:1037B80008F036FC38E00D2838D1FFF721BB5A1E37
:1037C800A95C202902D11346FFF726BB304A2360A3
:1037D8000021D1542F4B304DD3F800A0D5F800B0BC
:1037E800DFF8AC9058460BF0A0FB06463246484638
:1037F80059460BF0A3FB294A28B919F80630534457
:103808005B78590703D010359542E7D306E0954217
:1038180004D2701CEB684844984702E0204808F03E
:10382800FFFB0023FFF7FBBA1E4807E07F280DD1F6
:10383800013B174A1C4823600021D15408F0F0FBD3
:10384800FEF7DBBA7F2804D1FEF7D7BA2F2B3EF656
:10385800D4AAA0F12002D2B25E2A3EF6CEAA13B9AB
:1038680020283EF4CAAA5A1C2260094AD05408F0FB
:10387800CFFBFEF7C2BA09B0BDEC028BBDE8F08FF2
:1038880000007A449C1B0020ED2200202221010820
:10389800C00E00200401002074090108F40A010880
:1038A8002D2101081D21010849210108F40E0020DD
:1038B8009B4A2DE9F04F15689A4C05F59C43203337
:1038C8002360994B196889B011F4804F05929B4683
:1038D80005D108F0A3FA10B9237901332371934B6A
:1038E8001F78C7B1924A1268954240F2E080013FC2
:1038F8001F70DCE0D8F800308E48072D98BF595D5E
:103908008D4B88BF29461B689847032D0BD904EBBC
:1039180045050137E880874BDFF834821E78FDB211
:10392800AE42E7D820E0D8F8002005F10E0302EBFC
:1039380083039988DA880028E9D04FF47A73401A0B
:103948005843531A90FBF3F040F6C90300F57A7018
:10395800984205DC40F2EE239842B8BF184601E0D1
:1039680040F6CA0080B2D2E70F23277984F82A30BC
:1039780094F82B300193032594F82C30B7FBF5F518
:1039880005EB45057D1B0393D8F800300293DFF85B
:10399800CC91EBB204930025B54254DA6749019BF8
:1039A80031F815A04FEA450853B908F037FA28B19D
:1039B800039B002B08BF4FF0000A01E0DDF804A0CC
:1039C800029B988A504502D8D88A50450ED2E8B250
:1039D80008F0D6F9032D8246DFBF94F82AE00120CB
:1039E800A8402EEA0000D8BF84F82A0008F016FA8A
:1039F80018B1534828F800A021E0049B94F87600F9
:103A080029F813A028B9022F15D94649012081F8B1
:103A18007600B9F80210B9F800000844B9F80410A3
:103A28000844484980B228F8010000B2032190FBFD
:103A3800F1F080B200E05046414928F80100013514
:103A480009F10609A8E794F82A203F483F4BA2F15C
:103A58000F014A424A4184F8902072B1314AD2F8A3
:103A68009420520109D40268D9689A60521AC82A67
:103A78001DD9012283F8212019E002689868DA60CC
:103A88005B68121A9A4288BF304B4FF0000184F8E5
:103A98002B1088BF83F821100025B54207DAE8B259
:103AA80008F06EF9264B23F815000135F5E7DBF829
:103AB8000030DF0405D5D4F89430DE0701D408F0CF
:103AC800A5FE059B1968224B1F68BB7A002B47D0BF
:103AD800013B1B483A7B30F813301AB1C3F53B63FE
:103AE80008339BB21BB2A3F57A73B3F57A7FA8BFEC
:103AF8004FF47A7323EAE37307EE903A9FED157A51
:103B0800F8EEE77AC7EE877A9FED137A67EE877A41
:103B1800FCEEE77A17EE903AA4F8983067E000BF19
:103B2800D0220020E00A00200822002010220020D5
:103B38000C220020C021002074000020E60A00208A
:103B4800E80C0020580B0020C41A00201422002082
:103B58000422002000007A4400C07F440E0B00209D
:103B6800DBF80020150442D5D4F89C208E4E8A1A22
:103B7800002A3CDB01F59C422032C6F89C208B4A87
:103B880050798B4A32F81050A8B2FD7A90FBF5F5BF
:103B980096F8A000013000F00F0286F8A020324409
:103BA80082F8A1501A46804800F1A1055D5D0133F5
:103BB8002A44102B92B2F6D112B292FBF3F31BB245
:103BC800642BA8BF642323EAE37307EE903A9FEDC2
:103BD800797AF8EEE77AC7EE877A9FED777A67EE1B
:103BE800877AFCEEE77A17EE903AA0F89830DBF87F
:103BF8000030724E13F4807F00F0F780704B714DE7
:103C0800994203D9AB780BB90123AB70AB78002B81
:103C180000F0EB806B4B96F8008093F82170D4F895
:103C28009430781E47424741002FC8F38008C3F3F9
:103C3800806914BF4FF0000A4FF0030A95F820304E
:103C4800052B00F2CC80DFE803F0034C5175829C11
:103C5800B8F1000F38D0D4F8B400B4F8B81003F0B5
:103C680093FE012808D1584A584B12681B68D2881D
:103C7800642101FB02332B61B9F1000F0CD0524BC8
:103C88001B681B7943B105F0AFFB032385F820308F
:103C98004FF47A73EB61D1E7002F40F0A0804B4BD3
:103CA80048491A682B699A420AD9019105F09CFB88
:103CB8000199032381F8203040F6B833CB61BDE782
:103CC800012381F82030B9E74FF48060B9F1000F83
:103CD80002D002F041F801E002F02DF800232B6138
:103CE8007DE0002F44D105F07FFBA7E727B105232E
:103CF80085F82030012100E03946B8F1000F0CD0DA
:103D0800D4F8B430DA89324B1A805A809A802E4A15
:103D180012685288DA804FF0020A2C4B1A686B69D5
:103D28009A4202D8B8F1000F56D147F23053EB61EE
:103D380003231EE0337843F00203337008F066FD76
:103D4800224BEA691B681344AB61042311E01F4B43
:103D580097B11A68AB699A4241D91E4B1B781BB9B7
:103D6800D4F89430D9073AD4337823F00203337067
:103D7800052385F8203061E71B68EA691344AB61C5
:103D88002DE0114A114B12681B68D288642101FB8F
:103D980002332B614FF48060002385F82030EB70EC
:103DA80001F0C9FF4AE700BFE00A0020EC0D00203F
:103DB800FC0D00200000C84200C07F44ED22002016
:103DC800404B4C001422002028110020C41A002067
:103DD800E80C00201400002000297FF42FAFBAF16E
:103DE800000F02D0504603F001FEA84D05F5C5703E
:103DF800B5F8521103F0C8FD074650B905F0E6FAC8
:103E0800A34B1F605F609F60A24B00221A605A603C
:103E18009A6033785A0738D5DBF80030DB0634D59A
:103E280094F8BA30DFF87882D8062ED49A4B1B78EB
:103E380033B395F8E2318FB95BB1984B1A68D8F86B
:103E4800BC309B1A002B04DA08F0E0FC88F8C0703C
:103E58001BE0102003F0CAFD01230EE03BB18F4A9E
:103E680012684FF47A7101FB0323C8F8BC3094F848
:103E7800C03053B103F0A2FD002384F8C03004E041
:103E8800002FE6D098F8C030F3E7002295F8E091CB
:103E980095F8E101B5F89AE1B5F89CC11346DFF849
:103EA800148238F912109B087145C4BF63F07F0370
:103EB800DBB201326145B8BF43F04003042AEED1BA
:103EC80094F8C12076499A4205D191F8C220F92A7E
:103ED80004D8013200E0002281F8C22084F8C13001
:103EE8006D4B6F4A19789A46C9B9D2F89430D907F8
:103EF80006D5A7B93378DA0711D508F051FC0EE0DA
:103F080033785B070BD592F82B3043B1654BDB78E0
:103F18002BB910B108F07AFC01E0002FFAD094F820
:103F2800C2305F4A604F142B40F083809AF800300B
:103F380019F1000918BF4FF001096BB392F8C130AD
:103F48005F2B11D1337803F0040303F0FF0113B1A1
:103F580008F05CFC08E00B200291019203F046FD9A
:103F6800019A029982F8C210B9F1000F14D094F89E
:103F7800C1307D2B10D1337803F0040303F0FF0226
:103F880013B108F043FC07E00B20019203F02EFD6B
:103F9800434B019A83F8C220337803F0040303F0FB
:103FA800FF01002B45D194F8C1303D4A572B0BD166
:103FB8003E4B4FF47A7119803D4B1B6813F0080390
:103FC80037D1A2F8C43034E0DBF80000400717D539
:103FD8005A2B15D192F8C6302BB1012382F8C6109E
:103FE80082F8C73025E092F8C83083F0010382F8E0
:103FF800C8300BB10C2000E00D2003F0F7FC18E0EE
:104008005D2B00F004845B2B00F003845E2B00F032
:104018000284562B01D102F039F99AF80030002BAE
:1040280000F0C98394F8C1306F2B40F0BE8308F0CC
:10403800B7FBDBF8003058074CD594F8C830184A5D
:1040480093B1337859070FD5B8F90610B5F89A31F6
:10405800994209DDD2F8943013F0010302BF3221EE
:10406800A2F8CC1082F8C830D4F894200C4BD203B4
:1040780022D593F8CE202AB993F8C62012B9322255
:10408800A3F8CC20012384F8CE3023E0CC1A0020FA
:104098005C170020BC17002014000020C41A002060
:1040A800E00A002014220020F40E0020E82200205C
:1040B80050220020E80C002093F8C62052B1327834
:1040C80002F0040202F0FF0122B9012283F8C610AF
:1040D80083F8C7203F680023C4F8943007F17B06B3
:1040E80007F1CB093278737816F8010C9A420DD291
:1040F800314603F023FC48B116F8022C012303FAD9
:1041080002F2D4F894301343C4F8943004364E4580
:10411800E8D1C34B1B783BB1D4F89430C14F13F0AE
:10412800020F40F0FB82F2E207F1CA0607F5897731
:104138003278737816F8010C9A4225D2314603F08A
:10414800FDFB08B3B37896F804E0B74A96F80390F5
:10415800B6480C21013B01FB0E4103EB430313441A
:10416800D1F8D4209A420FD0C1F8D430002390F867
:104178000021C1F8D830012303FA0EF322EA030321
:1041880081F8D09080F800310636BE42D0D1A849D7
:10419800A84B0A680192D3F8009094F82B20A64FF8
:1041A8000292002603933868002800F0A98201785B
:1041B800002900F0A5827B68019AD31A002B0ADB3C
:1041C80002F5FA7394F800E17B600123B3402EEA0C
:1041D800030384F80031029B002B00F0918217F84A
:1041E800043C42780433DBB2002A40F04F8238F9AD
:1041F80013E0B5F8983103F1C80CE64502DD90F8F4
:1042080002A013E0C83B9E4503DA8378C3F1000A95
:104218000CE094F800110123B34021EA030384F869
:104228000031019B03F5FA737B6069E294F80001A1
:104238003041C30700F16482BAF1000FCCBF0220FD
:104248000120049103F0F8FB0499784A481E1328CA
:1042580000F24F82DFE810F0140020002F00400029
:1042680059006200C10030018F01BE01EB014D020F
:1042780040004D006200C10030019200030160015E
:1042880099F8001001EB0A03FA2BA8BFFA2323EAD6
:10429800E37389F800300AE099F8011001EB0A038A
:1042A800642BA8BF642323EAE37389F801304846E6
:1042B80003F02AFB1DE299F8031001EB0A03642BB3
:1042C800A8BF642323EAE37389F803304846D2F889
:1042D800041103F0CFFA0CE299F805005044642861
:1042E800A8BF642020EAE0700D2989F8050000F0D5
:1042F800008299F8041001EB0A03642BA8BF642319
:1043080023EAE37389F80430F3E199F8061001EB26
:104318000A0383F3080389F80630EAE1D2F8083182
:10432800187802281FD107EE90AAF8EEE77AB2EEC5
:10433800047AC7EE877A93ED097A77EE877AF5EEF5
:10434800C07AF1EE10FA09D49FED3D7AF4EE477A7F
:10435800F1EE10FAC8BFF0EE477A01E0DFED397AE6
:10436800C3ED097A07E098785044C828A8BFC82048
:1043780020EAE07098700F2900F0BB81D2F808019C
:10438800017802291FD107EE90AAF8EEE77AB2EE7B
:10439800047AC7EE877A90ED087A77EE877AF5EE99
:1043A800C07AF1EE10FA09D49FED257AF4EE477A37
:1043B800F1EE10FAC8BFF0EE477A01E0DFED217A9E
:1043C800C0ED087A95E1417801EB0A03C82BA8BF34
:1043D800C82323EAE37343708BE1D2F808311878D5
:1043E800022831D107EE90AA9FED157AD3ED0C6A19
:1043F800F8EEE77AC7EE877A77EEA67AF5EEC07A16
:10440800F1EE10FA07D4F4EE477AF1EE10FAC8BFCD
:10441800F0EE477A01E0DFED0B7AC3ED0C7A1BE092
:10442800EC2200202C17002038090108E00A00209F
:10443800C41A0020E8210020B40B002000007A44B0
:104448000000C84200000000187B5044C828A8BFDC
:10445800C82020EAE0701873102900F04A81D2F8C9
:104468000801017802291DD107EE90AA1FED0C7AE8
:10447800D0ED0B6AF8EEE77AC7EE877A77EEA67A80
:10448800F5EEC07AF1EE10FA07D4F4EE477AF1EEC1
:1044980010FAC8BFF0EE477A01E05FED167AC0ED7A
:1044A8000B7A26E1C17A01EB0A03C82BA8BFC823FF
:1044B80023EAE373C3721CE1D2F8083118780228A2
:1044C8001FD107EE90AA1FED237AF8EEE77AC7EE20
:1044D800877A93ED0F7A77EE877AF5EEC07AF1EE68
:1044E80010FA09D41FED2A7AF4EE477AF1EE10FAA1
:1044F800C8BFF0EE477A01E05FED2E7AC3ED0F7A80
:1045080007E0987D5044C828A8BFC82020EAE0707A
:104518009875112900F0ED80D2F808010178022978
:104528001FD107EE90AA1FED3B7AF8EEE77AC7EEA7
:10453800877A90ED0E7A77EE877AF5EEC07AF1EE0B
:1045480010FA09D41FED427AF4EE477AF1EE10FA28
:10455800C8BFF0EE477A01E05FED467AC0ED0E7A0B
:10456800C7E0417D01EB0A03C82BA8BFC82323EA93
:10457800E3734375BDE0D2F80801017802291FD121
:1045880007EE90AAF8EEE77AB2EE047AC7EE877AD9
:1045980090ED0A7A77EE877AF5EEC07AF1EE10FAA6
:1045A80009D41FED597AF4EE477AF1EE10FAC8BF34
:1045B800F0EE477A01E05FED5D7AC0ED0A7A98E0A7
:1045C800C17801EB0A03C82BA8BFC82323EAE37309
:1045D800C3708EE0D2F80801017802291DD107EED8
:1045E80090AA1FED697AD0ED0D6AF8EEE77AC7EE6A
:1045F800877A77EEA67AF5EEC07AF1EE10FA07D44C
:10460800F4EE477AF1EE10FAC8BFF0EE477A01E00F
:104618005FED747AC0ED0D7A6BE0417B01EB0A0324
:10462800C82BA8BFC82323EAE373437361E0D2F819
:104638000811087802281FD107EE90AA1FED817A89
:10464800F8EEE77AC7EE877A91ED107A77EE877AF7
:10465800F5EEC07AF1EE10FA09D41FED877AF4EE80
:10466800477AF1EE10FAC8BFF0EE477A01E05FED45
:104678008B7AC1ED107A3CE0C87D00EB0A03C82BA9
:10468800A8BFC82323EAE373CB7532E0012A30D1EF
:1046980090F802E038F91300B0F5617F05DB40F6C9
:1046A80033039842A8BF184601E04FF461700C2903
:1046B8001FD16D4A4FF4966393FBFEFE1378A0F565
:1046C800617090FBFEF0C0B2834212D0042834BF60
:1046D80003460223137001FB0351039B049001F26C
:1046E800CA61196001F01CFC04980130C0B203F0E3
:1046F800A3F994F800110123B3400B4384F8003167
:104708000136042E07F10C077FF44DAD04E5DBF804
:104718000030DE0510D5554BDB786BB1544B1B6868
:10472800980709D53B8813F001060AD104F04EFE1C
:10473800012001F011FB04E0012001F0FCFA012343
:1047480000E00023D4F8942051070CD55BB1012078
:1047580001F0F1FA3B889A0708D404F037FE0220EA
:1047680001F0FAFA02E0022001F0E5FA3B8813F0C2
:10477800030F404B4FF020020CBF9A611A85D4F802
:1047880094301B054FF4807002D501F0E5FA01E082
:1047980001F0D1FA6B79082B01D00E2B61D14020A2
:1047A80009B0BDE8F04F01F0C6BAB9F1000F02D068
:1047B8007E2B3FF43CAC94F8C1302F4A972B04D1A0
:1047C8004FF4C873A2F8CA3033E4A72B06D192F885
:1047D800BA3043F0040382F8BA302AE40022BB2B33
:1047E800079201D1022303E0B72B04D14FF6FE73E1
:1047F800ADF81E301FE0BE2B01D1022304E0BD2B13
:104808007FF417AC4FF6FE73ADF81C3013E00120AF
:1048180002E0022000E003205FFA80F909F1FF338B
:1048280085F8C83601F0E2FA01F09EFB484603F02D
:1048380003F9FFF7FEBB3B68BDF81C10B3F858201E
:104848000A44A3F85820BDF81E10B3F85A200A44A9
:10485800A3F85A2001F01AFD002384F8C230FFF7AC
:10486800E8BB09B0BDE8F08FE42100201422002045
:104878005022002000040048E00A002010B5214A18
:1048880018B9136802221A8210BD1F481468002341
:104898000380217811F07F0102460DD1637A9906D1
:1048A80044BF0221017013F0400F037814BF43F096
:1048B800010323F0010315E0012921D002291ED1AB
:1048C800637913F0800F03F00F034FEA830303F1BA
:1048D800804303F5B8431B6806D003F03003102B60
:1048E80007D10123137004E003F44053B3F5805F4C
:1048F800F6E7064B1B681B699847034810BD184626
:1049080010BD00BF881A0020F00B0020781A002084
:1049180010B5064C18B9236801221A8210BD044B41
:104928001B689B68984720680C3010BD881A0020C7
:10493800781A002010B5064C18B9236801221A828B
:1049480010BD044B1B681B68984720680A3010BDCF
:10495800881A0020781A002003788B4283BF034B03
:1049680003EB410148880020704700BFF00B00208E
:1049780070B500221346244914180C44A47E83EA17
:104988000423082413F4004F4FEA430318BF83F4A9
:10499800815304F1FF3418BF83F0010314F0FF04BE
:1049A8009BB2EFD10132192AE5D100F1190200F1C9
:1049B8001A050A440D44967EAA7E02EB062292B29C
:1049C8009A421FD1104B93F83B50E2B2AA4216D23A
:1049D800431C03EB4203DBB2CA1801330B44927E3B
:1049E8009B7E03EB02239BB24FF4AF6253431B132E
:1049F800064A03F5487322F814300134E5E7012329
:104A080081F83C3070BD00BFF00B0020F20B002095
:104A180003788B420BD9074B1A78074B8900194446
:104A2800086C02B1400800F5777080B2704700202A
:104A3800704700BFC4210020F00B002007299DBF4C
:104A4800034B03EB8101B1F870000020704700BFF1
:104A5800F00B0020034B03EB4101B1F89000C008B4
:104A6800704700BFF00B00200A4BDFED0B7A03EB19
:104A7800810191ED2C7AB8EE477AF6EE046AE7EEFA
:104A8800267A82B0FCEEE77ACDED017ABDF8040013
:104A980002B07047F00B002000005C44024B03EBAF
:104AA8004101B1F8F8007047F00B0020024B03EB0E
:104AB8004101B1F81C017047F00B002070B5334C70
:104AC800054605F051FBD4F83431C4F83401C31A53
:104AD800B3F5FA5FC4F8383182BF002384F83C315B
:104AE80084F83D3194F83C312BB9A12D02BF274AF7
:104AF800012182F83D1194F83D11244A29B1D118B9
:104B0800EDB201338D7682F83C3194F83C5194F83B
:104B18003E31AB4239D11D4B93F83F31052B02D0C2
:104B2800062B03D02CE00020FFF722FFE37E1E2B8C
:104B380026D100200246C1B26B1E994219DA2144DF
:104B48008B7E0821DBB283EA0206F60744BF83F0B6
:104B58001803C3F3460301F1FF3154BF5B0843F068
:104B6800800311F0FF01C2F34702ECD101301A466D
:104B7800E1E723449B7E9A4202D10320FFF7F8FE27
:104B8800002384F83D3184F83C3170BDF00B0020DF
:104B980010B5044605F0E8FA0F4BD3F84021C3F8E6
:104BA8004001821A41F288318A42C3F8442184BF05
:104BB800002283F8482193F84821074913440F2A13
:104BC800E4B218BF013283F8494112BF81F8482185
:104BD800012381F8593110BDF00B002010B50446AF
:104BE80005F0C2FA0F4BD3F85C21C3F85C01821AB6
:104BF80041F288318A42C3F8602184BF002283F8D9
:104C0800642193F8642107491344142A18BF013218
:104C180083F8654112BF81F86421012381F87A3154
:104C280010BD00BFF00B002038B5044605F09CFA13
:104C3800274A2749D2F87C31C2F87C01C31AB3F558
:104C48007A6F84BF002382F8803192F8803133B9BB
:104C5800A82C3BD181F88131A1F8823106E0022BE2
:104C680002D181F8844101E0242B02D8D11881F8BF
:104C7800854192F88411164D01330231DBB24900A7
:104C88008B4282F8803118DAB5F88231E0B283EAD3
:104C98000020082310F4004F4FEA400018BF80F4AA
:104CA800815003F1FF3318BF80F0010013F0FF03B8
:104CB80080B2EFD1A2F8820138BD01318B4201BF29
:104CC800002385F88031012385F8813138BD00BF84
:104CD800F00B002010B5044605F046FA104AD2F849
:104CE800AC3140F6AC51C31A8B42C4BF002382F8E2
:104CF800B03192F8B031D11881F8B14123B90F2CF5
:104D08000DD10749C1F8AC010133DBB2192B0449B5
:104D180082F8B0310CBF0123002381F8CA3110BDDD
:104D2800F00B00202DE9F843324F3D682A8A2E7A8D
:104D3800B2B9042E14D1304C30482378012B0BD152
:104D48002F4B19682F4B89B20B445B0019681A6006
:104D580030230380227048E010230380072644E0B4
:104D6800AC8AAB69A24294BF04260226944228BFAB
:104D780014461FFA84F840469847214A13689BB2A4
:104D880003F1005303F540535B0004F1010E1B6867
:104D98009BB203F1005303F540534FEA6E0E5B00DC
:104DA8000021714500F1020009D010F8019C10F8AB
:104DB80002CC4CEA092C23F821C00131F1E7126832
:104DC800104B92B213445B001A681C602B8AC8EB24
:104DD80003032B826B8A9844084BA5F81280302273
:104DE8001A80094B4FF440521A803B681E72BDE886
:104DF800F88300BF881A0020EF220020721A0020D2
:104E0800505C004002300020701A00200E4B0F4A00
:104E18001B689BB203EBC00002443E294FEA4202E2
:104E280009D94B09C80604BF03F1FF339BB29B02A3
:104E380043F4004304E04B08C90748BF01339B0211
:104E480011681360704700BF505C004006300020B6
:104E580010B5454B1A68107810F07F0004D1537ACA
:104E680023F02003537210BD02287AD15388002BF7
:104E780078D11379002B75D1537923F08000840001
:104E880004F1804101F5B84113F0800F096814BF9F
:104E980001F0300101F44051032862D8002960D0A4
:104EA800927A002A5DD004F1804404F5B8441906CA
:104EB800226825D502F03002102A4CD103F07F0376
:104EC8009B0003F1804303F5B8431A68510641BFBC
:104ED800196840F60F720A4042F4004244BF42F09B
:104EE800C0021A601A6822F4E04222F0400292B22C
:104EF80082F0300242F4004242F080021A602AE056
:104F080002F44052B2F5805F25D128B9174B93F8C7
:104F18002C10FFF77BFF11E09B0003F1804303F5A2
:104F2800B8431A68520441BF196840F60F720A4024
:104F380042F4404244BF42F080021A60236823F4DE
:104F4800804323F070039BB283F4405343F400433F
:104F580043F080032360064B1B685B699847002079
:104F680010BD022010BD00BF881A0020AC00002030
:104F7800781A00208A68036810B50C6A14430A6915
:104F880014434A6914438A691443CA6914434A6A30
:104F980014438A6A23F4FF4323F070032243134324
:104FA80003608B8943600B6883604B68C36010BDE6
:104FB80002684FF6FE7313400360002303604360EA
:104FC8008360C360284B984201D1284A27E0284BC8
:104FD800984201D1254A2AE0264B984201D1234A1A
:104FE8002DE0254B984201D1204A30E0234B9842CE
:104FF80001D11E4A33E0224B984204D11B4A536820
:1050080043F470032EE01F4B984204D1174A5368AB
:1050180043F0706326E01C4B984204D11B4A536846
:1050280043F00F031EE01A4B984204D1174A536805
:1050380043F0F00316E0174B984204D1134A536823
:1050480043F470630EE0144B984204D10F4A53683E
:1050580043F4704306E0114B984204D10B4A53685D
:1050680043F4702353607047080002400000024078
:105078001C00024030000240440002405800024038
:105088006C00024080000240080402400004024014
:105098001C04024030040240440402405804024008
:1050A800084BDA68D10709D4DA68D20608D4DB6875
:1050B80013F0040F14BF0320042070470120704729
:1050C8000220704700200240994A536803F00C03FD
:1050D800042B2DE9F04105D0082B06D09549016035
:1050E800B3B916E0934B036012E053685468C3F3F6
:1050F8008343991CE30349BFD36A8F4B8D4C03F05C
:105108000F0344BF0133B4FBF3F34B43036000E0E8
:1051180000235168894FC1F303117D5C0168EDB22A
:1051280021FA05F444605668C6F30226BE5D24FAE7
:1051380006FEC0F808E05668C6F3C226BE5DF6B2A1
:10514800F440C460D2F82C80C8F3041808F00F0C9F
:1051580007EB4C0C18F0100FBCF810C01FFA8CFCB1
:1051680007D0BCF1000F04D0B3FBFCFCC0F810C0A2
:1051780000E00161D2F82CC0CCF3442C0CF00F08ED
:1051880007EB48071CF0100F3F8ABFB204D01FB1CD
:10519800B3FBF7F7476100E04161176BFF065ABFA1
:1051A800644F87618161176BBF065ABF614FC76142
:1051B800C161176B7F065ABF5E4F07620162176BAA
:1051C800FF0506D5994204D1AE4202D14F0047628D
:1051D80000E04462176BFF0406D5994204D1AE4241
:1051E80002D14F00876200E08462176BBF0506D5C5
:1051F800994204D1AE4202D14F00C76200E0C462B6
:10520800176B7F0506D5994204D1AE4202D14F00F3
:10521800476400E04464176B3F0506D5994204D102
:10522800AE4202D14F00876400E08464176BBF046C
:1052380006D5994204D1AE4202D14B00C36400E0C6
:105248008464156B3A4BAD0701D1046315E01C6B00
:1052580004F00304012C01D101630EE01C6B04F07F
:105268000304022C02D14FF4004305E01B6B03F04A
:105278000303032B01D12F4B0363146B2C4B14F442
:10528800403F02D1C0F834E018E01C6B04F440340D
:10529800B4F5803F01D1416310E01C6B04F4403445
:1052A800B4F5003F02D14FF4004306E01B6B03F452
:1052B8004033B3F5403F01D11E4B4363146B1C4B85
:1052C80014F4402F02D1C0F838E018E01C6B04F445
:1052D8004024B4F5802F01D1816310E01C6B04F4E5
:1052E8004024B4F5002F02D14FF4004306E01B6BB5
:1052F80003F44023B3F5402F01D10E4B8363146BA5
:105308000B4B14F4401F02D1C0F83CE020E01C6BAA
:1053180004F44014B4F5801F01D1C16318E01C6B7C
:1053280004F44014B4F5001F0AD14FF400430EE012
:105338000010024000127A0000093D00160000200B
:105348001B6B03F44013B3F5401F01D1134BC36328
:10535800126B134B12F4400F03D1C0F840E0BDE8C4
:10536800F0811A6B02F44002B2F5800F02D1016499
:10537800BDE8F0811A6B02F44002B2F5000F02D1C9
:105388004FF4004306E01B6B03F44003B3F5400FF2
:1053980001D1024B0364BDE8F08100BF00127A001E
:1053A80000100240F0B500230E681C460125A540F8
:1053B80005EA060EAE452BD10F797A1E012A15D8BB
:1053C800856803229A4025EA020282604D79826844
:1053D8009D4015438560828892B222EA0E0282803F
:1053E8008A798588A2402A4392B28280032205687E
:1053F8009A40D2431540056005689F402F430760D7
:10540800C7681740CA7902FA03F547EA0502C2607D
:105418000134102C03F10203C8D1F0BD38B52DEDCD
:10542800048B4A4C0368C4F8CC318388A4F8D03183
:10543800013A0D46072A42D8DFE802F0040A10189C
:1054480022292F35B4F8CC310B80B4F8CE3113E0D3
:10545800B4F8CE310B80B4F8CC3105E0B4F8CC31D7
:105468005B420B80B4F8CE315B4205E0B4F8CE3134
:105478005B420B80B4F8CC316B80B4F8D0311DE0BE
:10548800B4F8CC315B420B80B4F8CE3112E0B4F8FA
:10549800CE310B80B4F8CC310CE0B4F8CC310B80B1
:1054A800B4F8CE3105E0B4F8CE315B420B80B4F8E5
:1054B800CC315B426B80B4F8D0315B42AB80244B7B
:1054C80093F83030002B3ED1B5F9003094ED780ACE
:1054D800D4ED757A09EE103AB5F9023008EE103AB3
:1054E800B8EEC88AB5F90430B8EEC99A28EE000AB1
:1054F80008EE903AA7EE890AF8EEE88AD4ED7B7AAE
:10550800A7EEA80A09F0DCFE94ED790AD4ED767AC4
:10551800288028EE000AA7EE890AD4ED7C7AA7EE47
:10552800A80A09F0CDFE94ED7A0AD4ED777A68805E
:1055380028EE000AA7EE890AD4ED7D7AA7EEA80A1C
:1055480009F0BEFEA880BDEC048B38BDF00B00202E
:1055580016000020094BD3F8F821137844F6FB71A4
:1055680003EB431300FB03135078C0EB0030B3FB8D
:10557800F0F39078B3FBF0F080B27047F00B0020A6
:1055880010B50A4C94F8FD3104EB43030A22B3F832
:105598000C1204F5067089B2A4F8141204F030FE57
:1055A80080B2FFF7D7FFA4F8A00210BDF00B0020CF
:1055B800F0B50124B0FBF4F58D4201D34C43F9E773
:1055C8000026D4B1B0FBF4F504FB1500B4FBF1F4EC
:1055D8001EB9002D01DC002CF3D1092D03F1010EB9
:1055E800EFB204DD002A14BF3725572500E0302527
:1055F8003D441D7001367346E3E71C70F0BDF0B5FD
:105608000124B0FBF4F58D4201D34C43F9E70026A1
:10561800D4B1B0FBF4F504FB1500B4FBF1F41EB9EA
:10562800002D01DC002CF3D1092D03F1010EEFB29E
:1056380004DD002A14BF3725572500E030253D44F6
:105648001D7001367346E3E71C70F0BD2DE9F84381
:10565800089E002B07468846144614BF4FF03009B1
:105668004FF02009334613F8012B0AB9254603E009
:10567800002CFBDD013CF6E7002D04DD38464946E9
:10568800C047013DF8E724EAE4743546A01B2844E6
:1056980015F8011B11B13846C047F7E7BDE8F88394
:1056A800014B186804F0A9BDD003002090ED017AE1
:1056B80007EE901AB5EE407AF1EE10FA01BFF8EE57
:1056C800E77A9FED0E7A67EE877AB7EE007A04BF25
:1056D800C7EE277AC0ED017A90ED017AD0ED007A15
:1056E80030EE877A30EE670AC0EE870AE0EE807AFD
:1056F800B0EE670AC0ED007A704700BFDB0FC94003
:1057080010B50278202A034600F10100F9D0092AD1
:10571800F7D02D2A03D10346BFEE000A04E02B2A56
:1057280008BF0346B7EE000ADFED387A1A4613467B
:1057380012F8010BA0F13001CCB2092C0AD807EEFF
:10574800101AB8EEC77AF2EE046AA7EEA67AF0EE5F
:10575800477AECE72E2816D1F2EE046A1146B0EE2D
:10576800666A0B4611F8012B303AD0B209280AD8DC
:1057780007EE102AB8EEC77A87EE267A66EE866AB2
:1057880077EE877AEDE71A7802F0DF02452A35D1FD
:105798005A782D2A02D10233012004E02B2A14BFA3
:1057A800013302330020013B002213F8011F303976
:1057B800CCB2092C03D80A2404FB0212F5E7B2F58F
:1057C8009A7F28BF4FF49A721346B7EE007A072BD8
:1057D80005D9DFED0F6A083B27EE267AF7E702F0D6
:1057E80007032BB1F2EE046A27EE267A013BF8E7AD
:1057F800F0EE476A20B1C7EE877A03E0F7EE006A59
:1058080067EEA67A20EE270A10BD00BF0000000050
:1058180020BCBE4C30B52DED028B87B0B0EE408A6F
:105828000C220021054603A809F03BFBB5EEC08A0F
:10583800DFED2A7AF1EE10FACCBF38EE278A38EE7F
:10584800678ADFED277A28EE278A6946FDEEC87A4F
:1058580017EE904A84EAE470A0EBE47006F012F9BF
:10586800002CACBF20232D2368468DF80C3009F09E
:105878005CFB012807D130238DF80D308DF80E30F0
:105888008DF80F300CE0022805D130238DF80D304B
:105898008DF80E3004E0032804BF30238DF80D3056
:1058A800694603A809F024FB03A809F03EFB033866
:1058B800C4B2224603A9284609F064FB00232B55ED
:1058C8002846084909F014FB03AB2846191909F0C2
:1058D8000FFB284607B0BDEC028B30BD6F12033AB0
:1058E80000007A448722010870B506461546084626
:1058F800B6FBF2F414B12046FFF7F6FF05FB14647B
:10590800024B1B5D00F8013B70BD00BF89220108F6
:105918000FB42DE9F04F7C4B89B012ACD3F800805E
:105928007A4B54F8046BD3F800900494002531782E
:10593800002900F08680252902D00136404674E00F
:105948007278302A08BFB278A2F1300319BFB71CA9
:105958004FF0000BF71C4FF0010B092B4FF0000A1A
:1059680019D8A2F13003D9B2092905D80A2202FBB5
:105978000A3A17F8012BF4E7A2F16103052B02D8C4
:10598800A2F1570305E0A2F14103052B03D8A2F1C8
:1059980037030A2BEADD6C2A30D13A78642A07F1FA
:1059A800010600F088800AD8252A3CD002D8002AAF
:1059B80047D0BCE7582A0CD0632A19D0B7E7732A16
:1059C80022D002D86E2A37D0B1E7752A62D0782A59
:1059D800ADD1271D2068A2F1580462424FF0100192
:1059E80062415BE02CD9582A38D0632A34D13E462C
:1059F80040462178271DC84701350FE0642A6AD040
:105A08000ED9732A14D13E4623680093404649466E
:105A180052460023FFF71AFE271D05443C4686E739
:105A2800252ADFD13E4640462521C84701357EE775
:105A38000ED86E2A10D13E46236804341D6076E7DE
:105A480052B9334B186804F0D5FB0028F9D054E05C
:105A5800752A28D0782A01D03E4668E7A2F1580373
:105A680004F1040C5A422068CDF80CC04FF0100124
:105A78005A4105ABFFF79CFDDDF80CC03E46644675
:105A880005AB00934046494652465B46FFF7DEFDAC
:105A980005444CE72068271D0A21002205ABFFF7C3
:105AA800AEFD3C46ECE704F1040CCDF80CC02068D0
:105AB8000A210022DDE72068002804F1040708DA3B
:105AC8002D238DF8143040420DF115030A210022D0
:105AD800E5E705ABFAE72068002804F1040C0ADAC8
:105AE8002D238DF8143040420DF11503CDF80CC06C
:105AF8000A210022BEE705ABF8E7284609B0BDE851
:105B0800F04F04B0704700BF7401002070010020FE
:105B1800D003002080EAE073A3EBE0738B4206DB3E
:105B2800002801DD401A704702D008447047002061
:105B38007047FDEEC07A17EE903A2033402B43D8D9
:105B4800DFED237AB4EEE70AF1EE10FA04DDDFEDBB
:105B5800217A30EE670AF3E7DFED1F7AB4EEE70A41
:105B6800F1EE10FA04D5DFED1B7A30EE270AF3E7E1
:105B7800DFED1A7AB4EEE70AF1EE10FA04DD30EE42
:105B8800670A37EEC00A0AE09FED157AB4EEC70A35
:105B9800F1EE10FA44BF30EE270A37EE400A60EE05
:105BA800007ADFED106A9FED107AA7EEA67ADFED96
:105BB8000F6AE7EE876A9FED0E7AA7EEA67A20EEC7
:105BC800276AA6EE070A70479FED0A0A704700BFCA
:105BD800DB0F4940DB0FC940DB0F49C0DB0FC93F72
:105BE800DB0FC9BF9A7C2E36FAAF4FB93587083C10
:105BF800A4AA2ABE0000000038B52DED068B90ED52
:105C0800008ADFED2D9A38EE290A0C460546FFF783
:105C180090FFB0EE40AAB0EE480AFFF78AFFD5ED34
:105C2800018AB0EE409A38EEA90AFFF782FFB0EE7B
:105C3800408AB0EE680AFFF77CFFD5ED02AAF0EEC5
:105C4800408A3AEEA90AFFF774FFF0EE409AB0EEE8
:105C58006A0AFFF76EFF60EE0A6A69EE297AF0EECB
:105C6800665AE7EEA85A29EE8A6A29EE007A69EEA2
:105C7800889A29EE489A28EE400A28EE0A8AC4ED46
:105C8800035AF0EE465AE7EE685AE6EEA87AA6EE10
:105C9800687AC4ED009AC4ED028A84ED059A84ED11
:105CA800088ABDEC068B84ED010AC4ED045A84ED24
:105CB800067AC4ED077A38BDDB0FC93F10B52DED64
:105CC800048B8AB090ED009AD0ED028A90ED018A9B
:105CD8000446084601A9FFF78FFFDDED047A9DED24
:105CE800017A68EE277AE9EE077A9DED077AE8EE01
:105CF800877A9DED027AC4ED007ADDED057A68EECB
:105D0800277AE9EE077A9DED087AE8EE877AC4EDFE
:105D1800017ADDED067A28EE278ADDED037AA9EE11
:105D2800278ADDED097AA8EEA78A84ED028A0AB0EF
:105D3800BDEC048B10BD074B1A8822EA0000904284
:105D480010B518801C4602D0012001F075FE20888D
:105D580010BD00BF2C170020064B1A881043904234
:105D680010B518801C4602D0012001F065FE20887D
:105D780010BD00BF2C170020024A936823EA0000D8
:105D880090607047CC1A0020024A936818439060CC
:105D9800704700BFCC1A002008B5104B1A780023B2
:105DA800D9B2914207D20E4951F823100968002050
:105DB80008600133F4E7322004F0FDF9094B1B6851
:105DC8005A0309D5084B9B685B0305D440F2DC50A5
:105DD800BDE8084004F0EFB908BD00BFD6170020A1
:105DE800F817002008220020CC1A00202DE9F341E2
:105DF80006F000F8454A692313704FF4DE635380B8
:105E0800BE231371EF2382F8EE36002382F8EF36B3
:105E180019461646F25C0133B3F5DE6F81EA0201DA
:105E2800F8D13A4B83F8EF16394B1A69120604D5A4
:105E3800384A5A6002F188325A6004270020013F2C
:105E480017F0FF074FD0324B3422DA60002444B1F8
:105E5800002356F80480019305F0E5FD0428EED1EF
:105E680017E005F0E0FD0428E9D1294D2B6943F03E
:105E780002032B61284B6B612B6943F040032B61B4
:105E880005F0D1FD2B69042823F002032B61DFD034
:105E9800D5E71F4D2B6943F001032B6104F1006323
:105EA80003F57E331FFA88F21A8005F0BCFD04283A
:105EB80010D11A4B23440193019B4FEA1848A3F8C9
:105EC800008005F0B0FD2B69042823F001032B6145
:105ED80005D0B4E72B6923F001032B61AFE7043445
:105EE800B4F5DE6FB3D10A4A1369042843F080037E
:105EF800136102D101F093FF10B9052001F0B4FD40
:105F080005F064FF02B0BDE8F08100BFCC1A0020A4
:105F1800002002402301674500F8030802F803083F
:105F280010B50E4C206801F0EFFC2068047A0022BE
:105F380002FB02F3193B634303F6C41353431921CD
:105F480093FBF1F3064921F812300132072AEFD109
:105F58000449BDE8104001F08DBC00BFE8210020D5
:105F6800F8020020101C00202DE9F04101F057FF35
:105F780010B9042001F078FDA64CA74D05F03AFFB2
:105F8800A6494FF4DE62204608F080FF94F8C83630
:105F9800022B84BF002384F8C83694F8C8264FF42F
:105FA800C67101FB02F3E018234400F5097028606C
:105FB80093F8780203F51C73022801FB024284BFA0
:105FC8000020187292F87832954A13700C2202FB5E
:105FD8000343944A03F2CA631360A26846F20903B2
:105FE80013401BB94FF40050FFF7CEFEA368D80743
:105FF80003D54FF40050FFF7BFFEA368590409D535
:106008000820FFF7B9FE4FF40050FFF7B5FE012056
:10601800FFF7B2FEA3681A0706D54FF40050FFF742
:10602800ABFE0120FFF7A8FEA3689B0402D5402021
:10603800FFF7A2FE012284F8152294F8E021754B9F
:106048002AB193F8E42112B1002283F8E421764BB7
:10605800764E1E604FF0000C674604EB0C03B3F855
:10606800F4E14FEA5E0101F077314FEA9E0303F055
:106078003333C1EB0E00C11A4FEADE0303F01133CC
:10608800CB1A03EB23131EF0010803F00F324FF075
:10609800FF0392FBF3F3C3EB032318BF0137A2EB13
:1060A800030318BFFFB2012B0ADD022B40F0AF80BB
:1060B800B8F1000F00F0AB801EF0BC0F00F0A78015
:1060C8000CF1080CBCF1200FC7D1013F012F00F2E1
:1060D8009E80FFF725FF002130225548554F08F0D4
:1060E800E0FE554BD5F800801F60544B08F179004D
:1060F800C3F8008005F088FC514B80F0010018704F
:10610800504B07F126021A6098F8000004F0B4FA20
:106118004D4B94F8D801DFED4D6A07F194021A60EF
:1061280064214B4BC82211FB00225A6000229A605E
:10613800DA601A615A619A61DA6183F8202083F87B
:106148002120444B07F12C021A602B68424A93ED38
:10615800187A03F219111160404A03F2891111608B
:106168003F4A07F1080111603E4A17603E4A07F1AD
:10617800A00111603D4A07F1AA0111603C4967EE90
:10618800266A0E60B4F86611B6EE007A07EE901A29
:1061980087EE267AB4F86811101DF8EE677AC2ED1A
:1061A800027A07EE901A93F85C10117193F8781040
:1061B800517194F8E3111174F8EE677AB3F8161177
:1061C800C2ED037A07EE901A2A4908602A495361FA
:1061D80003F1640008602949936181ED007AF8EEC3
:1061E800E77A9FED277A27495762C7EE277ABDE8F5
:1061F800F0419FED257A67EE877AC1ED007A03F1C9
:10620800680103F21113D161136205F0DFBD05F0D7
:10621800CDFB5EE7CC1A0020F40E002000F803083E
:10622800E4210020E821002004220020561C002040
:10623800B00B0020101C0020E40B0020E80B00200D
:10624800140000202C04002028110020DB0F4940F6
:106258001422002084040020F80E0020900600205C
:10626800F0180020F4180020A4050020980E002043
:1062780068060020B4040020EC040020E804002094
:1062880000006144A00500204C3D0F4408B5FFF70D
:10629800ADFDFFF769FE0120BDE8084001F0CCBB69
:1062A80038B500240B4D6059254405F0B9FE6968DE
:1062B80011B10948FFF72CFBA96811B10748FFF78E
:1062C80027FB0748103405F0ABFEB4F5C07FE9D1D1
:1062D80038BD00BF7409010880230108862301081E
:1062E800F12C010870B50546284608F01EFE064642
:1062F80058B91A4B1A485A791A4B03EB8203BDE86E
:106308007040D3F87C11FFF703BB28461649324684
:1063180008F014FE60B91548154C05F081FE54F8D4
:10632800041F19B11348FFF7F3FAF8E7124805E01C
:106338000024124B53F8241021B91148BDE87040CD
:1063480005F06EBE2846324608F0F8FD01340028F4
:10635800EFD1024B0B4D5C71C6E700BFCC1A002091
:106368008C23010874090108982301089D2301085A
:10637800F00A0108B0230108F12C0108F40A010809
:10638800B42301084C210108F0B585B0044608F093
:10639800CCFD082826D1621EE01D1F4912F8013FD6
:1063A80009681944497801F00301022908BF203B14
:1063B80082421370F1D1254604F1080715F8016BE4
:1063C8001648314608F0A3FD20B12846314608F0AA
:1063D8009EFD10B100F0DCFE1CE0BD42EED120466F
:1063E80005F033FB0E4805F01BFE00230D4A1A4446
:1063F80004A992F88A210A440849595C02F80C1C3D
:106408000133082BF2D1002307488DF80C3001A97D
:10641800FFF77EFA05B0F0BD040100209B2B0108B0
:10642800C3230108CC1A0020332C01082DE9F041C0
:10643800054608F07AFD2F4B04469E6888B92E4819
:1064480005F0EEFD2D4B53F8241041B10123A34074
:10645800334202D02A48FFF75BFA0134F2E72948B1
:1064680021E028462849224608F068FD58B92748FF
:10647800274C05F0D5FD54F8041F0029EFD020481B
:10648800FFF746FAF7E72B782D2B03BF013504F108
:10649800FF344FF001084FF000080026174B53F85F
:1064A800267027B91B48BDE8F04105F0B9BD28465C
:1064B8003946224608F042FDC8B90120B04002061C
:1064C80001D51548EFE78305FBD4B8F1000F03D0D9
:1064D800FFF752FC114802E0FFF756FC104805F0A0
:1064E8009FFD39460F48BDE8F041FFF711BA013664
:1064F800D4E700BFCC1A0020C92301085C0B0108AF
:10650800B0230108F12C010898230108D3230108BE
:10651800580B0108B4230108DF230108ED23010803
:10652800F6230108322C010810B5084805F078FD5B
:10653800074B00241C701C63064B1C7003F0E0FF23
:1065480005F0FAFE044B1C6010BD00BFFE230108D5
:10655800C00E0020EC2200204822002070B506461C
:1065680000240B4BE518AA8816420AD0E1580948BE
:10657800FFF7CEF92846002105F0DFFC064805F0B4
:106588004FFD143440F618339C42EAD170BD00BF69
:10659800441401082A240108F12C0108F0B50478F4
:1065A8008BB005460CB1002436E04B4B596B0E23DB
:1065B80003FB041101F58C70B1F91D51B1F91921D2
:1065C800B1F91B31009591F82051019591F82151AD
:1065D800029590F90700039001F590713F4891F9F1
:1065E8000210049121460134FFF792F9082CDCD1FE
:1065F80070E02D2B14D1072C1BDC284608F0ECFC8E
:106608000AAB661C03EB440424F8100C15F8013F90
:10661800303B092BFAD934462B78002BE9D104E01A
:10662800A3F13002092A09D8E5E7082CBDF818209B
:1066380009D00BB0BDE8F04000F0AABD202BF8D17E
:1066480001352646E7E7072AF3D8BDF81A00224B9A
:10665800A0F2EE2189B240F2DC55A9425B6BE8D882
:10666800BDF81C10A1F2EE24A4B2AC42E1D8BDF8EA
:106678001E6004B237B2A742DBDB0DB2AF42D8DCF2
:10668800A542D6DBBDF8247007F16404A4B2C82C77
:10669800CFD8BDF826E00FFA8EF4112CC9DCBDF86E
:1066A8002050B42DC5D8BDF82240B42CC1D812B2A0
:1066B8004FF00E0C0CFB0233A3F81901A3F81B11C1
:1066C800A3F81D6183F8205183F8214183F81F71D5
:1066D80083F822E10BB0F0BDC00E0020342401087D
:1066E8002DE9F041047806467CB9334DB5F8C6214A
:1066F800B5F8C831314821460134FFF709F9042CAF
:1067080005F10405F2D1BDE8F0812D4908F0D2FB6E
:10671800B0B9294B4FF47A714FF4FA62A3F8C61155
:10672800A3F8C821A3F8CA11A3F8CC21A3F8CE1165
:10673800A3F8D021A3F8D211A3F8D421BDE8F081A1
:10674800304608F049FC032805462DD8304620215C
:1067580008F0DDFB044630B10134204608F03CFC6B
:106768000126074600E006462046202108F0CFFB18
:1067780018B9BDE8F04100F00BBD013008F02CFC61
:10678800012EF6D1A7F2EE2240F2DC539A42F0D85D
:10679800A0F2EE229A42ECD8074B703503EB850342
:1067A800DF801881BDE8F0810648074900220323ED
:1067B800BDE8F041FFF7ACB8CC1A0020542401081A
:1067C800672401086D2401083F2E01082DE9F041D6
:1067D8002DED048BAB498AB0044608F06BFBAA493F
:1067E800002820460CBF0126072608F063FBA749AE
:1067F8000028204608BF022608F05CFB002808BFD6
:106808000426F10740F1E480A148A24C05F008FCF9
:10681800002005F0B3F9A04805F002FC9F4805F0F8
:10682800FFFB62799E4B9F4803EB82032546D3F812
:106838007C11FFF76DF89C48FFF76AF84FF00008E5
:10684800274695ED058AB5EE408AF1EE10FA04D197
:106858009648FFF75DF8002570E09548D5ED069A53
:1068680095ED079AD5ED088A4146FFF751F8B5EE40
:10687800C08AF1EE10FA02D5202005F0C9FBB0EE6F
:10688800480A06A8FEF7C6FF01468A48FFF740F8FF
:10689800F5EEC09AF1EE10FA02D5202005F0B8FB0B
:1068A800B0EE690A06A8FEF7B5FF01468148FFF772
:1068B8002FF8B5EEC09AF1EE10FA02D5202005F0B7
:1068C800A7FBB0EE490A06A8FEF7A4FF01467948DF
:1068D800FFF71EF8F5EEC08AF1EE10FA02D5202077
:1068E80005F096FBB0EE680A06A8FEF793FF08F1DC
:1068F800010801467048FFF70BF8B8F10C0F05F1D5
:1069080010059ED1A4E749B294F8D42094F8D53064
:10691800009194F8D710019194F9D810029194F944
:10692800D910039194F8DA10049164482946013586
:10693800FEF7EEFF102D04F1070403D094F8D610EB
:106948000029E0D15E485F4C05F06AFBD7F8088063
:1069580054F8041F19B15C48FEF7DAFFF8E70D4652
:106968005A4B53F8254054B10123AB4013EA080FA2
:1069780003D057482146FEF7CBFF0135F0E75548CD
:1069880005F04EFB21467B180AAA93F88A31134476
:10699800514A8A5C03F8102C01310829F3D10023ED
:1069A80006A94E488DF82030FEF7B2FF4C4805F096
:1069B80037FB4C4800F096FE4B48FEF7A9FF4020F5
:1069C800FFF7CCFD494805F02BFB464800F098FC42
:1069D800B20739D5464805F023FB464805F020FBA9
:1069E800404805F009F9444805F01AFB3D4800F015
:1069F80056FB424805F014FB3A4800F0CFFB4048EC
:106A0800FEF786FF3748FFF76BFE3E4805F008FBA8
:106A18003448FFF7C3FD00270E257D4300243A4A7A
:106A2800926B2A440123D2F80A20A34013421ED1B4
:106A380001340E2CF3D10137082FEDD12A48FEF787
:106A480067FF8020FFF78AFD730716D52F4805F0EA
:106A5800E7FA2F4805F0E4FA224805F0A9F8224899
:106A6800FEF756FF4FF48070FFF778FD05E03946D2
:106A780022462848FEF74CFFDAE70AB0BDEC048B43
:106A8800BDE8F0818C240108C92801089324010875
:106A980099240108CC1A0020A7240108B924010868
:106AA80074090108C5240108D0240108DD2401085F
:106AB800EA24010889230108332C0108022501086A
:106AC800F2240108580B0108212501085C0B010874
:106AD8002F2501083C2501089B2B010848250108A2
:106AE800512501084C210108F12C010860250108F5
:106AF8006D250108802501088E25010898250108C3
:106B0800A7250108B5250108C00E0020C1250108E8
:106B1800D2250108E4250108F0B504468FB02046C7
:106B280008F003FAC5B225BBAC48AD4C05F078FABD
:106B380094F8D61009B9AB4854E049B294F8D42077
:106B480094F8D530009194F8D710019194F9D810A1
:106B5800029194F9D910039194F8DA100491A2489B
:106B680029460135FEF7D4FE102D04F10704DFD1C4
:106B7800E1E720469D49052208F0E0F90546B8B945
:106B880029469B48702208F08CF99A4B596B284685
:106B98000E2303FB001301300022082883F8232169
:106BA80083F8242183F8252183F82621F0D113E1E5
:106BB80020469149042208F0C1F905462046002DD7
:106BC8004AD1202108F0A3F9002800F00581461CCD
:106BD800304608F0AAF92C460746884B53F824504B
:106BE8002DB987480FB0BDE8F040FEF791BE30469A
:106BF8002946FAB208F0A2F901340028EDD1784A02
:106C080002F170011646002382F8DA3082F8D63095
:106C180082F8D53082F8D43007328A42F3D17949E4
:106C280001EBC40191F84022934210DAD1F8447282
:106C3800C3EBC302B0183A4400F1D4011768C0F896
:106C4800D4709088888092798A710133E7E7294661
:106C58006D48FEF75DFE90E06C49072208F06EF97A
:106C680005462046002D4AD1202108F050F9064655
:106C780008F05BF9C4B274BB6548FEF749FE2146CB
:106C880064480134FEF744FE0E2CF8D15548FEF74F
:106C98003FFE002460482146FEF73AFE0025554A8B
:106CA8005E48516B0E2202FB04120123D2F8232105
:106CB8005B49AB4013425B4B05F1010508BF194620
:106CC800FEF726FE0E2DEAD146480134FEF720FED7
:106CD800082CDFD180E03046534908F081F92C4672
:106CE80000284CD0022C4FD008F076F906AB4E495C
:106CF80043F82400002008F073F90134F0E74A490A
:106D080008F06EF9002460B1082C38D008F064F956
:106D180006AB454943F82400002008F061F9013426
:106D2800F1E7082C2BD1069B0F2B28D8DDF81CE0A7
:106D3800BEF1070F23D8089F0D2F20D8099E06F112
:106D48006402C82A1BD80A9DFF2D18D80B986428FE
:106D580015D80C99642912D8884210DA0D9C032C96
:106D68000DD8324AC3EBC303134483F804E05F71C0
:106D78009E71DD71187259729C722D4CCFE60FB05E
:106D8800BDE8F04000F004BA069B072B20D807990D
:106D98000D291DD80278722A0DD06E2A18D1154AED
:106DA800526B0E2000FB032301228A40D3F82311E3
:106DB80021EA020209E00F4A526B0E2000FB03236E
:106DC80001228A40D3F823110A43C3F8232101E0A2
:106DD80000F0DEF90D4CA2E60FB0F0BD0326010865
:106DE800CC1A0020F12C01082E260108672401087E
:106DF800A01B0020C00E00204A260108F40A010842
:106E0800B4230108740901084F260108FB2501086D
:106E18008A2301085B2601084B2C0108602601081B
:106E2800772F010817300108642601089C1B0020F1
:106E38004C2101082DE9FF4104780546002C39D181
:106E48007348744D05F0ECF8D5ED057AF5EE407A07
:106E5800F1EE10FA00F0D98021466F48FEF758FD90
:106E680095ED050A6846FEF7D5FC01466B48FEF726
:106E78004FFD95ED060A6846FEF7CCFC01466748CB
:106E8800FEF746FD95ED070A6846FEF7C3FC014686
:106E98006248FEF73DFD95ED080A6846FEF7BAFC24
:106EA800013401465E48FEF733FD0C2C05F1100550
:106EB800CAD1AAE05B49052208F040F840B9554B11
:106EC80003F1C0020021596110339342FAD19CE0CA
:106ED80028465549042208F031F804462846002C73
:106EE80040D1202108F013F8002800F08E80451CBE
:106EF800284608F01AF807464C4B53F824601EB988
:106F08004B4805F08DF880E028463146FAB208F083
:106F180015F801340028EFD13E4B03F1C0029E461C
:106F28000021596110339342FAD1424B03EBC4025A
:106F38009846D2F804C0BCF1000F04D131463E484F
:106F4800FEF7E6FC57E0002718F834309F42F5DAE0
:106F58003B010EEB030563440FCB143585E80F00A6
:106F68000137F1E708F038F80B28064647DC2846D1
:106F7800202107F0CCFF054650B101352846FEF721
:106F8800BFFB244B03EB061383ED050A012400E045
:106F980004462846202107F0BAFF054648B10135C6
:106FA8002846FEF7ADFB1B4B03EB061383ED060AE1
:106FB80001342846202107F0AAFF054648B10135CB
:106FC8002846FEF79DFB134B03EB061383ED070AD8
:106FD80001342846202107F09AFF10B900F0D8F8AC
:106FE80013E00130FEF78CFB0A4B032C03EB06166B
:106FF80086ED080AF2D11148FFF71CFF05E010489A
:10700800104901220C23FEF783FC04B0BDE8F0818F
:1070180066260108CC1A0020812601088726010867
:10702800332C0108672401084A260108F40A0108DC
:10703800B4230108B02201084F2601084C21010899
:107048006D2401088B260108F8B504460E4617463C
:1070580000252046202107F05AFF0446D0B101340C
:10706800204607F0B9FFB0F5617F05DB40F6340331
:107078009842A8BF184601E04FF46170A0F561700E
:10708800192390FBF3F00DB9307000E070703B7875
:1070980001333B700DB90125DBE72046F8BD7FB50C
:1070A80004780646E4B9364B1B6803EB84031921C0
:1070B80093F87B0093F87C6093F8792093F87A3002
:1070C8004FF4617511FB005011FB065100900191BE
:1070D8002C4821460134FEF71BFC142CE3D14CE06C
:1070E80007F07AFF1328054641DC254B701C1C6805
:1070F800202100238DF80F3007F009FF1E350646C2
:1071080070B10136304607F067FF1A289FBF04EBBD
:10711800850358709DF80F30013398BF8DF80F30F4
:107128003046202107F0F3FE064670B1013630469E
:1071380007F052FF0D289FBF04EB850398709DF858
:107148000F30013398BF8DF80F3004EB85043046BB
:10715800E11C0DF10F02FFF777FF9DF80F30042BAC
:107168000BD0601C0021042207F09BFE05E00648B6
:10717800064900221323FEF7CBFB04B070BD00BF05
:10718800F40E0020022B01086D2401088B2601084B
:10719800014804F045BF00BF172B0108F0B504787B
:1071A80087B006461CBB524B1968062303FB041123
:1071B800192091F8CA5091F8CB7091F8CE2091F827
:1071C800C9304FF4617610FB056510FB0760009528
:1071D800019091F8CC000290C83146484979039152
:1071E80021460134FEF794FB0C2CDCD17DE007F03E
:1071F800F3FE0B28044672DC3D4B701C1D682021F1
:1072080000238DF8173007F082FE064680B101365C
:10721800304607F0E1FE03289FBF062303FB045313
:1072280083F8CE009DF817309CBF01338DF81730D6
:107238003046202107F06BFE074680B101373846FB
:1072480007F0CAFE0D289FBF062303FB045383F8EB
:10725800C9009DF817309CBF01338DF817300626FA
:107268006643A9193846CA310DF11702FFF7ECFE3B
:10727800202107F04CFE074670B10137384607F069
:10728800ABFE14289FBF9DF817307619013386F896
:10729800CC0098BF8DF817303846202107F037FE0C
:1072A80078B1013007F098FE0D289FBF062303FB35
:1072B800045383F8CD009DF817309CBF01338DF837
:1072C80017309DF81730062B0FD0062202FB04500A
:1072D8000021C93007F0E5FDFFF75AFF05E0064831
:1072E800064900220B23FEF713FB07B0F0BD00BFD1
:1072F800F40E0020252B01086D2401088B260108B7
:107308002DE9F347047806464CB9204601A904F054
:10731800B9FB0134FFF7F4FF122CF6D17AE007F03D
:107328005BFEC5B2112D6FD83C4C05F1D00704EBBC
:107338004703701C202193F80280394E07F0E7FDBF
:10734800034630B9A8F10202D2F1000848EB02085E
:1073580045E000F1010A5978304607F0D8FD60B1E0
:10736800032D8CBF03230023801B334453FA80F082
:1073780090F80490B9F1030F02D1FFF709FF49E033
:10738800A9F10203D3F1000850464FF0200148EB61
:10739800030807F0BCFDD8B1B8F1000FEDD00130FB
:1073A80007F01AFE40F2ED2380B2984205DD40F660
:1073B800CA039842A8BF184601E040F2EE2004EB49
:1073C8004703A0F2EE20192290FBF2F0D87002E0F9
:1073D800B8F1000FD1D104EB470383F8029004EB16
:1073E8004704A378F25CB8F1000F08D0E3780D48A1
:1073F800294640F2EE24192505FB034308E02946F7
:107408000948FEF785FA05E00848094900221123D2
:10741800FEF77EFA02B0BDE8F08700BFCC1A002064
:1074280004120108452B0108572B01086D24010897
:107438003F2E01082DE9F04F87B0814602919DF853
:10744800444011461A469DF840300026884D0C20CD
:1074580005F130077043C7574F4506D1284490F8C7
:1074680038B0BBF1000F04D0FEE00136042EEDD198
:10747800FAE0B9F1010F00F0E38006DCB9F1000F82
:1074880040F0F28000947B48DFE0B9F1020F00F091
:10749800DA80B9F1140F40F0E780DFF81CA2DAF8BF
:1074A800183043F00103CAF81830DAF814304FF0F6
:1074B800904443F40033CAF81430012703224FF4F0
:1074C800805804A94FF090408DF815200392CDF80C
:1074D80010808DF814708DF816708DF817B0FDF7C0
:1074E80061FFA4F82880C82002F065FEC4F818805F
:1074F800DAF81430039A43F40033CAF814302046FB
:107508004FF4C0538DF8152004A9022204938DF876
:10751800142003928DF816B08DF817B0FDF742FFCE
:10752800636A23F470436362636A43F4604363628B
:10753800636A23F470236362636A43F460236362BB
:107548004D4B4FF48021196001F18041A1F53F3185
:1075580012232B66082385F865300B6885F866705A
:1075680023F480230B604B6823F480234B6095F849
:10757800643003F1804303F58233196841F48021B4
:107588001960296E3D4B21F01F0401F01F01E058DE
:1075980007FA01F120EA0101E150296E384821F08B
:1075A8001F0401F01F0154F800E007FA01F12EEA68
:1075B80001012150296E21F01F0001F01F01C4585C
:1075C80007FA01F12143C1502E4B2F49C3F800B0EF
:1075D800DAF81C3043F40003CAF81C302B4B04A81B
:1075E800D9608DF81090039A8DF811208DF812B09B
:1075F8008DF8137004F072F82A238DF810309DF876
:1076080013308DF811708DF812B01BB104A804F076
:1076180065F804E01E4B4FF48062C3F884201D4ACD
:107628001D4B136002221A721C4A1D4B13601D4A1F
:107638001D491B68116098470D481C4B036007E003
:1076480000941B4801E01B48009401F0ADFF58B1BD
:10765800074B80F804900C2202FB06369DF8083090
:1076680086F83830706300E0002007B0BDE8F08F7E
:10767800FC0E0020003801401404014008040140B9
:107688000C040140D80042420005FA0500ED00E074
:1076980000E100E0881A0020C82100207C1A0020A0
:1076A800AC000020781A00204800002010120108C1
:1076B80000440040004800400010024010B5084B4C
:1076C800996E002201EBC20393F90240844201D172
:1076D800981C10BD0132042AF4D1002010BD00BF4F
:1076E800FC0E0020F0B5027887B08AB94B4C04F143
:1076F800200694F8F22100234949595650B2814294
:107708006CD00C33302BF7D10834B442F1D183E07C
:10771800002204920592451C07F05EFCC4B260B2D8
:10772800FFF7CCFF074618B18DF81040012400E0A0
:1077380004462846202107F0EAFB054638B1013502
:10774800284607F049FC0134ADF81200E4B20026DF
:107758002846202107F0DBFBA8B3451C284607F084
:107768003BFC00222F4951F822108142D3B203D0AA
:107778000132082AF6D100232B4A02EB8302526A0F
:10778800824220D1022E0FD0032E12D05A1E012E73
:10779800D2B204D0042A13D88DF814300EE0042A8B
:1077A8000ED88DF8153009E0052B09D88DF817305B
:1077B80004E09A1E052A03D88DF816300134E4B285
:1077C8000136042EC4D1052C03D807B0BDE8F0401B
:1077D800DEE404AB03CB386079601DE094F8F70170
:1077E800114B94F8F651B4F8F42103EB800003EB45
:1077F8008505406A009094F8F90103EB8000406A1F
:10780800019094F8F80103EB800308485B6A02933F
:107818006B6AFEF77DF877E707B0F0BDCC1A002059
:107828002C0F00202812010804120108662B0108F9
:1078380030B50B4B9C6E93F86C101A4603290BD885
:107848000B4604EBC3034D1CE9B29D882842F5D0D2
:1078580082F86C10981C30BD82F86C10002030BD86
:10786800FC0E0020024B002283F86C20E0E700BFEA
:10787800FC0E00202DE9F047877890F803C0214DD1
:10788800BBB2C7F1640E03EB83065C42C3F1780018
:107898005FFA8EFE7600CCF16408A4B280B2A3B27F
:1078A8000FFA83F9B9F1000F05DC002B14BFBA46B3
:1078B8004FF0010A00E0F24613FB03F303FB0CF25E
:1078C8001AFB0AF392FBF3F3434403FB09F30A227E
:1078D80093FBF2F333449BB225F8023FB1F80090D2
:1078E8004A880A34C9EB020AA4B21AB202FB0AF2A5
:1078F8004FF47A73844292FBF3F34B442B80CED13E
:10790800BDE8F087680F002010B5447800780022A1
:1079180002FB02F3193B634303F6C413534340F6D7
:10792800C411434393FBF1F3034921F812300132A8
:10793800072AEDD110BD00BF820F00200430114B83
:1079480033F91000B0F5617F10B506DB40F633035C
:1079580098420246A8BF1A4601E04FF461720C78BB
:10796800192340F2833013FB0404944207DA497860
:1079780013FB01039342B4BF0020012010BD002077
:1079880010BD00BFE80C00200A4B1B6813F4805F91
:10799800094BB3F9063005D0C089421A934207DD76
:1079A800084400E0008A8342B4BF002001207047E9
:1079B8000120704708220020E80C002010B50020A4
:1079C80002F012FC074B00241C7004F033FA064B3B
:1079D80083F89440C3F89840A3F89C40C3F8A040AB
:1079E80010BD00BF38220020FC0E002010B510B9D1
:1079F800BDE81040E2E700230C225A430C4C111951
:107A0800125D824203D00133102BF5D110BD094B12
:107A1800D3F8A00018B14A784078824206D20022F2
:107A2800C3F8A010A3F89C20C3F8982010BD00BF8D
:107A3800A4120108FC0E002010B540001428A8BFAD
:107A480014200023074A022199540B44991814243E
:107A5800834201F8014CF5DBFF21D1540F20BDE82A
:107A68001040C3E7662200202DE9F84380460B2525
:107A7800013D3DD0214B20221A8510229A6108F140
:107A8800010632274FF005091C4CA38A9BB283F0EC
:107A98002003A382A38A9BB283F01003A382012050
:107AA80002F0A2FB384602F086FBA38A9BB283F061
:107AB8002003A382A38A9BB283F010030020A38231
:107AC80002F092FB384602F076FBB9F1000F08D0BD
:107AD800B9F10109D8D14FF4FA7002F06CFBFA271A
:107AE800D2E7013ED0D14FF47A7002F064FBBFE7D1
:107AF800034B044ADA60BDE8F88300BF000400487D
:107B080000ED00E00400FA0582B01B4B1B4A8DF81B
:107B180007101968106860B31268052A29D1184A35
:107B2800106810BB9DF808109DF8073043EA012340
:107B380014490B80144B1968144B89B20B445B0031
:107B480019680121196013680B441360104A1368FF
:107B580023F4E04323F040039BB283F0300343F463
:107B6800004343F08003136003E01A68521A312A75
:107B7800D5D902B0704700BFC41A0020D82200200F
:107B8800C022002080610040505C00400A30002084
:107B9800045C0040014B1868C0B270477C2200208A
:107BA8000120704770477047054B1A7802F0FF01B3
:107BB80022B10122027000221A70704701707047CA
:107BC800A00F0020F7B51C4B1A680AB91C6800E022
:107BD80001241A494E780022D0B2A04202F10102D3
:107BE80007D202AD2F18164D3544285C07F8040C4F
:107BF800F2E71A68121B1A604A781D6822444A7014
:107C08009DB903204021FDF701F90E4A136823F4BA
:107C1800804323F070039BB283F4405343F4004342
:107C280043F080031360054B5D70002CCBD09DF8AA
:107C3800040003B0F0BD00BF7C220020A00F00208C
:107C4800802200200C5C004013B504460621432026
:107C58006A4603F0DDFCA8B19DF800209DF80130CC
:107C680043EA022323809DF802209DF8033043EA6B
:107C7800022363809DF804209DF8053043EA02231F
:107C8800A380012002B010BD13B5044606213B2095
:107C98006A4603F0BDFCA8B19DF800209DF80130AC
:107CA80043EA022323809DF802209DF8033043EA2B
:107CB800022363809DF804209DF8053043EA0223DF
:107CC800A380012002B010BD0F4B9A7813B51C4653
:107CD800BAB90E4B1B68A3B11A681AB10C494869A6
:107CE80002434A619A88ADF8042002228DF80720E1
:107CF8009868002201A98DF8062002F0E7FE01230A
:107D0800A37002B010BD00BFA00F0020E402002045
:107D18000010024008B5FFF7D7FF80216B2003F061
:107D28001BFC642002F047FA03216B2003F014FCCB
:107D38000D4B1920197803F00FFC0F2002F03BFAC5
:107D48000A4B1A20197803F007FC18211B2003F0AE
:107D580003FC10211C2003F0FFFB37200021BDE8A5
:107D6800084003F0F9BB00BFE90200200000002032
:107D780008B5FFF7A9FF074B1B7813B1012B03D0F8
:107D880008BD4FF4006201E04FF48052024B1A80A4
:107D980008BD00BFE8020020020000202DE9F041E4
:107DA8000369C76805460E461F40002F35D0B7FA4D
:107DB80087F24FF00043D340DB432B611F40A2F111
:107DC8001B03042BF1D8DFE803F0221F1C19030062
:107DD800746A24B1013C0023A4B2736201E0EC6A26
:107DE800A4B2D6F82080B8F1000FDED0D8F8003061
:107DF800404621469847D8F80480F4E73068696B14
:107E080007E07068A96B04E0B068E96B01E0F0680E
:107E1800296C036889B29847C7E7BDE8F0810F4B22
:107E28001A78692A16D15A88B2F5DE6F12D11A79F2
:107E3800BE2A0FD193F8EE26EF2A4FF000000BD19F
:107E480013F8012B5040064A9342F9D1B0FA80F05A
:107E58004009704700207047704700BF00F80308CA
:107E6800F0FE03082DE9F04F2DED028BE74C85B0AD
:107E780000214FF4DE62204607F013F8E44B04F5C6
:107E880009721A60E34B00251D70E34B04F2CA62C5
:107E98001A60692323704FF4807003236371FDF720
:107EA80073FF4FF416732022A4F8663184F86A2110
:107EB800FA236E22A4F8683184F87C21BC230A22B4
:107EC800A4F8643184F87D214FF4FA732B22A4F8C6
:107ED8006E3184F87F210123212284F8623184F8ED
:107EE8007E3184F8802184F886312322002384F8A7
:107EF8008121C4F818324FF4C872C4F81C32052323
:107F080084F8C856A4F87251A4F87051A4F87451B2
:107F180084F8585184F8595184F85A51A4F85C519E
:107F2800A4F85E51A4F8605184F8635184F86B5149
:107F380084F86C51A4F88451A4F88221A4F88851DB
:107F480084F8155284F8145284F8205284F82332A5
:107F580040F2DC53A4F8983140F24C43A4F89A312B
:107F680040F26C73A4F89C3140F27533A4F89E314A
:107F780040F6430384F8215284F8225284F892513F
:107F880084F89351A4F8A03122462B462546032BAA
:107F9800CCBF0121002103F1010382F8A21114BF13
:107FA8001E217521122B82F8A31102F10202EED1D3
:107FB8004FF4FA63A5F8C831A5F8CC31A5F8D0314B
:107FC800A5F8D43140F27E41052340F27E5E85F863
:107FD800E231A5F84411C82340F23A71A5F84CE102
:107FE800DFF82C82A5F8E63140F2EA5E0026012788
:107FF8004FF47A791E2019224FF4C8734FF0320BD0
:10800800A5F84611A5F84EE140F2DC5140F2B45E05
:1080180085F89501039085F8E3210192A5F8EA31E6
:10802800A5F84A110291A5F850E185F8946185F800
:108038009661A5F8C691A5F8CA91A5F8CE91A5F8BC
:10804800D29185F8D66185F8E06185F8E17185F807
:10805800E47185F8E57185F8E87185F8EC6185F8D3
:10806800EE71A5F84891A5F852B1A5F85431A5F8D4
:1080780056B103F09BFCD8F8003003982F74EF73C7
:10808800AE73AE81D87218735520019AD8700F203C
:108098005871DA712220212298715A740E205322C5
:1080A8004FF0170E1874DA7635200A224FF0280A96
:1080B80083F815E083F816E098764FF02D0E5A20D5
:1080C8009A740192642283F80DE018721A771E7070
:1080D80083F801A083F802A0DE7583F804B09E73CC
:1080E8001E76DE735E7683F809A083F814E04FF4F9
:1080F800FA7EA3F84EE04FF03C0E83F851E04FF0C3
:10810800110E83F850E0DFF828E1C3F838E0C3F82F
:108118003CE0DFF820E1C3F828E04FF0780CDFF806
:1081280018E183F80AC0C3F834E0DFF810C1DFF8BB
:1081380010E19FED3A8AC3F82CC0C3F830C0C3F8E9
:1081480048E0F7EE087ADFF8FCC002999F774FF015
:108158004B0E83F85260C3ED087AC3ED097A83EDBC
:10816800108AC3F844C083F84CE085F8CA06A5F81D
:10817800D4164120042185F8CB0685F8CCB685F8BD
:10818800CD6685F8D16685F8D26685F8CE6685F81D
:10819800CF6685F8D066A3F85860A3F85A60A3F8AC
:1081A800566083F85C10152183F868101C49D9665D
:1081B8001C4919671C495967C3F860C083F864A053
:1081C80083F865A083F87870184803F03EFCD8F867
:1081D8000010019A81F811614FF44873A1F8163123
:1081E800C82381F8126181F813A181F8147181F80C
:1081F800186185F8D931642385F8D821A5F8DA9172
:1082080085F8DC61A5F8DE310A461DE0CC1A0020AD
:10821800F40E0020E4210020E821002000000000E6
:108228009A99193FF6287C3F3D0A773F852B01082C
:108238008FC2F53C000060406666663FCDCCCC3E00
:10824800000040400000A0400E2303FB06136FF01F
:10825800170083F81901032083F81A016FF02F0023
:1082680083F81B01072083F81C016FF0230083F8B3
:108278001D01052083F81E01642382F81F31013691
:108288005A2382F8203182F82131082E4FF0FF035B
:1082980082F8223102F10E02D6D1002381F8893109
:1082A8004A4B84ED058A10349C42FAD10820484C88
:1082B800484FFDF769FD1020FDF766FD4023A4F83F
:1082C8000432052384F893314FF47A73A4F84431C7
:1082D8004FF4FA63A4F846314FF4FA43A4F8543142
:1082E800D8F80030142201250021032084F87C21CD
:1082F800A18184F8925125741870242058709870C0
:108308003B6884F8D911022684F8D86182215A7111
:108318001A71642219709A712F4803F096FBD8F8E5
:1083280000802E4A2E482F49A0614FF07E532262CA
:10833800A062E262A163A164E2642265A265E065CD
:108348002266E066A267E167C4F88C10C4F8902042
:10835800414604F56C704FF4C6726361E361636271
:1083680023636363E3632364636463656366A3668B
:1083780023676367C4F88030C4F88430C4F8883051
:1083880006F084FD04F23C5041464FF4C67206F0F4
:108398007DFD3B681A68C4F8D6265A68C4F8DA2600
:1083A8009A68C4F8DE261A68C4F8E2265A68C4F83F
:1083B800E6269A68C4F8EA2684F8045484F8906596
:1083C80005B0BDEC028BBDE8F08F00BF8C1B002010
:1083D800CC1A0020E82100208E2B0108000080BF65
:1083E800240FD4BE240FD43E1549D1F8883043F465
:1083F8007003C1F88830134B1A6842F001021A6002
:108408005868114A02405A601A6822F0847222F4AD
:1084180080321A601A6822F480221A605A6822F49C
:10842800FE025A60DA6A22F00F02DA62186B074A13
:1084380002401A6300229A604FF000638B60704715
:1084480000ED00E0001002400CC07FF8CCFC00FFFB
:1084580007B5232001F0AFFE752001210DF10702B9
:1084680003F0D6F828B19DF80700A0F16803584238
:10847800584103B05DF804FB014802498EE400BF8F
:1084880000480140C81800200148024986E400BF9E
:1084980000400140A0180020014802497EE400BFC6
:1084A80000040040781800204FF08040004975E42F
:1084B800501800200148024970E400BF002C014018
:1084C800281800200148024968E400BF002C014038
:1084D80028180020224B10B5224C5A43224BB3FBDC
:1084E800F2F203880139013AA04289B292B29BB2F2
:1084F8000ED004F50064A0420AD0B0F1804F07D036
:10850800A4F59834A04203D004F58064A04202D1B7
:1085180023F070039BB2154CA04206D004F580648A
:10852800A0421CBF23F440739BB203800D4BC16271
:10853800984202850FD003F5006398420BD003F5EB
:108548004063984207D003F58063984203D003F54F
:108558008063984201D1002303860123436110BD43
:1085680040420F00002C014000A24A0400100040C5
:108578000E4B800A984216D007D8B0F5801F0CD051
:108588004A3B98420DD102207047094B984206D0C9
:108598000233984205D10420704701207047032018
:1085A8007047FE2070470020704700BF4B00100046
:1085B80050001000F8B50468064620460F461546D8
:1085C800FFF7D6FF04284BD8B27A910847B902239F
:1085D8008B40D4F80CE0DB439BB203EA0E03E36064
:1085E8000A23204A03FB001342F82370043342F89D
:1085F800235015463FB1B17AE268890802238B40BF
:108608009BB21343E360282202FB00522032EFF3AF
:108618001286502383F3128803B203EB8303DB0033
:1086280003F10C011C3329442B4451F8047F17B182
:1086380017600A6804329942F7D100231360F3B235
:1086480083F31188282303FB0050036A1BB1E368F6
:1086580043F0010303E0E2684FF6FE731340E36062
:10866800F8BD00BF28180020014800F045BF00BF32
:10867800A40F0020014800F03FBF00BFF80F002002
:10868800014800F039BF00BF4C100020064B1B7892
:1086980003F0040303F0FF001BB1044B1888C0F378
:1086A800C01000F001007047ED2200202C170020B8
:1086B8002DE9F04F2DED028B87B000250493BF4BB9
:1086C8000391B3F90280B3F900300292B8F1000FB8
:1086D800B8BFC8F10008002BB8BF5B429845B8BFC7
:1086E8009846B8F5FA7F0746A8BF4FF4FA7882464D
:1086F800A9460195AB462C46B14E338899074FD011
:10870800AE4B33F91420029B52005B429A424FEA67
:10871800440103DB029B9342A8BF1346A94A8A5E21
:108728009B1A049A32F91420134408EE103AFFF702
:10873800ADFF68B1B8EEC80AA34BB2EE048A80EE6A
:10874800080A185D03F014F820EE080ABDEEC08A86
:1087580018EE102A3B7A5343642293FBF2F33A7FD4
:108768006FF0040B0BFB02FB5B4504DB02EB820B97
:108778009B45A8BF9B46954A18EE103A52F824101C
:108788000B4442F210718B42A8BF0B4690498B42B2
:10879800B8BF0B4642F82430BA7C53431B130193ED
:1087A800368806F00303012B37D0844B894933F907
:1087B8001490894B9AF801C033F9140051F824E059
:1087C80080EAE073A3EBE073B3F5206F4FEA84050A
:1087D80016DC09EB89031A0192FBFCF3042290FBD7
:1087E800F2F0181A8644BEF57A5FA8BF4FF47A5E95
:1087F8007A4B9E45ACBF41F824E041F8243002E0B2
:10880800002341F824304B597D2593FBF5F59AF860
:108818000B306B43402593FBF5F5B20711D5019852
:10882800C8F5FA7208FB09F308FB05F64FF4FA716C
:1088380002FB0B3302FB006693FBF1F396FBF1F6A8
:1088480005E0F3074DBF019E2E464B465B46624A44
:1088580032F91410042291FBF2F26149615C4A4337
:108868006FF04F0192FBF1F297F8511013444FEA61
:10887800440C08EE103A79B15A4B5B48D3ED000A24
:10888800CDF814C0B8EEC80A00EBC400FCF70EFF20
:10889800DDF814C0BDEEC08A4F4B544A3CF80300C3
:1088A8003CF902302CF8020001B2101D0C32CB1A30
:1088B80050F824E0042193FBF1F152F8243040F8F9
:1088C800241073440B4497F8501042F824E000EE4B
:1088D800103A79B1434B4648D3ED000ACDF814C09D
:1088E800B8EEC00A00EBC400FCF7E0FEDDF814C0E7
:1088F800BDEEC00A18EE103A3E493F4A095D3344BE
:108908001E4610EE103A4B43202193FBF1F3F61A62
:108918002CF802600AF1010A0CB90124ECE6274B95
:108928002C48B3F90410039B85689B790F335B00CF
:108938004B4329495B11B1F90440797B002BA3EB28
:108948000404B8BF5B42322B0BDC2C4B01FB0451F7
:108958008B42A8BF0B462A498B42ACBF836081601B
:1089680001E000238360F97801FB04F325490978C5
:1089780003294FEAA3130CD9B7F84E10B1F5FA7FC3
:1089880007D24C42A34203DB8B42A8BF0B4600E050
:108998002346816841F34F31B1F5807FA8BF4FF47A
:1089A80080716FF0FF008142ACBF5B181B18938089
:1089B80007B0BDEC028BBDE8F08F00BF2E1700207A
:1089C8002C1700209A1A002060120108A01000201D
:1089D800F0D8FFFF5C1700203617002080C1FFFF8A
:1089E800D01700205817002040170020A81000209A
:1089F8008C170020D3170020A4170020FEFFFF0FBC
:108A0800020000F0D61700202DE9F04F2DED028B63
:108A180085B083460293AC4B01911C88009204F008
:108A28000204A4B294B1A94BB3F90240B3F90030DF
:108A3800002CB8BF6442002BB8BF5B429C42B8BF51
:108A48001C46B4F5007FA8BF4FF40074D946002532
:108A58009E4B9F4833F915109E4B50F8256033F90B
:108A6800153083EAE37EAEEBE37EBEF5206F4FEA76
:108A780045084FEA41074FEA850A12DC4FF0040E19
:108A880093FBFEF3FB1A1E44B6F57A5FA8BF4FF4BA
:108A98007A56914B9E42ACBF40F8256040F825308D
:108AA80002E0002340F8253050F80A6099F80B30AE
:108AB800F6115E4399F801305F43834B1B889B078F
:108AC8004FEAA6164FEAA71751D0009B49005B4210
:108AD800994203DB009B8B42A8BF0B467F4938F9BC
:108AE8000110591A029B33F91530CB1808EE103AC9
:108AF800FFF7CCFD68B1B8EEC80A794BB2EE048A2C
:108B080080EE080A585D02F033FE20EE080ABDEE3A
:108B1800C08A744874495AF8003018EE102A42F294
:108B2800107E13447345A8BF73468B42B8BF0B46EB
:108B38004AF800309BF808109BF81C00514300EBE2
:108B48008000C911C0F1000E714503DB8142A8BF46
:108B580001468E469BF812104B431B13F61ACEEBB8
:108B680007076643674303EB66260EEB6727594BF7
:108B7800042138F9030090FBF1F15C48405D414362
:108B8800A7EBA1129BF8511008EE102A69B15848BA
:108B9800584F0393B8EEC80A00EBC500D7ED000A9A
:108BA800FCF784FD039BBDEEC08A534933F80830B7
:108BB80038F9010028F801300FFA83FEC0EB0E0ED9
:108BC80004209EFBF0F001F1040E0C315AF80E70EF
:108BD8005AF801304AF801703B449BF850104AF8A3
:108BE8000E00034400EE103A59B1424B4348D3ED0E
:108BF800000AB8EEC00A00EBC500FCF757FDBDEE51
:108C0800C00A3F4A10EE103A575D3E4A18EE101A55
:108C18007B433144A1EB631628F8026009F101098E
:108C28000DB9012514E7294B2948B3F90410019B14
:108C380084689B790F335B004B4326495B11B1F97C
:108C480004509BF80D10002BA3EB0505B8BF5B4241
:108C5800322B0BDC01FB05442B492C4BA142A8BF4E
:108C680021469942ACBF8160836001E000238360A4
:108C78009BF8031001FB05F32549097803294FEAFE
:108C8800A3130CD9BBF84E10B1F5FA7F07D24C42AA
:108C9800A34203DB8B42A8BF0B4600E02346816852
:108CA80041F34F31B1F5807FA8BF4FF480716FF069
:108CB800FF008142ACBF5B181B18938005B0BDEC68
:108CC800028BBDE8F08F00BF2C1700202E17002064
:108CD8005C1700203617002080C1FFFF9A1A002079
:108CE80060120108A0100020F0D8FFFFD017002064
:108CF8004017002058170020BC1000208C170020B7
:108D0800D3170020A4170020FEFFFF0F020000F079
:108D1800D61700202DE9F04F2DED028B85B00025E8
:108D28000393A94B0292B3F90270B3F90030009093
:108D3800002FB8BF7F42002BB8BF5B429F42B8BF2D
:108D48001F46B7F5FA7F8146A8BF4FF4FA77A846C1
:108D58000195AA462C469D4E3388990757D0022C78
:108D680055D0994B33F91420029B52005B429A422A
:108D78004FEA440103DB029B9342A8BF1346944A7F
:108D880031F902B0039A32F91420CBEB030303EB59
:108D9800020BFFF77BFC88B107EE90BA8D4BB8EE5B
:108DA800E70AB2EE048A185D80EE080A02F0E0FCD9
:108DB80020EE080AFDEEC07A17EE90BA99F808304E
:108DC80099F81C10642203FB0BF393FBF2F36FF08A
:108DD800040202FB01FA534505DB01EB81029342D1
:108DE800A8BF13469A467C4951F8243042F21070C5
:108DF8005B448342A8BF034678488342B8BF034612
:108E080041F8243099F812104B431B13019333880F
:108E180003F00301012901D1022C42D1704D6A49A6
:108E280035F91450009A6F4831F9148092F801E02E
:108E380050F8242085EAE576A6EBE576B6F5206FAE
:108E48004FEA840120DC022C18D008EB88000001CE
:108E580090FBFEFE042095FBF0F5C5EB0E0E02EB31
:108E68000E0CBCF57A5F5F485F4DA8BF4FF47A5C83
:108E7800AC45ACBF41F800C00D5007E088EAE87681
:108E8800A6EBE876642EE0DD002545505548009AAB
:108E980009587D2591FBF5F5D17A6943402591FB69
:108EA800F5F59A0713D5022C11D0019AC7F5FA7374
:108EB80007FB05F607FB08F103FB0A114FF4FA70EC
:108EC80003FB026391FBF0F193FBF0F608E0DB078C
:108ED80004D5022C02D0019E514601E02E4641469F
:108EE8003F4B042033F9143093FBF0F33F48205CE8
:108EF80043436FF04F0093FBF0F3CB1899F85110F0
:108F08004FEA440B08EE103AB1B1022CB8EEC80A89
:108F1800374B08D1480803D08142A8BF014600E07A
:108F28000121344802E0344800EBC400D3ED000AC4
:108F3800FCF7BCFBBDEEC08A294B30493BF803E087
:108F48003BF901002BF801E00FFA8EF301F1080E4E
:108F580014311B1A5EF82420042093FBF0F051F81A
:108F6800243041F82420134499F850104EF8240076
:108F7800034400EE103A59B11D4B2148D3ED000AC5
:108F8800B8EEC00A00EBC400FCF790FBBDEEC00AC7
:108F980018EE103A1B493344095D1E4610EE103A8C
:108FA8004B43202193FBF1F3F61A174B2BF8036080
:108FB800009B01340133032C00937FF4CCAE05B041
:108FC800BDEC028BBDE8F08F2E1700202C17002077
:108FD8009A1A002060120108A0100020F0D8FFFFA4
:108FE800361700205C17002080C1FFFFD017002033
:108FF800581700205017002040170020D0100020DC
:109008008C170020D3170020A41700202DE9F04F5B
:1090180099462DED088BD54B09EE902A1A8883B016
:1090280012F0020F04460193B7EE009A4CD0149B3D
:10903800CF48DD89B0F900305B1B03F2F31640F22C
:10904800E632964203D8002BB8BF5B4201E04FF4EA
:10905800FA73B0F90220521B02F2F31540F2E6301F
:10906800854203D8002AB8BF524201E04FF4FA7291
:1090780094F84C0058B39342B8BF1346C3F5FA733B
:1090880007EE903A9FEDBB7AF8EEE77A6423C7EED5
:10909800877A93FBF0F307EE103A77EEC97AB8EEC9
:1090A800C77AF0EE498AE7EE878AF7EE006AF5EEAE
:1090B800C08AF1EE10FA0AD4F4EE668AF1EE10FADC
:1090C800C8BFF0EE668A04E0F0EE498A01E0DFED01
:1090D800AA8ACF1C25464FF0000ABAF1020F17F8EA
:1090E80001BFDFF8DC824FEA4A06B2EE04AA0ED1CD
:1090F800B8F904209FEDA17A0BF10A0B02FB0BF3E0
:1091080007EE903AF8EEE77AC7EE877A5FE038F92B
:109118001A30DFED986A07EE103AF8EEC77AB8EE23
:10912800697A19EE903A87EE267A5B4227EE877ABB
:1091380007EE903AF8EEE77AB4EEE77AF1EE10FA35
:1091480008D4F8EEE97AB4EEE77AF1EE10FAD8BF6F
:10915800F0EE477A8A4B9B5F08EE103A39F91A30DD
:10916800B8EEC88A77EEC87A08EE103AB8EEC88A20
:1091780037EE888A88EE0A8AFFF788FA40B1814B71
:1091880013F80A00B0EE480A02F0F2FAB0EE408A8C
:10919800019B1A88D10704D5D4ED117A68EE277A95
:1091A80015E038F906309FED757A0BF1140B03FBC7
:1091B8000BF307EE903AF8EEE77A9307C7EE877A53
:1091C80042BF94ED127A28EE078AE8EE287A6E4BB1
:1091D800DFF8F0B19B5FD5ED08AA94F85110DFF8DD
:1091E800E88107EE103A694BB8EEC77AD3ED186AF2
:1091F8001AF80B30E7EE667AB0EE678A67EEAA7A5D
:109208000AEE903AF8EEEAAA67EEAAAADFED607ACB
:10921800CAEEA7AAB0EE67BAC1B1BAF1020F0AD175
:109228004A0803D09142A8BF114600E00121B0EEE0
:109238006A0A584804E05848B0EE6A0A00EBCA00C7
:10924800D8ED000AFCF732FAF0EE40AAD8ED000A91
:10925800524995ED0B7A4FEA8A0268EE207A11445A
:1092680067EE877A91ED000AA7EE8A0ADFED4C7A5D
:10927800B4EEE70AF1EE10FAB0EE40AA09D4DFED39
:10928800497AB4EE670AF1EE10FAC8BFB0EE67AAE1
:1092980001E0B0EE67AAC9EE207A434B81ED00AA3F
:1092A800991891ED007A81ED008A38EE477A03F13A
:1092B8000C011144183327EE277A1A44D1ED007AAD
:1092C80092ED000A81ED007AC2ED007A37EE800A4D
:1092D80094F8501030EE070A21B1344800EBCA0068
:1092E800FCF7E4F9B0EE087A80EE070A1BF80A30BA
:1092F800D5ED0E7A20EE277A07EE903AF8EEE77A67
:1093080067EE277A9FED2A7AC7EE8B7AF4EEC77A52
:10931800F1EE10FA09D49FED277AF4EE477AF1EED0
:1093280010FAC8BFF0EE477A01E0F0EE477A3AEE5D
:109338008A0A0AF1010A30EE270A05F0C1FF1E4B1E
:10934800B0F57A7FA8BF4FF47A709842B8BF184634
:109358001A4BBAF1030F985305F104057FF4BDAE1B
:1093680003B0BDEC088BBDE8F08F00BF2C170020C0
:10937800E80C00200000FA4300000000000048420A
:109388009A1A00206012010836170020A010002049
:109398000000C8425017002040170020BC170020CA
:1093A80000007AC300007A43041100208C170020C3
:1093B800000096C30000964318FCFFFFA417002086
:1093C8002E1700203C17002058170020044B0022BD
:1093D8001A605A60034B00221A605A60704700BF37
:1093E800A0100020C817002010B50C4C0123E37012
:1093F8004FF48060022384F82030FCF7ADFC084A63
:10940800084BD2F888201B685178642212FB01337C
:10941800636123880133238010BD00BF142200201C
:10942800A0100020C41A0020026BC168034610B5C2
:10943800406942B11A6C8C1A013A005D08BF0A46AD
:10944800C0B21A6410BD1A6A805C01328A4228BF11
:109458000022C0B21A6210BD436B13B190F84400E9
:109468007047836A406A1B1A584258417047036B19
:1094780013B15B68016C01E0C369016A8B423CBFB0
:10948800C2689B18581AC0B27047836A8169426BD8
:109498001944D160416A99429DBF0169CB1A536052
:1094A800CB1A96BF0023536083624FF0000380F805
:1094B8004430136888BF816243F00103136070472A
:1094C800436A8269D154436A02690133934228BFCF
:1094D80000234362436B1BB11B68DB0705D4D4E749
:1094E800026D136843F0800313607047417101F007
:1094F8008BB9816001F088B9026D036B70B50446C1
:10950800D5699BB9A90611D5C36A1BB1908C80B2E5
:1095180098470BE0E169928C40694E1CD2B2E66133
:109528004254E169E268914228BFE361616BA1B9E5
:109538002A0612D5636AA26A9A42236D09D0501C82
:10954800A669A062B25C1A852369984205D3A16214
:1095580003E01A6822F080021A602B0742BF236DCD
:1095680008221A6270BD0D4B0D484FF400525A6024
:109578000C4A11684FF6FE730B401360426B11687A
:109588004FF6FE730B401360426A836A9A4200D01A
:109598007BE7012380F84430704700BF0000024099
:1095A8004C100020440002402DE9F0471E46A14B14
:1095B8008CB09842894690469DF850507ED19E4B7B
:1095C8009E4A1A609E4A5A6102F580729A614FF467
:1095D8008072DA601A619B4A1A63143A5A63A2F5D8
:1095E8004842203ADA6404329A64C3F8088018655D
:1095F800954B9A6942F480429A615A6942F0010295
:109608005A6102238DF80830032315F0010A8DF8FA
:1096180009304FF000038DF80A3014BF02230123EC
:109628002C078DF80B3017D5884C402701978AF006
:1096380001038DF80A30236A23F070632362236ADA
:1096480043F0E0632362204601A9FBF7ABFEBAF1C1
:10965800000F23D1A76121E0B0070ED50CA9402344
:1096680041F82C3D7948036A23F070630362036A6A
:1096780043F0E0630362FBF795FEF1070ED50CA9F2
:10968800802341F82C3D7148036A23F0704303623C
:10969800036A43F0E0430362FBF784FE0E238DF870
:1096A80000300022012368468DF801308DF8022031
:1096B8008DF80330604C02F011F808E1644B9842D1
:1096C80074D1644B5D4A1A604FF48072DA601A6193
:1096D800614A5A6102F580729A615B4AC3F8088050
:1096E8001865D36943F40033D36102238DF8083039
:1096F800032315F0010A8DF809304FF000038DF8A7
:109708000A3014BF022301232A078DF80B3019D51C
:109718004FF09044042701978AF001038DF80A302E
:10972800236A23F470632362236A43F4E0632362A9
:1097380020460DEB0701FBF735FEBAF1000F25D1E6
:10974800A76123E0B3070FD50CA9042341F82C3DEA
:109758004FF09040036A23F470630362036A43F492
:10976800E0630362FBF71EFEF7070FD50CA9082379
:1097780041F82C3D4FF09040036A23F47043036294
:10978800036A43F4E0430362FBF70CFE26238DF8DB
:1097980000300022012368468DF801308DF8022040
:1097A8008DF803302B4C01F099FF90E02B4B984239
:1097B80040F006812A4B214A1A604FF48072DA6021
:1097C8001A61284A5A6102F580729A611E4AC3F8E2
:1097D80008801865D36943F48023D36102238DF888
:1097E8000830032315F0010A8DF809304FF0000303
:1097F8008DF80A3014BF022301232C078DF80B3093
:1098080032D5124C4FF4806701978AF001038DF826
:109818000A30636A23F470636362636A43F4E06343
:109828006362204601A9FBF7BDFDBAF1000F3FD1E5
:10983800A7613DE0003801404C10002048120108A3
:109848002C1100205800024000100240000400487B
:1098580000440040F80F00202C130020004800406E
:10986800A40F00202C150020B0070FD50CA94FF429
:10987800806341F82C3D5448436A23F47063436283
:10988800436A43F4E0634362FBF78CFDF1070FD5AD
:109898000CA94FF4006341F82C3D4B48436A23F46C
:1098A80070434362436A43F4E0434362FBF77AFD43
:1098B80027238DF800300022012368468DF80130F7
:1098C8008DF802208DF8033001F008FF3F4CC4F8F2
:1098D8002C900027012384F844302762E761A762AF
:1098E80067626671C4F80880A571204600F08CFF95
:1098F800F2072FD5206B30B3E36C01934FF48053FC
:109908000A9380230693E368ADF810302023099367
:109918006369029303970597079708970B97FBF7D7
:1099280047FB01A9206BFBF725FB236B216D1A6808
:1099380042F001021A608A6842F040028A605B685D
:109948009BB2236406E0236D20221A621A6842F053
:1099580020021A60B3072CD5606B28B3A36C01935F
:109968004FF480530A93802306932369ADF810308F
:1099780000251023039302950595079508950995E9
:109988000B95FBF715FB606B01A9FBF7F3FA636B0B
:109998001A6842F002021A60226D5D605D60936889
:1099A80043F08003936004E0226D136843F0800362
:1099B8001360226D136843F001031360204600E032
:1099C80000200CB0BDE8F08700040048A40F002078
:1099D8004FF09043202208B19A6170471A8570476A
:1099E8004FF09043202208B11A8570479A6170475A
:1099F8002DE9F04F2DED028B87B006460593984B65
:109A0800B3F800A00AF002081FFA88F393460393FC
:109A1800B3B3129B9348DC89B0F900301B1B03F2E7
:109A2800F31540F2E632954203D8002BB8BF5B42EB
:109A380001E04FF4FA73B0F90220121B02F2F3149A
:109A480040F2E630844203D8002AB8BF524201E00F
:109A58004FF4FA729342B8BF1346C3F5FA7305225E
:109A680093FBF2F30A22643B5343327FD2105343F1
:109A7800642293FBF2F3134423EAE373DBB200E0BE
:109A88006423019301F1030937464FF00008B8F148
:109A9800020F19F8014F06D1714AB2F906201B349A
:109AA8005443621142E0704A32F91850CBF1000277
:109AB800690091424FEA480003DB59450A46A8BFAE
:109AC8005A466A49059B415E511A33F918208B188A
:109AD80008EE103AFEF7DAFD70B1B8EEC80A644A2B
:109AE800B2EE048A80EE080A12F8080001F040FE7F
:109AF80020EE080ABDEEC08A1AF0010F11D11B34FE
:109B0800039B6C4322118BB1B17C9DF9040018EEC4
:109B1800103A59434143642091FBF0F102EB2112C2
:109B280004E0347A18EE103A5C4322114C4D05F1EA
:109B38000A01042431F9181091FBF4F4141B05F1FF
:109B480010024FEA4803049318F802307A78029317
:109B580062435A43642192FBF1F296F85110D311F3
:109B680008EE103AB9B1B8F1020FB8EEC80A08D138
:109B78004A0803D09142A8BF114600E001213D48A0
:109B880003E005F1140000EBC800D5ED0B0AFBF764
:109B98008DFDBDEEC08A324B374AFD7A108803F13D
:109BA800300C00FB04F25CF82810D21205FB0215F9
:109BB800B5F5001F314AA8BF4FF4001503F13C0169
:109BC8009542B8BF154651F8282041F82840A21AF6
:109BD8004FF6FF7103F154040009B1FBF0F0424362
:109BE80003F148004CF8285054F8281050F828C0C1
:109BF80044F828C092116144114400EE101A96F8F6
:109C0800501040F828206D1359B103F16000B8EEE8
:109C1800C00A00EBC800D3ED0B0AFBF747FDBDEE09
:109C2800C00A18EE103A2B44797D029A1D4610EEB0
:109C3800103A59434A43049B642108F1010892FBF6
:109C4800F1F10F4A05EB2121B8F1030F995207F101
:109C580001077FF41CAF07B0BDEC028BBDE8F08FA5
:109C68002C170020E80C00202E1700209A1A00203C
:109C78006012010850170020642200200000E0FF55
:109C8800A41700202DE9F04F2DED0A8B87B004466C
:109C9800049390F85030039102921BB1322BA8BF65
:109CA800322300E0012307EE903AF8EEE7BADFED41
:109CB800D67AD64B9FEDD6CA1B88D64AC7EEABBA22
:109CC800002B08BF012307EE903AF8EEE79A1388B5
:109CD800009329EE8CCA03F002077BEE8CBABBB264
:109CE800CCEE2BBA019333B3B2F90230B2F90420A7
:109CF80083EAE37182EAE270A1EBE371A0EBE27020
:109D080088420546B8BF0D46B5F5E17F16DA8842A8
:109D18009FEDC1BA05DD002AD8BF524207EE902A4E
:109D280004E0002BD8BF5B4207EE903AF8EEE77AE2
:109D380087EE8BBA04E09FEDB9BA01E0B7EE00BA3E
:109D4800DFF80CA39FEDB59A0AF108090AF1100B88
:109D580026460AF11C050027F0EE49AAB04931F958
:109D680017300AEE103AB8EECAAAF5EE047A0839A6
:109D78002AEE27AA31F91730BDEECAAA08EE103A22
:109D8800009BF8EECA7A9FEDA7AA9A074FEA470800
:109D980027EE8AAAB8EEC88A75D078EE087A029BB0
:109DA800FDEEE77A594217EE900A884203DB8342B8
:109DB800A8BF034619469C48049B38F90000091AB5
:109DC80033F91700014407EE901AF8EEE78AFEF718
:109DD8005DFC48B19549B2EE049A88EE890AC85DDF
:109DE80001F0C6FC60EE098A237FDFED916A0AEE76
:109DF800903A237A07EE903AF8EE677AF8EE6AAA74
:109E080068EEA77AB1EE047A67EEA67A2AEE877A28
:109E1800FDEEE77A17EE901AF1EE477AFDEEE7AA23
:109E28001AEE903A994208DBFDEEC7AA1AEE903A6C
:109E38008B42A8BF0B460AEE903AD5ED007AE8EEC1
:109E48008C7ABBEE0E7AF4EEC77AF1EE10FAF8EEE1
:109E5800EAAA09D4B3EE0E7AF4EE477AF1EE10FAD4
:109E6800C8BFF0EE477A01E0F0EE477AC5ED007A18
:109E7800A37C09EE103AB8EE499A67EE897A9FED0D
:109E88006D9A27EE899A009BDB0750D4644938F90C
:109E980001100029B8BF4942B1F5206F03DD002148
:109EA800CBF8001025E09FED647A737868EE077AA6
:109EB80007EE103AB8EE477A87EE877ADBED007A3C
:109EC80037EE4A7AE7EE0C7A9FED5C7AF4EEC77AC1
:109ED800F1EE10FA09D49FED5A7AF4EE477AF1EED2
:109EE80010FAC8BFF0EE477A01E0F0EE477ACBED02
:109EF800007AF37ADBED008A00EE103AB8EE400AF9
:109F0800019B20EE280ADFED4F8A60EE288A93B184
:109F180038EE6A8AF0EE6A7AEBEE087A38EEC90A09
:109F2800F0EE498AB0EE678AEBEE008A03E0F0EEC5
:109F3800498AB0EE6A8A374B9FED437A03F1A40150
:109F4800B0EE480A7A5C94F8511007EE902AF8EEC1
:109F5800E77A67EECA7AA7EE870A39B103F11400E7
:109F680000EBC700D3ED0B0AFBF7A0FBDAED007A94
:109F78002849D9ED006A05917AEE677A01F1A700C0
:109F8800C7EE8C7A3B5C0BF1040B0136043530EEDE
:109F9800280A77EEE67AAAEC01AAEBEEA76A07EEA2
:109FA800903AB8EEE77AE9EC016A67EE667A9FEDD7
:109FB800277AA7EE870A05F083F9059901F1780E4B
:109FC8002EF8080088460FB90127C7E6039AB1F9A9
:109FD800063095796D0028355D43B1F90E3000EEF5
:109FE800103ABAEECF0A05F06BF96D11281A002D58
:109FF80007EE900AB8BF6D42322DF8EEE76A2BDD06
:10A008000023C8F8383050E083F9223E642200204B
:10A01800BD3786352C1700200000E1430000000002
:10A0280036170020CDCC4C409A1A00206012010847
:10A038006F12033C0AD7A33D0000A043000040C3B1
:10A04800000040430AD7233CA69B443BF7CC9238F8
:10A05800AC17002000803B45FDEEE99A19EE903AD6
:10A0680023F0030307EE903AF8EEE79A5FED077ADC
:10A07800637BC9EEA77A07EE103AB8EE477AD8F8AC
:10A08800383026EE877A67EE277AFDEEE77A17EE04
:10A09800902A1344314A9342A8BF1346304A934248
:10A0A800ACBFC8F83830C8F83820D8F838305B1357
:10A0B800B3F5807FA8BF4FF480736FF0FF0293421F
:10A0C800B8BF134607EE903AB8EEE78AFDEEE67A97
:10A0D800E27817EE903A53439B1100EE103A98F845
:10A0E800AA30032BB8EEC00A14D9B4F84E20B2F542
:10A0F800FA7F0FD2FDEEC07A534217EE901A9942BA
:10A1080004DB914217EE903AA8BF134607EE903A47
:10A11800B8EEE70A94F8511059B14B0803D09942A8
:10A12800A8BF194600E001210E48D8ED0B0AFBF73D
:10A13800BDFA30EE080ABDEEC00A8DED000ABDF981
:10A14800003000EE103AB8EEC00A05F0B9F8A8F8E9
:10A158007C0007B0BDEC0A8BBDE8F08FFEFFFF0F57
:10A16800020000F05017002010B50A4A0A4B116887
:10A178009B6800BF12689142F7D1084AD2F8AC40F8
:10A188004FF47A7000FB04F2D31AB3FBF4F300FB2C
:10A19800013010BDC41A002010E000E02C17002088
:10A1A80038B50446FFF7E0FF0546FFF7DDFF401B23
:10A1B800A042FAD338BD10B504462CB14FF47A70DA
:10A1C800FFF7EEFF013CF8E710BD024A13680133C0
:10A1D80013607047C41A0020024BD3F8B03003B1A3
:10A1E800184770472C170020014B1B68184700BF01
:10A1F800D422002003681B69184703681B681847A6
:10A208002DE9F84FB0F90230934218BF00232DED25
:10A21800028B18BF0370057804460E469146002D40
:10A2280040F08B8007EE902A9FED770AF8EEE77AE8
:10A23800B6EE008A27EE800ADFED747A20EE270A50
:10A24800A04620EE080A05F081F8DFED716A60EE9D
:10A25800266AB7EE006AB0EE667AA0EE007A40F29F
:10A26800DC536365D0EE006A1023A4F8523037EE51
:10A27800067A76EE866AC6EE077A1823A4F8503076
:10A28800274684ED046A27EE807A27EE007A77EE77
:10A29800075A84ED017AC4ED025A70EE005A84ED33
:10A2A800037AB8EE007AA5EE807A27EE877A67EE11
:10A2B800A67A84ED057AC4ED067ADFED567A98ED34
:10A2C800047A27EE277AF0EE678AB5EEC07AF1EEC7
:10A2D80010FA4CBF77EE487A77EE087A013517EE18
:10A2E800900A02F0D7FAD8ED017A67EEA87AC7E9A2
:10A2F8000E01F5EEC07AF1EE10FA4CBF77EEC87A8F
:10A3080077EE887A08F1040817EE900A02F0C2FA8C
:10A31800032DC7E9080107F10807CED1A6F2DC53DF
:10A328001B042367E3676367C4F88030A367C4F836
:10A3380084300123A4F802902370D4F85490B4F91F
:10A348005280636A276A206FE26FD4F840C0D4F85D
:10A358008010C4F88020C9EB060606FA08F64FEA12
:10A36800E67B734307FB0B332667A7FB06671F448F
:10A37800636C656F60674FEAE27B53430CFB0B3EEF
:10A38800ACFB02237344B61A67EB0307E36AA26ABD
:10A39800C4F884104FEAE07B434302FB0B3EA2FB68
:10A3A80000237344B6185F41E36CA06CB4F95020E5
:10A3B800A5674FEAE17B4B4300FB0B33A0FB010190
:10A3C8001944636B361A206B4FEAE57B05FB03F3F0
:10A3D80000FB0B3367EB0107A0FB0501194480194B
:10A3E800794102F02DFA08F1FF3201239340E0672A
:10A3F800C01841EBE371424602F022FABDEC028B31
:10A408004844BDE8F88F00BF6F12833ADB0F49401C
:10A41800F404B53F0000804B2DE9F8430024244B99
:10A4280093F8AA60E0B2B0420ED203EB400203EB0D
:10A438008003B2F8B410D3F8CC301BB10B2801D884
:10A44800DB6898470134EAE71A4B1B685B032DD594
:10A4580000242346E2B2B24228D2DFF8549009F130
:10A46800CC074FEA840857F8242055689D4215D038
:10A478002846FEF77DF8EFF31283502282F3128804
:10A4880028216A6A01FB00900132C0F820216A691C
:10A4980042F001026A61DBB283F3118857F8083091
:10A4A8001B6800221A6001342B46D3E7BDE8F88305
:10A4B8002C1700200822002008B50E4B1B6813F447
:10A4C800805F0D4B14BFD3F8C421D3F8C82193F88B
:10A4D800AA1092880023D8B2884204D2074820F8EC
:10A4E80013200133F7E7FFF797FF3220BDE8084054
:10A4F80061E600BF082200202C170020E01700208A
:10A508000A4B1A680A4B30B502F48052D3F8C4419A
:10A51800D3F8C85100230AB1A18800E0A9880548EA
:10A5280020F8131001330C2BF5D130BD0822002080
:10A538002C170020EC21002070B5124D0024214674
:10A5480005F2CD10702285F8CC4104F0AAFC214612
:10A55800D5F840320B4A0B4493F9020080B102F25D
:10A56800CD141E680E5108199C8884809B798371CC
:10A5780092F8CC3107310133702982F8CC31E7D118
:10A5880070BD00BF2C170020094B1A680E2303FB6F
:10A598000020437AFF2B07D0064A12789A4203D943
:10A5A800054A32F8130000E0808800B2704700BF07
:10A5B800F80E0020C0210020E80C002038B52A4CF5
:10A5C8002DED048B94ED918ADFED289A38EE290A57
:10A5D8000546FBF7AEFAF0EE408AB0EE480AFBF704
:10A5E800A8FA94ED929AB0EE408A39EE290AFBF760
:10A5F800A0FAF0EE409AB0EE490AFBF79AFA95ED08
:10A60800017AD5ED027A95ED006A68EE676A27EE61
:10A61800088AE7EE286A68EE000A67EE807AE6EEB6
:10A62800290AB0EE660AE7EEA80A04F01BFFDFED80
:10A63800107A20EE270ADFED0F7A80EE270AD4ED94
:10A64800937A30EE270AF2EE047A80EE270A04F0B5
:10A6580037FEBDEC048B83B21A0444BF00F5B47016
:10A6680083B218B238BD00BF2C170020DB0FC93FDA
:10A678000000E144DB0F494001380A4B042804D8A4
:10A68800DFE800F00507090B0D00074A08E0074A54
:10A6980006E0074A04E0074A02E0074A00E0074AE2
:10A6A8001A607047F80000201D8D0008F99900080D
:10A6B80015900008118A0008B98600088D9C0008CA
:10A6C80010F80A3C0133DBB20A2B84BF10F8131CC4
:10A6D800044A00F80A3C82BF002322F8113000F82F
:10A6E8000A3C70470C0D0020334A136C90681944DB
:10A6F800081A40F68C23984270B513469160D060D2
:10A7080051603BD9127893F945108A4210460BD113
:10A71800111F082908D893F84610182901D80131C3
:10A7280003E083F8442002E0002183F8461093F9FF
:10A7380044402149A24219D191F84740B4B10C31A3
:10A748000024944206DA1D4D51F8046F25F8146070
:10A758000134F6E70C2805D01849002421F81040E8
:10A768000130F7E7164801780131017083F8452078
:10A77800002201211A7083F8471070BD92F8471023
:10A78800C9B1A0F2EF2440F2DA518C4208D811780E
:10A798000B2905D80B1D0131117042F8230070BD3B
:10A7A800002283F84720074B03F13002002143F8C9
:10A7B800041F9342FAD170BD980100200C0D0020AF
:10A7C8001C040020A4010020024A136C0133194420
:10A7D8001164704798010020024B53F820301B6821
:10A7E80019607047F8170020064B53F820301A6894
:10A7F8001B89A1F57A7159434FF47A7391FBF3F1F0
:10A8080011607047F8170020F0B5046D866823685A
:10A8180023F0010323608379054613F0020F407982
:10A828000CBF4FF0000E4FF4005E13F0040F14BF7E
:10A838004FF48067002710F0010F14BF0421002196
:10A848008307206820F001002060626822F44052EB
:10A858004EEA02026260226822F4B05323F00C032D
:10A8680048BF41F008013B430B432360A36895B000
:10A8780023F44073A3606846FAF726FC284B9C42F1
:10A8880001D10C9B0EE0274B9C4201D10D9B09E0A6
:10A89800254B9C4201D10E9B04E0244B9C420CBFEB
:10A8A8000F9B109B2268A879170448BF5B00B3FB75
:10A8B800F6F206FB1233B3EB560F236828BF0132BA
:10A8C8001E0441BF4FF6F073C2F34201134041EA40
:10A8D80003026B7992B213F0020FA28100F001011A
:10A8E80014BF4FF400320022DC0748BF42F4803224
:10A8F8002B6D11B159680A4302E0596821EA020236
:10A908005A609A6801074CBF42F0080222F0080218
:10A918009A601A6842F001021A6015B0F0BD00BFD3
:10A92800003801400044004000480040004C00400E
:10A938003D4B1B78012B30B514BF00240324B1B95B
:10A94800036A23F0010303628169036A21F0F301BA
:10A9580023F00A0341F0010142F001021A4341EADF
:10A96800041181610262836923F00C031BE004294E
:10A978001DD1016A4FF6EF730B4003628169056AC6
:10A98800120121F473414FF65F7342F0100241F453
:10A9980080712B4092B2134341EA04318161036212
:10A9A800836923F4406383618369836130BD082927
:10A9B800016A1AD14FF6FF630B400362C169036A4B
:10A9C8009BB289B223F4206343F4807321F0F3012E
:10A9D80043EA022241F0010192B241EA0411C16145
:10A9E8000262C2694FF6F37319E04EF6FF730B402B
:10A9F8000362C369056A40F6FF41194045F6FF73D3
:10AA08002B4043F4805343EA023241F4807192B2FE
:10AA180041EA0431C1610262C2694FF2FF33134057
:10AA2800C361C369C36130BD9401002038B510F813
:10AA38000E2C50F8043C044652B9012200F80E2CA2
:10AA480020F80C1C997A18680222BDE838406FE794
:10AA580030F80C2C20F80A1C891A89B220F8081C36
:10AA6800074A10F80F0C002522F8101004F80E5CA5
:10AA78001868997A2A46FFF75BFF04F8065C38BD28
:10AA88000C0D0020044B53F820301BB107289CBF45
:10AA98001B681960704700BFC0020020084A13688D
:10AAA8009B050BD5074B00211970074908684FF61D
:10AAB800FE7303400B604FF400735360704700BF90
:10AAC80000000240EE2200203000024073B5064626
:10AAD8000D46002401232A88A34013421AD0AA78DD
:10AAE800009302F003038DF80430EB78022B03D0B7
:10AAF800032B0CBF032301238DF805303046C2F326
:10AB080001136946C2F381028DF806308DF80720DB
:10AB1800FAF748FC0134102CDCD102B070BD2DE9E5
:10AB2800F743DFF8149299F8004005468E464F46E1
:10AB380011460068164698467246631C07F8043B9F
:10AB4800FDF7C8FC2B89ADF8043001A90223686819
:10AB58008DF806308DF80730FFF7B8FFAB7A2A6812
:10AB68002401274449460C2B00F2B780DFE803F0A4
:10AB780007B5B5B53EB5B5B56AB5B5B59300136AB1
:10AB8800DFF8B8C123F001031362136AD2F804E0B6
:10AB9800906920F4803020F07300624540F0700026
:10ABA80012D00CF5006C62450ED00CF5406C624575
:10ABB8000AD00CF5806C624506D00CF5806C6245B5
:10ABC80002D043F0030307E023F00E032EF4407E87
:10ABD80043F003034EF4807EC2F804E09061C2F8AB
:10ABE80034801362936943F0080329E0136ADFF89D
:10ABF8004CC123F010031362136AD2F804E0906981
:10AC080020F0807020F4E640624540F4E04006D031
:10AC18000CF5006C624502D043F0300307E023F0E6
:10AC2800E0032EF4406E43F030034EF4806EC2F819
:10AC380004E09061C2F838801362936943F40063BA
:10AC480093614AE0136ADFF8F4C023F48073136257
:10AC5800106AD2F804E0D369624523F0730343F025
:10AC6800700306D00CF5006C624502D040F44070C9
:10AC780007E020F460602EF4405E40F440704EF42B
:10AC8800805EC2F804E0D361C2F83C801062D369E8
:10AC980043F0080320E0136ADFF8A0C023F48053D0
:10ACA8001362106AD2F804E0D369624523F4E643DC
:10ACB80043F4E04340F4405003D00CF5006C624587
:10ACC80001D14EF4804EC2F804E0D361C2F840804E
:10ACD8001062D36943F40063D3612B7B1BB1536CBF
:10ACE80043F40043536413889BB243F00103138079
:10ACF800AB7A0C2B18D8DFE803F0071717170B17D8
:10AD080017170F17171713000B1902F134000AE071
:10AD18000B1902F1380006E00B1902F13C0002E0C1
:10AD28000B1902F1400058600C443846A681A26015
:10AD380003B0BDE8F08300BF7C190020002C01405F
:10AD4800054B98420CBF054A054A138801339BB24C
:10AD580013800020704700BF00540040602200208C
:10AD680062220020704708B50B4B002093F82C1086
:10AD7800FAF74CF8094B1B68187A082801BF084BEA
:10AD88004FF480521A80102208BF5A80A0F109039C
:10AD98005842584108BD00BFAC000020881A002066
:10ADA800701A0020704770477047FEE7FEE7FEE71D
:10ADB800704730B50024E3B293420DD2030F092B3C
:10ADC80094BF3033373301F8143001EB44030025C6
:10ADD80000015D700134EEE730BD30B5002202F1AC
:10ADE800805303F5B8539B0042F400441D6840F6B5
:10ADF8000F7144F08004294001322143042A19606C
:10AE0800EDD1024B40F08000186030BD4C5C004032
:10AE18002DE9F347884D894C2B68894E9BB2A38056
:10AE2800A28831880A40970507D54FF6FF53854A0F
:10AE38002B6013780133DBB21370A3880B4018041E
:10AE480040F100830023ADF802302B687B4F9AB2A3
:10AE58001804A28040F1F682BB8803F00F03BB718F
:10AE6800002B40F0C182784A13689BB23B803B8834
:10AE780003F030037B803B8803F440533B80116828
:10AE88004BF6BF730B4083F4005383F0200343F465
:10AE9800004343F080031360BB88D90621D41168AE
:10AEA80048F60F730B40694913600B681A7A022A37
:10AEB800884601D0042A02D1F9F734FF5AE2062A5B
:10AEC80040F06B825A78052A08D11A78520605D1C3
:10AED800D878FFF782FFBB681B6A9847E3689B68CE
:10AEE8005AE213689BB2ADF80230BDF802301F0574
:10AEF80040F1D0811168554F40F68F730B4054498B
:10AF080013600A68534B92B213445B0088461A6870
:10AF18003B68187A092817D092B2520002F1804291
:10AF280002F5C04211781970517859709188C8B2E9
:10AF3800090A41EA002159801189C8B2090A41EA7F
:10AF4800002199809289DA8001221A72DA8893F8AE
:10AF58000190002A40F0DC801A7812F07F024AD172
:10AF6800B9F1090F0FD1DA78012A00F2B88099787F
:10AF7800002940F0B4809988002940F0B0809A7286
:10AF8800A3685B68A9E0B9F1050F10D193F9032014
:10AF9800002A01DA0823B9E09A78002AFAD19A88B7
:10AFA800002AF7D19B7A002B00F0A280F2E7B9F1D2
:10AFB800030F0ED1DA78012A40F091809A88002A8E
:10AFC80040F08D805A7A42F020025A72A368DB69F9
:10AFD80083E0B9F1010F40F08280DA78012A7ED14E
:10AFE8009A88002A7BD15B7A980678D5F9F730FFE2
:10AFF80000287DD073E0012A2ED1B9F10B0F6ED154
:10B00800E26858799269D97890473B689A7A002A19
:10B0180065D0002863D11A79002A60D19B78002B6B
:10B028005DD1064B9B68DB689847084B1B685A79CB
:10B03800DA72DA781A735BE0445C0040701A002018
:10B04800C4220020F0220020005C0040881A002062
:10B05800505C004004300020022A40D1B9F1010FB1
:10B06800C4D0B9F1030F3AD1587920F0800E4FEAD5
:10B078008E0202F1804101F5B84110F0800F096895
:10B0880014BF01F0300101F44051BEF1030F26D87E
:10B09800B3F802E0BEF1000F21D101B39B7AF3B1FE
:10B0A80002F1804202F5B842010613684BBF23F44F
:10B0B800E04323F4804323F0400323F070034BBFA5
:10B0C8009BB29BB283F0100383F4805343F4004394
:10B0D80043F080031360A3689B69984708E0E3681E
:10B0E80048465B69984703280FD000287FF452AF81
:10B0F800D8F80020A14B92B213445B001A680022D2
:10B108001A6030236380062300E009233A6847E188
:10B11800B9F1060F12D11A78520678D19B78012B13
:10B1280002D1E368DB6967E0022B02D1E3681B6A9E
:10B1380062E0032B6BD1E3685B6A5DE0B9F1000F55
:10B1480038D15988002962D15A6822F47F42B2F571
:10B15800003F5CD11A7812F07F0204D19B88002B43
:10B1680000F0D58153E0012A08D1E2685879926944
:10B17800904700284BD13B689B7A17E0022A46D1BA
:10B188005A7902F00F010BB29B0003F1804303F5DB
:10B19800B84312F0800F1B6814BF03F0300303F4A8
:10B1A8004053032933D812F0700F30D1002B40F0F0
:10B1B800AE812CE0B9F1080F04D11B785B0600F0D2
:10B1C800A88124E0B9F10A0F21D11A7802F07F0290
:10B1D800012A1CD19A7AD2B15988C1B95A6822F485
:10B1E8007F42B2F5803F12D1E26858799269904760
:10B1F800002800F090810AE04BB13A684FF000084F
:10B20800A2F8128093614046984740460BE0E368F5
:10B218003A681B6950789847032804D1584B1B6833
:10B2280009221A72BDE03A68138A4FF6FF718B4201
:10B2380001D10923B4E0022800D00BB90823AFE0FC
:10B2480092F9001000291FDAD188019101988342F0
:10B2580002D9019B138210E08B420ED2E16891F86B
:10B268002C00834201D2002105E093FBF0F100FBA2
:10B27800113313B90121434B1970E36893F82C304B
:10B288009382F9F74FFD8CE0032313724FF4405378
:10B29800238086E0BDF802301BB2002BBFF6D5AD87
:10B2A800116840F68F730B401360354A17683B7A74
:10B2B800022B904671D0042B6FD0032B01D0052BA5
:10B2C80066D1BB693A8A8BB9398A00293BD04FF4D9
:10B2D800405323802C4B1A68284B92B213445B00CE
:10B2E8001A6800221A60302363802CE0002AEBD011
:10B2F800B7F81490914528BF91461FFA89FA50462D
:10B3080098473B8ACAEB03033B827B8A53447B8280
:10B318001D4B1A681D4B92B213445B0009F10102E0
:10B328001B689BB203F1005303F5405352105B00B6
:10B338004FF0000E9645C7D053F82E1020F81E1077
:10B348000EF1010EF6E7BB8A8B42D8F8003001D81F
:10B35800032201E011B105221A720BE006221A72CB
:10B36800094B1A68054B92B213445B001A681960BE
:10B3780030236380D8F800301B7A0FE002300020B9
:10B38800881A0020EF220020505C00400430002082
:10B39800072B02D1E368DB6898470823D8F8002018
:10B3A8001372FFF7E0FC5E4B1A684BF6BF7313404D
:10B3B8002288D704228848BF83F480539004628887
:10B3C80048BF83F40053D106628848BF83F0100356
:10B3D800920648BF83F0200343F4004343F0800300
:10B3E8004F4A9BB213602DE09A0002F1804202F5A9
:10B3F800B842116889B2ADF80210BDF8021009B25E
:10B40800002909DA106840F68F7101401160013B8C
:10B41800444A52F823309847BDF802301F067FF59A
:10B4280014ADA1798B0003F1804303F5B84348F6C6
:10B438000F72186802401A603A4B03EB81039B694C
:10B44800984702E5A28833881340590505D54FF679
:10B45800FF332B60344B5B689847A28831880A40D9
:10B46800920444BF4DF6FF732B60A3882F4A0B400C
:10B47800DB0452D54EF6FF732B6000231374137C44
:10B48800052B41D8DFE803F0030D1418222D63695A
:10B49800264D1BB900F04CFB062300E005232B7456
:10B4A8003BE000F045FB042323740123636134E08F
:10B4B80002236374032328E0637C013BDBB26374DB
:10B4C800637C53BB194B04221A7426E0184A13688C
:10B4D8009BB243F010031360052323740A2363749B
:10B4E8001BE0637C114A013BDBB26374637C03F0AD
:10B4F800FF0093B90E490C684FF6EF7323400B60B9
:10B5080006231374506108E00623237405E0094BF1
:10B5180073E6094B71E6094B6FE602B0BDE8F087A8
:10B52800005C004064120108AC000020701A002082
:10B53800405C0040854800083D490008194900085A
:10B5480020B9034B1B6808221A82704701487047CC
:10B55800881A00206C00002038B5294B05464FF4A6
:10B56800204298685A608469240404D51446013A34
:10B57800002CF8D10FE04268224C1440224A2243A2
:10B5880042604FF420425A608469A4070AD41446E2
:10B59800013A002CF8D15A60FFF7D2FB003018BFEF
:10B5A800012038BD4FF4204285625A60846925061F
:10B5B80004D41446013A002CF8D1ECE74268114C47
:10B5C8001440124A224342604FF420425A60846970
:10B5D800A40704D41446013A002CF8D1DBE74FF451
:10B5E800204281625A608169890604D41146013A71
:10B5F8000029F8D1CFE75A602023C361012038BD64
:10B60800881A0020009800FCD0200101D000010217
:10B618002F4B70B505464FF4204498685C608669E6
:10B62800360404D52646013C002EF8D111E04668C0
:10B63800284C344044F4903444F0D00444604FF42F
:10B6480020445C608669B60716D42646013C002E65
:10B65800F8D15C600AE098685C60224681698906D6
:10B6680031D41146013A0029F8D15A60FFF768FB36
:10B67800003018BF012070BD4FF4204485625C6023
:10B6880085696E0604D42546013C002DF8D1E0E713
:10B698005C60104D446825400F4C2C4344EA01443B
:10B6A80044604FF420440029D5D0986885696D0717
:10B6B80003D414F1FF34F9D2CBE7406A02F8010B46
:10B6C8000139C9B2EDE75A602023C361012070BD7A
:10B6D800881A0020009800FCD02400020C4B0D4969
:10B6E800DA684378D243C2F30222C2F104029340DB
:10B6F80002781B010A44DBB282F800330378012286
:10B70800580903F01F0302FA03F341F82030704789
:10B7180000ED00E000E100E073B505460021006897
:10B728000122FCF7D7FE2A6813889BB243F0010375
:10B738001380EB7A8DF804300124002601A88DF8D7
:10B7480005408DF806608DF80740FFF7C7FFEB7AD4
:10B758001B2B0BD1192301A88DF804308DF8054057
:10B768008DF806608DF80740FFF7B8FF02B070BD8E
:10B77800864B1A7B013A012A30B500F20681597BC3
:10B78800814240F002819A7B022A00F0FE80804AC2
:10B798001C7C505CD8734900B2EE047A1CB15A186C
:10B7A800B2F9122009E05A18D3ED067AB2F912203C
:10B7B800F1EE677AC3ED067A524207EE902AD3ED8E
:10B7C800076A724AF8EEE77AF5EE406AF1EE10FA87
:10B7D800C7EE877A49D1D2ED086AF4EEE67AF1EE3F
:10B7E80010FA04DD9069C2ED087A5062B9E0F5EE0E
:10B7F800C06AF1EE10FA40F3B48092F8285045B1CF
:10B80800022D00F2AE80D06BC2ED077AFA301064D8
:10B81800A7E0D2ED066A77EEE67AF7EE006AF4EE74
:10B82800E67AF1EE10FAD2ED0C7A0DDBDFED596A0B
:10B8380067EEA66ADFED587AF4EEE76AF1EE10FAE1
:10B8480058BFF0EE667A03E0DFED546A67EEA67A39
:10B85800C2ED0C7A012283F828209A6B024484F006
:10B8680001040020D0721C7478E0F4EEE67AF1EE60
:10B8780010FA48BFC2ED077A1C6CDA6B93ED086AC0
:10B88800D3ED075A121B002A76EE656A0BDAB7EE7B
:10B89800005AF4EEC56AF1EE10FA62DDF4EEE57ACC
:10B8A800F1EE10FA5DDDD3ED097A384AB4EEE76AB5
:10B8B800F1EE10FA0CDDD2ED0B7ADFED366A67EEA9
:10B8C800A67ADFED366AC2ED0B7AD2ED0D7A0AE080
:10B8D800F0EE007AF4EEE76AF1EE10FA08DDD2ED48
:10B8E8000D7ADFED2C6A67EEA67AC2ED0D7A07E0D5
:10B8F800D2ED0B7ADFED296A67EEA67AC2ED0B7AF4
:10B90800D3ED0B7A9A6B214C67EE877A0244FCEEF2
:10B91800E77A17EE900A5070D3ED0D7AFCEEE77ACD
:10B9280017EE900A507593F82800022801BFD4ED4D
:10B938000C7ADFED1B6A67EEA67A002003BFFCEEE7
:10B94800E77A84F8280017EE900A02220CBFD0721A
:10B9580084F828201A7C82F001021A740022DA6125
:10B968001A62187C094A08B10E4800E00E48906136
:10B978001944D3ED067AB1F9122000EE102AB8EE78
:10B98800C00A80EE070A37EEC00A30BD881A0020C8
:10B99800A0120108EC51783F6F12833A0AD7833F0F
:10B9A80000007A440000A0410000A0C108B522228E
:10B9B8001148002103F075FA104B002210490420A9
:10B9C800515C83F8F2110132052183F8F701042A4A
:10B9D8004FF0000083F8F61183F8F90183F8F811A5
:10B9E80003F10803EAD1074B0122A3F838225222B7
:10B9F80083F8342208BD00BFBC1C0020CC1A0020EC
:10BA0800972B0108881A002000F1500302781AB910
:10BA18008178C278914204D304309842F6D100204C
:10BA280070470120704710B5F9F73AFB4FF43024FE
:10BA3800012806D11CB1F9F733FB013CF8E70520D2
:10BA480010BD002C08BF052010BD70B50646441E69
:10BA580014F8011F89B1094D284603F058FA002847
:10BA6800F6D005F1080398423FBF054B401BC018AC
:10BA7800A31B38BF80F8CE31EAE770BD9B2B0108C5
:10BA8800881A0020031EB8BF2D2210B5B8BF58422F
:10BA98000C46B8BF01F8012B0A22F9F725FF00234D
:10BAA8000370204610BD07B51B4B03F5E762C3F8CA
:10BAB800342793F8D6215AB1012A14D1032183F8E7
:10BAC8003A17072183F83C2783F83B170C2208E034
:10BAD800022183F83A17032183F83C2783F83B17A0
:10BAE800072283F838270D4B0D4A9A604020FBF750
:10BAF800B9FE70B10122002390F9000040218DE8C1
:10BB08000C00084A4FF4E133FBF794FC003018BFEF
:10BB1800012003B05DF804FB881A00206C000020A7
:10BB2800194A0008994B00080120002100F0D2B9F9
:10BB38000B4B10B519684FF6FB720A401A60094A98
:10BB480092F84A271C46084B0AB1052200E0012258
:10BB58001A60FCF749FC4FF43643236010BD00BF60
:10BB6800405C0040881A0020D8220020014B33F89E
:10BB7800110070470C0D00200020704707B5064BD8
:10BB88000093064B01930649064A074B0748F9F705
:10BB9800BFFE03B05DF804FB912101089A2101085A
:10BBA800D02B0108DB2B010885210108B02B0108E7
:10BBB80008B5037833B90C4B0C481978BDE8084030
:10BBC800F9F7A6BE03F008FA02280BD8064B084A74
:10BBD80018700C2101FB002002305860FAF7A0F918
:10BBE8000448E6E708BD00BFE4210020E22B010875
:10BBF800942100204C21010808B503783BB90B4B70
:10BC08000B4893F8C816BDE80840F9F781BE03F061
:10BC1800E3F9022808D8054B83F8C806FAF7E6F8CE
:10BC2800FAF7A2F90348E8E708BD00BFCC1A0020DC
:10BC3800E62B01084C21010838B5037803BB214BDA
:10BC48001B6801330F2B07D81F490C2202FB031274
:10BC58001C4695682DBB00E01C4601340F2C01DD05
:10BC6800002400E005D818490C2202FB041295684C
:10BC7800BDB99C42F1D11548BDE83840F9F748BE36
:10BC880003F0AAF90F28044605D80F4A0C2303FB32
:10BC980000239D682DB921460D48BDE83840F9F7C5
:10BCA80037BE084B1C60FBF789FE21462A46094827
:10BCB800F9F72EFE0C235C43034B185DBDE83840B2
:10BCC800FBF794BE78000020A4120108F32B0108AA
:10BCD800092C0108212C010873B5037813B9FBF767
:10BCE80057FA3FE001AA204903F0D7F90024024699
:10BCF800264625469AB134B1012C08D1104603F0E6
:10BD08006BF9064603E0104603F066F9054601AAFA
:10BD18000020154903F0C1F901340246EAE70B2D6A
:10BD280003D9124812490C230CE0022C11D1A6F5B4
:10BD38007A73B3F57A7F08D90C480E494FF47A72B2
:10BD48004FF4FA63F9F7E4FD0CE00B4B03EB450302
:10BD58001E81094B094803EB45032946B3F908201E
:10BD6800F9F7D6FD02B070BD642601086D240108FC
:10BD78008B26010823280108E4210020382C01081B
:10BD8800104910B50B6A03EB4002147E14B1022C63
:10BD98000FD00AE0022804D9032806D14A6AD2043F
:10BDA80001D5D88910BD988A10BD074B33F810000B
:10BDB80010BD507E00EB800000EB800000F2EE200A
:10BDC80080B210BDE4210020E80C002008B5FEF781
:10BDD800CBF9064B022283F82C20054A9862126898
:10BDE8009A63012283F8512008BD00BFE421002096
:10BDF800C41A002008B5FEF7B7F9074B022283F8EA
:10BE08002C209A6B00F5B71000F5587002F2DC523E
:10BE180098629A6308BD00BFE4210020044B5B6A66
:10BE280042F201021A420CBF01200020704700BFF5
:10BE3800E42100200F4B93F85420012A10B51C462A
:10BE48000DD008D3022A0DD10B4A938A9BB283F0F6
:10BE58001003938206E0084B10229A6102E0064B19
:10BE680010221A85FEF780F900F5F42000F590708D
:10BE7800A06510BDE421002000040048034BDA6DE2
:10BE8800D379591C1344D171187A7047E4210020E2
:10BE980010B5FFF7F3FF84B2FFF7F0FF04EB0020C3
:10BEA80080B210BD10B5FFF7F3FF0446FFF7F0FFAF
:10BEB80004EB004010BD38B5054D04462146286EF8
:10BEC800FEF79BF9EB6D98796040987138BD00BF1B
:10BED800E421002038B5044624200D46FFF7EBFF87
:10BEE8004D20FFF7E8FF002C084C14BF21203E200E
:10BEF800FFF7E1FFE36D002228469A71FFF7DBFFA9
:10BF0800E36D93F84900BDE83840D4E7E421002008
:10BF180001460020DEE710B50446C0B2FFF7CBFFAC
:10BF2800200ABDE81040C6E710B5044680B2FFF706
:10BF3800F2FF200CBDE81040EDE737B58288836832
:10BF4800044610060D4641BF2B4991F8C8164FF418
:10BF5800C67000FB0133D10544BF2849097802F0B7
:10BF68003F0244BF01EB410103EB8103042A12D0D5
:10BF780006D8012A0DD0022A32D193F9001030E0F8
:10BF8800102A0AD0202A0AD0082A29D1B3F9001089
:10BF980027E0197825E0198823E0196821E093ED56
:10BFA800000A6846F9F736FC01461548F9F7B0FC6F
:10BFB80005B3D4ED037A6846B8EEE70AF9F72AFC28
:10BFC80001461048F9F7A4FC94ED040A6846B8EE57
:10BFD800C00AF9F71FFC01460A48F9F799FC09E07D
:10BFE80000210948F9F794FC25B10848E16822695D
:10BFF800F9F78EFC03B030BDCC1A0020E4210020F4
:10C0080089230108822301084B2C0108472C0108C9
:10C01800024B0146586EFEF7F0B800BFE42100203D
:10C0280010B5441E14F8011F21B1034B586EFEF7DA
:10C03800E4F8F7E710BD00BFE42100202DE9F34143
:10C048002B4C2C4B94F868002B4E1D682B4B06EBA1
:10C0580080001A882A4BD0F8C0101B782948009114
:10C068004FF47A71B5FBF1F1F9F752FC26484821F3
:10C07800F9F74EFCD4F86C800027FBB206EB83027C
:10C08800D2F8D010E9B101259D4015EA080F16D065
:10C098002A0714D01D4AD25C0B2000FB0323164A42
:10C0A8001B4802EB8303D3F8F020F9F731FC022D8B
:10C0B80005D194F8781011B11648F9F729FC013721
:10C0C800DBE71548FFF7ACFF144B15481A68154B0A
:10C0D800B4F880109A420CBFB4F87C20B4F87E20E3
:10C0E8004FF4DE6392B202B0BDE8F041F9F710BC3C
:10C0F800E4210020C41A0020A4120108900E002098
:10C10800000100204E2C0108912C0108FC000020A1
:10C11800A12C0108A92C0108F12C0108901A002073
:10C12800AD2C0108005400402DE9F0410024804660
:10C1380025460F4EA7594146384602F035FF58B1FB
:10C1480039460C48F9F7E4FB30190021FFF7F5FEF2
:10C158000948FFF765FF0135143440F618339C424F
:10C16800E7D11DB90548BDE8F04159E7BDE8F081C0
:10C17800441401082E240108F12C0108B4230108F5
:10C188002DE9F04F2DED028B83B0054602F0CDFE70
:10C19800064620B1012818D12B782A2B15D15C48E6
:10C1A800FFF73EFF00245B4D5B486159F9F7B0FB90
:10C1B80028193146FFF7C1FE5848FFF731FF1434FC
:10C1C80040F618339C42EED19CE028463D2102F00F
:10C1D8009EFE002800F08F800346994613F8012D33
:10C1E800202AFAD0441C204602F0F6FE804620465B
:10C1F800F9F786FAC5EB0909B0EE408A0026DFF8A0
:10C2080034A1142202FB06F40AF5D07B54F80B7013
:10C21800384602F08AFE03461A46284639460193F4
:10C2280002F08CFE019B00285BD15FFA89F29A42EA
:10C2380057D10AEB0402D2ED6B7AF8EEE77A0BEBF2
:10C248000405B4EEE78AF1EE10FA48DBD2ED6C7A19
:10C25800F8EEE77AB4EEE78AF1EE10FA3FD8B2F8D2
:10C26800A431D2F8A82113F0200F08BF08EE108AD5
:10C278001C0641BF2A4991F8C8164FF4C67404FB3E
:10C288000122D90544BF2749097803F03F0344BF79
:10C2980001EB410102EB8102042B18EE100A0BD0CE
:10C2A80004D8013B012B0ED810700CE0102B05D0E0
:10C2B800202B06D0082B06D1108004E082ED008ADE
:10C2C80001E082ED008A39461748F9F721FB284634
:10C2D800002103B0BDEC028BBDE8F04F2DE61348FA
:10C2E80003E001368E2E8AD1114803B0BDEC028BD3
:10C2F800BDE8F04F94E6284603B0BDEC028BBDE8DC
:10C30800F04F11E703B0BDEC028BBDE8F08F00BF22
:10C31800DF2C0108441401082E240108F12C01081F
:10C32800CC1A0020E4210020F42C0108FF2C01087D
:10C33800B4230108A412010810B50A48FFF770FEDB
:10C34800094B5C6E2046FDF755FF18B90A20FDF72A
:10C3580032FFF7E7FEF7B0F8F9F71EFD034B044A82
:10C36800DA6010BD1F2D0108E421002000ED00E077
:10C378000400FA0508B50548FFF752FEFBF772FD01
:10C38800F9F734FDBDE80840D6E700BF2B2D0108BA
:10C3980008B50448FFF744FEF9F728FDBDE8084052
:10C3A800CAE700BF412D010820B9034B1B680822CA
:10C3B8001A82704701487047881A00206C000020D4
:10C3C80021B901288CBF0220002070470220704745
:10C3D80010B50A4B1968CA78042A0CD84C8A084B3D
:10C3E80028B903EBC2039B881B1B0B8210BD53F8B3
:10C3F8003230181910BD002010BD00BF881A002067
:10C408007C000020054B1968054B4A8A18B99B8C9B
:10C418009B1A0B827047186A10447047881A0020CC
:10C428007C000020054B1968054B4A8A18B99B8D7A
:10C438009B1A0B827047986A10447047881A00202C
:10C448007C000020074B1B681B7803F07F03212B1F
:10C4580006D100F0DF00022814BF02200020704738
:10C4680002207047881A0020212810B508D1114BE6
:10C478001B681B7803F07F03212B10D0022010BD0E
:10C488002028FBD10B4B0C4A1B6810701B7803F05B
:10C498007F03212B094B18BF00230BB9EEE7084B8C
:10C4A800044A126800249361548220469847204623
:10C4B80010BD00BF881A0020F122002049B50008ED
:10C4C800B1C300087047034B1A78202A04BF002222
:10C4D8001A707047F1220020014B04221A6070473D
:10C4E800D8220020034B9B7A13B1034B05221A6014
:10C4F800704700BFC8210020D82200200D4B0E49EC
:10C508001A680E4B92B213445B000D4A1B68C3F3C2
:10C51800090310B5136013689BB201335B10002246
:10C528009A4206D0074851F8044B20F812400132CD
:10C53800F6E710BD505C0040206200401E3000202D
:10C548007C22002080220020014B00225A64704780
:10C558007C2200202DE9F843664B674E1B68DFF804
:10C56800B881664A00254FF0C0099D7283F809908A
:10C57800DD723560D8F8003023F4EC4323F0700303
:10C5880043F400739BB2C8F80030D8F8003023F4A5
:10C59800E04323F040039BB248F2800483F0100389
:10C5A8002343C8F80030336812FA83F35B0040274E
:10C5B8001A681F6033689BB203F1005303F54053B8
:10C5C8005B0028461A6880221A60D8F8003023F4E5
:10C5D800F8731B051B0D2343C8F80030484B93F82C
:10C5E8005C10F8F713FCD8F80030464A464923F4A3
:10C5F800804323F070039BB283F440532343C8F86D
:10C608000030136823F4EC4323F070039BB21360EB
:10C61800336811FA83F35B0003201968C3F80090AC
:10C6280013683A4923F4E04323F040039BB283F0B4
:10C63800200323431360136823F4804323F070031B
:10C6480023439BB21360536823F4EC4323F0700335
:10C6580043F4C0639BB25360336811FA83F35B0001
:10C6680019684FF480711960536823F4804323F0EC
:10C67800700323439BB25360536823F4E04323F0D1
:10C6880040039BB283F0200323435360D8F80C3057
:10C698001F4A23F4EC4323F070039BB2C8F80C3014
:10C6A800336812FA83F35B0039461A684FF48872CC
:10C6B8001A60F8F7ABFBD8F80C3023F4804323F06A
:10C6C80070039BB283F440532343C8F80C30D8F866
:10C6D8000C3023F4E04323F040031C43A4B2C8F811
:10C6E8000C402846FEF779FB0A4B01221A60BDE888
:10C6F800F88300BF881A0020505C004004300020F6
:10C708007C000020045C004008300020103000202D
:10C718001C300020D8220020005C0040134A144B33
:10C7280050681B68181810B5146808D011490822F9
:10C73800FEF73FFB204610490422FEF73AFB0F4B59
:10C748001A68002393720E4A012111600D49136083
:10C758004FF4E0500B6010600B480B604FF436410B
:10C76800A0F848101160094A136010BDB0F7FF1F08
:10C77800ACF7FF1FDE000020EE000020881A002022
:10C78800405C0040445C00407C220020D82200200D
:10C79800024B4FF480221A60704700BF1404014016
:10C7A80013490B7813F0010F03F004021BD0F2B900
:10C7B8001048006840011AD4980714D443F00403C1
:10C7C8000B700D4B1A880D4B1A800D4B0D4A1B68C8
:10C7D80092F8E2214FF47A7101FB02330A4A0520EC
:10C7E8001360FBF703B912B90120FBF725B97047AD
:10C7F800ED220020740B0020A40B0020C82200208A
:10C80800C41A0020CC1A00209C0B0020054A13787B
:10C81800590705D523F0040304201370FBF7E6B885
:10C82800704700BFED22002008B5044B1B7803F0C9
:10C838000503052B01D1FDF73FFEFEE7CA220020C4
:10C84800D0400B1C1141203A03D49C461341184395
:10C858006346524293401843704700BF7BB972B990
:10C868000029BEBF00204FF0004106E008BF0028A5
:10C878001CBF6FF000414FF0FF3000F073B882B07A
:10C88800EC462DE9005000F03DF8DDF804E002B078
:10C898000CBC704707EE900AF5EEC07AF1EE10FA7C
:10C8A80001D400F009B808B580F0004000F004F8A1
:10C8B800404261EB410108BDD0B500F0B9F9002252
:10C8C8000E4B06460F4600F007FA00F017FC044628
:10C8D80000F08CF900220A4B00F0FEF902460B46E4
:10C8E8003046394600F044F800F008FC23460022A0
:10C8F80042EA000210461946D0BD00BF0000F03DD4
:10C908000000F0412DE9F041069C154606460F4609
:10C91800984600F013FC05FB01F300FB0838A5FB63
:10C928000023B21A434467EB0303C4E90023BDE8BC
:10C93800F08100BF2DE9F041069C904606460F465F
:10C948001D4600F049FD00FB05F5A0FB082308FB88
:10C958000155B21A2B4467EB0303C4E90023BDE871
:10C96800F08100BF704700BF81F0004102E000BFC6
:10C9780083F0004330B54FEA41044FEA430594EA97
:10C98800050F08BF90EA020F1FBF54EA000C55EAD2
:10C99800020C7FEA645C7FEA655C00F0E2804FEAA3
:10C9A8005454D4EB5555B8BF6D420CDD2C4480EA85
:10C9B800020281EA030382EA000083EA010180EAB5
:10C9C800020281EA0303362D88BF30BD11F0004F03
:10C9D8004FEA01314FF4801C4CEA113102D0404239
:10C9E80061EB410113F0004F4FEA03334CEA133374
:10C9F80002D0524263EB430394EA050F00F0A7808C
:10CA0800A4F10104D5F1200E0DDB02FA0EFC22FA86
:10CA180005F2801841F1000103FA0EF2801843FA7A
:10CA280005F359410EE0A5F120050EF1200E012A6B
:10CA380003FA0EFC28BF4CF0020C43FA05F3C018A9
:10CA480051EBE37101F0004507D54FF0000EDCF122
:10CA5800000C7EEB00006EEB0101B1F5801F1BD3CB
:10CA6800B1F5001F0CD349085FEA30004FEA3C0CCF
:10CA780004F101044FEA445212F5800F80F09A80C5
:10CA8800BCF1004F08BF5FEA500C50F1000041EBC9
:10CA9800045141EA050130BD5FEA4C0C404141EBCD
:10CAA800010111F4801FA4F10104E9D191F0000FF4
:10CAB80004BF01460020B1FA81F308BF2033A3F177
:10CAC8000B03B3F120020CDA0C3208DD02F1140C6E
:10CAD800C2F10C0201FA0CF021FA02F10CE002F1A9
:10CAE8001402D8BFC2F1200C01FA02F120FA0CFCA2
:10CAF800DCBF41EA0C019040E41AA2BF01EB0451EB
:10CB0800294330BD6FEA04041F3C1CDA0C340EDCE8
:10CB180004F11404C4F1200220FA04F001FA02F32B
:10CB280040EA030021FA04F345EA030130BDC4F1E9
:10CB38000C04C4F1200220FA02F001FA04F340EADE
:10CB48000300294630BD21FA04F0294630BD94F08F
:10CB5800000F83F4801306BF81F480110134013D76
:10CB68004EE77FEA645C18BF7FEA655C29D094EAE7
:10CB7800050F08BF90EA020F05D054EA000C04BF65
:10CB88001946104630BD91EA030F1EBF0021002050
:10CB980030BD5FEA545C05D14000494128BF41F0EF
:10CBA800004130BD14F580043CBF01F5801130BD53
:10CBB80001F0004545F0FE4141F470014FF00000DE
:10CBC80030BD7FEA645C1ABF194610467FEA655C8F
:10CBD8001CBF0B46024650EA013406BF52EA033531
:10CBE80091EA030F41F4002130BD00BF90F0000F1F
:10CBF80004BF0021704730B54FF4806404F132045B
:10CC08004FF000054FF0000150E700BF90F0000F13
:10CC180004BF0021704730B54FF4806404F132043A
:10CC280010F0004548BF40424FF000013EE700BF0A
:10CC380042004FEAE2014FEA31014FEA02701FBF9A
:10CC480012F07F4393F07F4F81F06051704792F06C
:10CC5800000F14BF93F07F4F704730B54FF46074E6
:10CC680001F0004521F0004120E700BF50EA010231
:10CC780008BF704730B54FF000050AE050EA0102DE
:10CC880008BF704730B511F0004502D5404261EB4E
:10CC980041014FF4806404F132045FEA915C3FF48F
:10CCA800DCAE4FF003025FEADC0C18BF03325FEA28
:10CCB800DC0C18BF033202EBDC02C2F1200300FADD
:10CCC80003FC20FA02F001FA03FE40EA0E0021FA02
:10CCD80002F11444C1E600BF70B54FF0FF0C4CF4EC
:10CCE800E06C1CEA11541DBF1CEA135594EA0C0FA2
:10CCF80095EA0C0F00F0DEF82C4481EA030621EADD
:10CD08004C5123EA4C5350EA013518BF52EA033517
:10CD180041F4801143F4801338D0A0FB02CE4FF0C9
:10CD28000005E1FB02E506F00042E0FB03E54FF0F9
:10CD38000006E1FB03569CF0000F18BF4EF0010EF1
:10CD4800A4F1FF04B6F5007F64F5407404D25FEAED
:10CD58004E0E6D4146EB060642EAC62141EA5551A0
:10CD68004FEAC52040EA5E504FEACE2EB4F1FD0CE2
:10CD780088BFBCF5E06F1ED8BEF1004F08BF5FEA60
:10CD8800500E50F1000041EB045170BD06F0004612
:10CD980046EA010140EA020081EA0301B4EB5C04BF
:10CDA800C2BFD4EB0C0541EA045170BD41F48011B7
:10CDB8004FF0000E013C00F3AB8014F1360FDEBFDC
:10CDC800002001F0004170BDC4F10004203C35DAB8
:10CDD8000C341BDC04F11404C4F1200500FA05F33B
:10CDE80020FA04F001FA05F240EA020001F00042DC
:10CDF80021F0004110EBD37021FA04F642EB060152
:10CE08005EEA430E08BF20EAD37070BDC4F10C047B
:10CE1800C4F1200500FA04F320FA05F001FA04F23F
:10CE280040EA020001F0004110EBD37041F100012B
:10CE38005EEA430E08BF20EAD37070BDC4F1200536
:10CE480000FA05F24EEA020E20FA04F301FA05F29E
:10CE580043EA020321FA04F001F0004121FA04F246
:10CE680020EA020000EBD3705EEA430E08BF20EA16
:10CE7800D37070BD94F0000F0FD101F00046400050
:10CE880041EB010111F4801F08BF013CF7D041EAD2
:10CE9800060195F0000F18BF704703F000465200D6
:10CEA80043EB030313F4801F08BF013DF7D043EAA7
:10CEB8000603704794EA0C0F0CEA135518BF95EA5D
:10CEC8000C0F0CD050EA410618BF52EA4306D1D1E4
:10CED80081EA030101F000414FF0000070BD50EA03
:10CEE800410606BF1046194652EA430619D094EA8D
:10CEF8000C0F02D150EA013613D195EA0C0F05D177
:10CF080052EA03361CBF104619460AD181EA0301CA
:10CF180001F0004141F0FE4141F470014FF0000082
:10CF280070BD41F0FE4141F4780170BD70B54FF01D
:10CF3800FF0C4CF4E06C1CEA11541DBF1CEA13559D
:10CF480094EA0C0F95EA0C0F00F0A7F8A4EB05047F
:10CF580081EA030E52EA03354FEA013100F0888076
:10CF68004FEA03334FF0805545EA131343EA12633F
:10CF78004FEA022245EA111545EA10654FEA0026F4
:10CF88000EF000419D4208BF964244F1FD0404F5AD
:10CF9800407402D25B084FEA3202B61A65EB030509
:10CFA8005B084FEA32024FF480104FF4002CB6EBC6
:10CFB800020E75EB030E22BFB61A754640EA0C0046
:10CFC8005B084FEA3202B6EB020E75EB030E22BF86
:10CFD800B61A754640EA5C005B084FEA3202B6EBC7
:10CFE800020E75EB030E22BFB61A754640EA9C0086
:10CFF8005B084FEA3202B6EB020E75EB030E22BF56
:10D00800B61A754640EADC0055EA060E18D04FEA13
:10D01800051545EA16754FEA06164FEAC30343EAB3
:10D0280052734FEAC2025FEA1C1CC0D111F4801F80
:10D038000BD141EA00014FF000004FF0004CB6E779
:10D0480011F4801F04BF01430020B4F1FD0C88BF18
:10D05800BCF5E06F3FF6AFAEB5EB030C04BFB6EB23
:10D06800020C5FEA500C50F1000041EB045170BD16
:10D078000EF0004E4EEA113114EB5C04C2BFD4EB43
:10D088000C0541EA045170BD41F480114FF0000EC7
:10D09800013C90E645EA060E8DE60CEA135594EA43
:10D0A8000C0F08BF95EA0C0F3FF43BAF94EA0C0F46
:10D0B8000AD150EA01347FF434AF95EA0C0F7FF4BB
:10D0C80025AF104619462CE795EA0C0F06D152EA0F
:10D0D80003353FF4FDAE1046194622E750EA4106F3
:10D0E80018BF52EA43067FF4C5AE50EA41047FF404
:10D0F8000DAF52EA43057FF4EBAE12E74A0011D2B6
:10D1080012F5001211D20DD56FF47873B3EB625299
:10D118000ED44FEAC12343F0004343EA505323FAA5
:10D1280002F070474FF00000704750EA013002D11A
:10D138004FF0FF3070474FF00000704700292DE98D
:10D14800F043C0F2A6800026002BC0F29C808846DF
:10D1580094469E46154604460F46002B3DD18A420A
:10D1680059D9B2FA82F33BB1C3F120029F4020FAA9
:10D1780002F29D4017439C40290C220CB7FBF1FE9C
:10D18800A8B201FB1E7742EA074700FB0EF3BB4239
:10D198000AD97F190EF1FF3280F00581BB4240F2B7
:10D1A8000281AEF1020E2F44FF1AA4B2B7FBF1F3CD
:10D1B80001FB137744EA074700FB03F0B84208D99C
:10D1C8007F1903F1FF3280F0F080B84240F2ED8021
:10D1D800023B43EA0E43002203E08B420FD90022B0
:10D1E8001346341C18BF012460424FF0000565EB5C
:10D1F80045015840514000196941BDE8F083B3FA30
:10D2080083F2002A40F086808B4202D3844500F2E4
:10D21800DB800123E5E712B90123B3FBF2F5B5FA88
:10D2280085F000283BD1781B4FEA154E1FFA85FC84
:10D238000122B0FBFEF8210C0EFB180741EA074754
:10D248000CFB08F3BB4207D97F1908F1FF3102D262
:10D25800BB4200F2BD808846FF1AA4B2B7FBFEF3BA
:10D268000EFB137744EA07470CFB03FCBC4507D9C0
:10D278007F1903F1FF3102D2BC4500F2A7800B46AB
:10D2880043EA0843ADE752426FEA060663EB4303FD
:10D298005DE7404261EB41014FF0FF3654E7C0F1D2
:10D2A800200224FA02F107FA00F385404FEA154EEE
:10D2B800D7401943B7FBFEF20B0C0EFB12771FFA8F
:10D2C80085FC43EA07430CFB02F79F4204FA00F48B
:10D2D80007D95B1902F1FF3074D29F4272D9023A22
:10D2E8002B44DF1B89B2B7FBFEF80EFB187341EA2B
:10D2F80003430CFB08F79F4208D95B1908F1FF317B
:10D308005CD29F425AD9A8F102082B44D81B48EA9C
:10D3180002428EE7C2F120032CFA03F10EFA02FE54
:10D3280020FA03F741EA0E0E08FA02F028FA03F190
:10D338004FEA1E453843B1FBF5F8030C05FB1811FD
:10D348001FFA8EF743EA014107FB08F38B420CFAF8
:10D3580002FC09D911EB0E0108F1FF3930D28B42DA
:10D368002ED9A8F102087144C91A80B2B1FBF5F3AD
:10D3780005FB131140EA014107FB03F78F4208D967
:10D3880011EB0E0103F1FF3016D28F4214D9023B84
:10D39800714443EA0843C91BA3FB0C89494509D3D7
:10D3A80005D000221DE79646FEE6134611E7944095
:10D3B8004445F6D2013BF4E70346EAE78846A5E789
:10D3C800C846D1E702468CE713460AE7023B57E70F
:10D3D800A8F102082F443FE72DE9F041002B44D182
:10D3E8008A42154604464FD9B2FA82F70E464FB123
:10D3F800C7F12003B94020FA03F602FA07F50E43F5
:10D4080000FA07F44FEA154E230CB6FBFEF0AFB254
:10D418000EFB106143EA014307FB00F1994209D969
:10D428005B1900F1FF3280F0EC80994240F2E9800C
:10D4380002382B445A1AA4B2B2FBFEF30EFB132295
:10D4480044EA024207FB03F7974208D9521903F14D
:10D45800FF3180F0D880974240F2D580023B43EA02
:10D46800004000263146BDE8F0818B4247D8B3FA28
:10D4780083F6002E48D18B4202D3824200F2CD803F
:10D4880001203146BDE8F08112B90125B5FBF2F55E
:10D49800B5FA85F8B8F1000F77D14A1B4FEA154E57
:10D4A800AFB20126B2FBFEF0230C0EFB102143EABB
:10D4B800014107FB00F38B4207D9491900F1FF32FC
:10D4C80002D28B4200F2BA801046C91AA4B2B1FB4C
:10D4D800FEF30EFB131144EA014407FB03F7A742CE
:10D4E80008D9641903F1FF3280F08F80A74240F217
:10D4F8008C80023B43EA00403146BDE8F0810026BB
:10D5080030463146BDE8F081C6F1200422FA04F520
:10D51800B3402B4320FA04FC01FA06F721FA04F57C
:10D528004FEA134E4CEA0707B5FBFEF8390C0EFB21
:10D5380018551FFA83FC41EA05450CFB08F1A9427E
:10D5480002FA06F204D9ED1808F1FF3467D3A046B1
:10D558006D1ABFB2B5FBFEF40EFB145547EA054140
:10D568000CFB04FC8C4504D9C91804F1FF355CD3C5
:10D578002C4644EA0844CCEB0101A4FB022399425F
:10D5880048D344D0204600266CE7C8F1200401FAAD
:10D5980008F305FA08F520FA04F7E1404FEA154EBA
:10D5A8001F43B1FBFEF63A0C0EFB16111FFA85FC61
:10D5B80042EA01430CFB06F29A4200FA08F407D942
:10D5C8005B1906F1FF3137D29A4235D9023E2B4416
:10D5D8009B1ABFB2B3FBFEF00EFB103347EA0343BE
:10D5E8000CFB00F1994207D95B1900F1FF3221D2F7
:10D5F80099421FD902382B445A1A40EA0646674610
:10D6080050E7104616E70B4629E7134672E7B04085
:10D618009042B7D2601E002624E7304622E7A9428E
:10D6280095D9A8F102081D4492E78C45A0D9023C7F
:10D6380019449EE71046DFE70E46C9E70238294439
:10D6480043E700BF4FEA4102B2F1E04324BFB3F51C
:10D65800001CDCF1FE5C0DD901F0004C4FEAC00261
:10D668004CEA5070B2F1004F40EB830008BF20F045
:10D678000100704711F0804F21D113F13872BCBFFF
:10D6880001F00040704741F480114FEA5252C2F154
:10D698001802C2F1200C10FA0CF320FA02F018BF9D
:10D6A80040F001004FEAC1234FEAD32303FA0CFCF0
:10D6B80040EA0C0023FA02F34FEA4303CCE77FEA7F
:10D6C800625307D150EA01331EBF4FF0FE4040F4C9
:10D6D8004000704701F0004040F0FE4040F4000078
:10D6E800704700BF11481249026800608A4218D08A
:10D6F800002103E00F4B5B58435004310E480F4B99
:10D7080042189A42F6D30E4A02E0002342F8043B3C
:10D718000C4B9A42F9D3FAF767FE00F019F87047F4
:10D72800FEE70948D0F800D040680047FC9F002079
:10D73800EFBEADDE743B0108000000207001002040
:10D7480070010020F822002000D8FF1FFEE700002B
:10D758002DE9804895B0F2F713FDB14CB14F23780D
:10D768003D6833B1B04B1B68EB1A002BA4BF0023F4
:10D778002370FEF753FB10B1AC4B00221A70AC4B70
:10D7880019680B0740F18E81AA4B1B681B7A062B80
:10D7980000F27C81DFE813F0070007003400D400B2
:10D7A80010013C013C01A44B1A78002A00F06E815C
:10D7B80000221A70A14B93F800E0A14B1B6893F864
:10D7C80000C0A04B93F8008002229F4EB35C43FA3E
:10D7D8000EF303F00F03634502F101090CD20B2B82
:10D7E8009FBFB05C16F8096000EA080006EB00204D
:10D7F8009CBF964E46F823000232102AE5D10CE170
:10D80800934B1A78002A00F0418100221A70914B3C
:10D81800914A93F802C093F803E058780CF0070691
:10D8280040EA06200EF03F06760146EADC06106064
:10D83800187956605E7993F806C0800040EA9E1019
:10D8480006F0010E40EA8E20906093F807E00CF095
:10D858000F00C00140EA56000EF07F06D060360186
:10D86800187A46EA1C1693F809C0166140000CF0B5
:10D87800030640EADE1040EA462093F80AE05061C9
:10D88800D87A0EF01F06B601C00046EA9C0640EAA8
:10D898005E1093F80DC093F80EE0D061187B966186
:10D8A8000CF0070640EA06200EF03F06760146EA2D
:10D8B800DC061062D87B56621E7C93F811C080008B
:10D8C80040EA9E1006F0010E40EA8E20906293F81E
:10D8D80012E00CF00F00C00140EA56000EF07F067F
:10D8E800360146EA1C16D062D87C166393F814C039
:10D8F800400040EADE100CF0030693F815E040EA19
:10D90800462050630EF01F06987DDB7DB60146EA7F
:10D918009C06C00040EA5E109663DE07D0634CBFE9
:10D9280040F21470AD20106498074CBF40F2147098
:10D93800AD2013F0080F506414BF03230123A6E0A1
:10D94800464A1378002B00F0A18000231370444A44
:10D95800DFF830E1167843480EEB460CB0F800804B
:10D968009CF803909CF8040040EA0920804540F0A8
:10D978008D809EF80100012804D0812840F087801E
:10D98800032300E00346102E84BF10201070364891
:10D9980092F800E00022D6B2764500F1020076D275
:10D9A80010F802CC10F8016C46EA0C26DFF8D8C053
:10D9B8002CF812600132EEE72C4B1A78002A65D059
:10D9C80000221A702A4B1A78A82A1E465ED1DA7CE1
:10D9D800002A5BD106EB42009FED267A90F803E01F
:10D9E800037903EB0E2307EE903AF8EEE77A224B21
:10D9F800C7EE877A9FED217A77EEC77AFCEEE77A51
:10DA080017EE900A43F822000132082AE2D104E016
:10DA18001B4B1A78D2B300221A70012337E000BFDB
:10DA28000B0B0020D0220020180400200C0B002033
:10DA38000822002004220020490D0020C2210020D5
:10DA4800BC210020C3210020390D0020300C00200B
:10DA5800BA0D0020A10D0020A00C0020710D00209F
:10DA6800740D0020720D0020780D00206A0D002032
:10DA7800550D0020CDCCCC40600C00200080BB436D
:10DA88002C0C0020750D0020800C00200023DA07E4
:10DA980041BF83F002038D4A0120C3F3400344BF12
:10DAA800107023704E0406D5894A13780BB10020F4
:10DAB8001070864A137044F208030B403BB1834B45
:10DAC8001B7823B105F5C333824AA0331360C80716
:10DAD8000CD5804B5A79187982421FBF01222270D7
:10DAE80005F5C332A0321CBF1A6058718A0408D5E4
:10DAF8000023794A32F81320002A2FD101330C2B46
:10DB0800F7D1724B734C1B7823B9744B1B68ED1A11
:10DB1800002D04DBF5F7CCFE0123A37104E0A36814
:10DB2800013303EAE373A3606D4DFCF71DFBEB7B48
:10DB38003860E66863B16B4B0DA8DB6898479DF8C1
:10DB480034309BB9684B1868801B64280ED504E6EE
:10DB5800AB895BB1801B002808DAFEE5012323703E
:10DB68005C4A05F5C333A0331360CAE7D4F8F02044
:10DB78003B685E48574EDFF874911344E3605C4B92
:10DB8800D3F80080574B5B689847002800F0C380A3
:10DB980048464946327CF7F741FC564B1B88002B18
:10DBA80074D073691B7808EE103A06F1180A4FF022
:10DBB800000B24364F4B39F91B001988B1F57A7FD1
:10DBC80002BF0023CAF800303361DAF8003003449A
:10DBD800CAF80030336907EE900A0133012B4FEA87
:10DBE8004B02F8EEE77A336106D10023C6ED017ADD
:10DBF800C6ED007AB3601BE0D6ED006A07EE103A76
:10DC080037EEE66AB8EEC77A86EE077A36EE877A96
:10DC1800D6ED026A86ED017A77EEC77A86ED007A4C
:10DC2800E6EE276AF0EE667AC6ED036AC6ED026A8A
:10DC380031480023012929F8023013522D4930D1E7
:10DC480033690591012BC3BF03F1FF3300EE103A8E
:10DC5800D6ED037A9FED290A0490C8BFB8EEC00A32
:10DC68000392C8BF87EE800A01F0FEFB039A04986E
:10DC7800059918EE103A5BB1F8EEC87AB4EEE70AE7
:10DC8800F1EE10FA04DD4FF47A730B80002337E0CD
:10DC9800DAF800304FF47A7E03F5FA7393FBFEF35B
:10DCA80083520BF1010BBBF1030F0AF1040A06F1D1
:10DCB80014067FF47FAF0888012803D10391F9F790
:10DCC80095FE03990B88013BDFE700BF0C0B002092
:10DCD8000A040020180400200C0D0020E00A00208F
:10DCE800CC1A0020F0100020D02200203617002087
:10DCF800F40E0020E8220020780400200000000034
:10DD0800C64939F8132031F81310521A29F813208C
:10DD18000133032BF4D1C24B1B6813F0020300F04C
:10DD2800D582C04EC04B06F166005B689847002854
:10DD380000F0E280BD4B06F166001A780146F7F75D
:10DD48006DFBBB4B1B88002B43D0F06E0023B84AF9
:10DD5800B8491288DFF8CCE2B2F5C87F04BF0022C8
:10DD680041F823204FEA83090EF1660C51F8092087
:10DD78003CF91360324441F8092000212CF81310B3
:10DD880020F813100133032BE1D1A94E3388012B5E
:10DD98001CD1DEF870304FF4C87CC83393FBFCF319
:10DDA8000380DEF87420C83292FBFCF24280A24A5B
:10DDB800DEF878301288C83393FBFCF39B1A838013
:10DDC800A8F85810A8F85A10F8F760FA3388013BF9
:10DDD80033809A4B1B685B077BD5994B1B88322B8A
:10DDE80012D1E36E1A88A4F87C205A889B88A4F87C
:10DDF8008030B8F85830A4F88230B8F85A30A4F80F
:10DE08007E20A4F8843001E0002B43D0D4F86CC005
:10DE180000238B4A834E1288322A8A4A04BF002183
:10DE280042F823104FEA830906F1660E52F80910EA
:10DE38003EF91300014442F8091000222EF813207D
:10DE48002CF813200133032B1146E2D1DFF8F091AF
:10DE5800B9F80030012B18D17B4A11707B4A0C208D
:10DE68001370F9F7C3FDF36EB6F87C201A80B6F884
:10DE78007E205A80B6F880209A80B6F88230A8F8BA
:10DE88005830B6F88430A8F85A30B9F80030013B59
:10DE9800A9F800306E4B1A78DAB1E16E0022322010
:10DEA8001A70D4F8883093FBF0F30B80D4F88C30D8
:10DEB80093FBF0F34B80D4F8903093FBF0F35E487B
:10DEC80000881B1A8B80A8F85820A8F85A20F8F761
:10DED800DDF9E26EB4F8663011885B1AA4F8663092
:10DEE8005188B4F868305B1AA4F868309288B4F89E
:10DEF8006A309B1AA4F86A30FCF736F9D4F89430E3
:10DF080094ED266AD4F89C80C4F89400C3EB000B07
:10DF180007EE90BAB8EE678A002628EE066A98F8E7
:10DF280000C04C484C490DF11C0E32464B4B33F99E
:10DF3800123007EE903AF8EEE77A494B67EE867AA8
:10DF4800EEEC017ABCF1000F1CD007EE90CAF8EE97
:10DF5800E76AB7EE007AC7EE266A33F9123007EEA1
:10DF6800903AF8EEE77A37EE667A67EEA67AD1ED60
:10DF7800006AE6EE877AC1ED007AFDEEE77A17EEE1
:10DF8800903A01E033F81230438030F8023F013212
:10DF9800032A13FB036601F10401C7D1DFF8989047
:10DFA800304864237343B9F80060764393FBF6F670
:10DFB800493E07A9B6B2F7F781FE3B2ED8ED016AB4
:10DFC80011D9B4F9B830D4ED2D0A07EE903AF8EE2D
:10DFD800E77A254BF4EEE70AF1EE10FA48DD1A78F5
:10DFE80042F0080247E0F7EE007A36EEA77A1D4ABB
:10DFF80087EE877A00231D4931F913100133032B6B
:10E0080007EE901A92ED006AF8EEE77AE6EE267AC5
:10E0180067EE877AE2EC017AEDD1D2E77804002046
:10E02800502200201804002054220020EB22002057
:10E03800AA0B0020880400200200002008220020EB
:10E04800AC0B0020A0040020AE0B0020A60B002083
:10E05800A70B0020EE030020B8040020361700208C
:10E068007E040020C40400209A0B0020F003002046
:10E078001A7822F0080294ED2C0A1A7001F0F2F9CD
:10E08800DFF8C4A3D4ED2C7A8AED000A94ED2D0AAA
:10E09800D4ED2B8ADC4E20EE000AF1EE688AA7EE5A
:10E0A800A70A01F0E1F9F0EE400AB0EE680A01F0C3
:10E0B800D9F9DFEDD68A8AED010A9AED000A20EE39
:10E0C800280A01F0FDF89AED010A308020EE280AAE
:10E0D80001F0F6F8CE4B70801B681E0721D5CD489D
:10E0E80007A9F7F7EBFDD8ED026ACA4AF7EE007AFE
:10E0F80036EEA77A002387EE877AC74931F91310DD
:10E108000133032B07EE901A92ED006AF8EEE77AD6
:10E11800E6EE267A67EE877AE2EC017AEDD1BD4821
:10E128002AE0BE4E07A93046F7F7C8FD96ED010A6A
:10E1380096ED007AD6ED027A20EE000AA7EE070ADD
:10E14800A7EEA70A01F090F9B5EE400AF1EE10FA31
:10E1580011D0D6ED007AC7EE807AC6ED007AD6EDFA
:10E16800017AC7EE807AC6ED017AD6ED027A87EE9B
:10E17800800A86ED020AA948FCF720FADFEDA87AA2
:10E18800A84B9FEDA97A188028EE278ADAED007A45
:10E19800A44BF1EE677ACDED0A7ADAED017AB3F99C
:10E1A8000030F1EE677ACDED0B7A07EE903A9F4B8F
:10E1B800F8EEE77AB3F9002067EEC77A0DA8CDED3F
:10E1C8000C7A07EE902AB3F90220B3F90430F8EE7E
:10E1D800E77A0AA9CDED0D7A07EE902AF8EEE77AEC
:10E1E800CDED0E7A07EE903AF8EEE77ACDED0F7A9C
:10E1F800F7F764FD98F801309DED0F7A012B19D1DE
:10E208008B4B1B7858070FD4D4F8C830402293FBA7
:10E21800F2F29B1A07EE903AF8EEE77A77EE877AF1
:10E22800FDEEE77AC4ED327AD4F8C830402293FB89
:10E23800F2F301E0B9F800309DED0D0A07EE903ACF
:10E24800F8EEE77A37EE677AD4ED337A8DED0F7A08
:10E2580094ED347A38EE077A88EE078A9DED0F7AC6
:10E2680037EE677AE8EE077AB0EE678AC4ED337A5C
:10E2780001F026F8D4F8D4603178F7F74BFCD4F8DD
:10E28800D8309DED0E0A1844C4F8D80001F018F8EB
:10E298003178F7F73FFCD4F8DC30B0EE480A184480
:10E2A800C4F8DC0001F00CF87178F7F733FCD4F807
:10E2B800E030604A18441368C4F8E0005B44136017
:10E2C800D4F8E4300133C4F8E43005E0A4F866304B
:10E2D800A4F86830A4F86A30FBF746FFD4F8E830B1
:10E2E8003860C31A9BB207EE903A534FDFF85CA12F
:10E2F8009FED4B7AAAF80030F8EE677A3B68DFF8B2
:10E30800509193F852304D4AC4F8E80067EE877A86
:10E31800BB46C9ED007A23B92B7C002B00F0BF80E7
:10E328002EE0D2ED3B7AF5EE407AF1EE10FA04BF1A
:10E33800D2ED3C7AF8EE677A4FF0000604BF67EE3C
:10E34800877AC2ED3B7ADFF80C813D4838F9163000
:10E35800D4ED3B0A00EE103ADBF8003000EBC600C3
:10E3680093F85210B8EEC00AF7F7A0F9FDEEC07A9C
:10E3780017EE903A28F816300136032EE3D1CBE792
:10E38800BAF80030DFF8B480D9ED000AB4F80C61AF
:10E3980000EE103A08F58870B8EE400A0121F7F748
:10E3A80085F9BCEEC00AA3798DED030ABDF80C000F
:10E3B800B6FBF0F0461CB6B2A4F81861002B4BD09F
:10E3C800B8F81AB100231D491E4A01F5927C01F5DF
:10E3D8008E7932F813803CF813E039F813202CF8C2
:10E3E8001380CEEB080E12FB0BF20FFA86FA92FBA3
:10E3F800FAF2964429F813E00133042BE3D1002301
:10E408008B71A1F81A012CE09A1A00204C3D0F4498
:10E4180050220020D40400200E0400200400002014
:10E42800BD378635A40B002035FA8E3CF00300205A
:10E43800ED220020CC220020F40E00201804002039
:10E448000C050020E80C0020701900206422002030
:10E458005817002036170020B8F81A31013BA8F8E1
:10E468001A31B4F81A01B64A03B2002B4FF0000370
:10E4780013DDB2F91861B34931F81320083112FBE2
:10E4880000F231F8131092FBF6F28A1AAE4921F81D
:10E4980013200133042BEED101E0A2F81A31F3F76F
:10E4A8005FF9AA4BDFF804A31B68DFF8049313F4A1
:10E4B800801300F09680B9F80030190600F1DF806B
:10E4C800A34B1B7803F0040303F0FF0B002B73D05E
:10E4D800A04AA14B117811B194F82C1139B19F4978
:10E4E8000020086001211973002184F82C111B7B7E
:10E4F800DAF800801370032B05D14046984954225E
:10E5080000F0C4FC51E0012B06D154229448414646
:10E5180000F0BCFC002202E0022B02D10122914B48
:10E528001A70914A01231370904A1370904A00237D
:10E538001360904A1360904BC3F800808F4B98F893
:10E5480000201A70874B8E4A1B78D05C8D4B8E4A00
:10E558001870824B40441A6042788C4B07EE902A20
:10E56800F8EEE77AB2EE047AC7EE877AC27A9FEDC0
:10E57800887AC3ED007A07EE902AF8EEE77A427DB2
:10E58800C7EE877A9FED837AC3ED017A07EE902A6A
:10E59800F8EEE77A67EE877AC3ED027AFCEEE77A5F
:10E5A80017EE903A43750023C3728020F7F7D4FB27
:10E5B800012384F8843162E0DFF8A081D8ED007A85
:10E5C800F5EE407AF1EE10FA59D0F7F75FFE002326
:10E5D800C8F800305F4B83F800B05F4B01221A7314
:10E5E8004DE0B9F8002012063ED55A4A1078411E6F
:10E5F800012959492DD8DFF894E15F4BDEED017A06
:10E608009FED637A1A685F4B67EE877A18789FEDFB
:10E61800627AFCEEE77A104417EE903AC372DEEDA8
:10E62800027A67EE877AFCEEE77A17EE903A43753E
:10E63800537807EE903AF8EEE77A77EEA77AFCEE91
:10E64800E77A17EE903AD370D37A5373537DD37524
:10E6580004E0032802D11370012301E00B7B01338E
:10E6680080200B73F7F767FB394B1B785B0706D4E1
:10E6780094F884311BB1324B012283F82C21474B8B
:10E68800DFF830811B78B3B12F4B454AB3F9061038
:10E69800B2F89A3199420EDC5379012B01D0192B2B
:10E6A80002D192F8E82132B90E2B04D0082B1CBFF6
:10E6B8000023A8F80430DAF8003093F818A1BAF16A
:10E6C800000F7FD0B9F800309E077BD094ED2C0A5C
:10E6D800D4ED2B7A94ED2D8A20EE000AA7EEA70A36
:10E6E800A8EE080A00F0C0FE88EE000ADFED2D7AD9
:10E6F800B4EEE70AF1EE10FA5ED900F055FE104BC1
:10E70800D3ED627A20EE270A00F0DAFDB0F5617FDA
:10E71800A8BF4FF4617007EE900AB8EEE70ADFED84
:10E72800227A80EE270AF7F704FA07EE90AAF8EEA5
:10E73800E77A27EE800A00F0C3FD80B23DE000BF13
:10E748001804002034050020E80C0020740B002079
:10E75800ED220020941A002004000020A01A0020B6
:10E7680048050020951A0020981A0020B01A0020A9
:10E77800A41A0020A81A0020C01A0020961A002007
:10E78800A0120108971A00200000A041B41A002026
:10E7980000007A445555553F9A99993F1400002036
:10E7A800CC1A00208FC2753CEFB6B044F40E00209E
:10E7B8002C1700202E1700200020B8F80630184427
:10E7C800A8F80600864B3868B5F86E210093854B8B
:10E7D8001D68854B196800F15803A847834B844985
:10E7E8001F78032F16D9D4F88C315D88B5F5FA7FD8
:10E7F80010D2B8F90400B1F904E080EAE076A6EB9B
:10E80800E0766A42931B9E4503DBAB197345A8BFAC
:10E8180073468B80B8F80650B1F802E0B1F800C032
:10E82800D4F88C81B1F90490724A0020B84202F100
:10E83800100233D298F9013052ED045ADFF8C0A122
:10E848005B4209FB03F307EE903A0FFA8CF306EEEE
:10E85800903A2BB206EE103A0FFA8EF3B8EEE77A3A
:10E8680007EE903AF8EEE77AB8EEC66A67EEA57A50
:10E8780052ED065AE6EE257AF8EEE66A12ED056ADA
:10E88800E6EE867A52ED036AE7EE267AFDEEE77A3F
:10E8980017EE903A2AF810300130C7E7564B1A782D
:10E8A80002F0040202F0FF03002A79D0534B544AC5
:10E8B800DB780493138801209646B8421AB207D22F
:10E8C8003EF910309A42B8BF1A4693B20130F4E7C5
:10E8D8004C48D4F8508200684588AA42C8BF5D1BDE
:10E8E800494B1B6803F480520592484AB2F906C0A6
:10E8F800474AD2F80090424A03F0100BD4F88C3102
:10E908000393CCBFADB2002502EB4707BA423ED015
:10E918001388059E5B1B9BB222F8023B1BB266B1B3
:10E92800B8F80EE0F445C7BFB9F802E0B0F802A0A5
:10E93800B0F804E0B9F800A005E0049EB0F802A021
:10E9480056B1B0F804E0734503DB5345A8BF5346FE
:10E958009E4622F802ECD9E7B0F800E0734503DBE5
:10E968005345A8BF53469E4622F802ECB8F810302B
:10E978009C45CBDABBF1000F01D0838804E0039BF0
:10E988001B78002BC2D1038822F8023CBEE794F81A
:10E998005432204D013BDBB2182B00F2448109E0D0
:10E9A800BB42F4D21C4A32F81300154A22F813006D
:10E9B8000133F5E701229A40184B1340002B00F071
:10E9C8003281174B1B8813F4807F104B2CD0154ACB
:10E9D8001188ADF834105188ADF83610928839E0B6
:10E9E800561C0020F8000020E8210020D61700203F
:10E9F800A4170020B0050020ED22002014220020DA
:10EA0800E0170020F418002008220020E80C00205D
:10EA1800F0180020F6030020EC210020992098012E
:10EA28002C1700202E1700200A88ADF834204A88B9
:10EA3800ADF836208A88B049ADF838200968C8048E
:10EA48000AD5AE49B3F90600D1F85012C9898842EF
:10EA580002DA5242ADF83820A94FB7F902204FF434
:10EA68007A7102F5E1624A434FF4616092FBF0F279
:10EA7800A2F5FA72ADF84C20B7F9002002F5E16270
:10EA88005143A04A91FBF0F11288A2F2DC52A1F5A1
:10EA9800FA71ADF83A20D4F85022ADF84E10D28968
:10EAA8001988891AADF83C105988891AADF83E10B2
:10EAB8009988891AADF84010D988891AADF842109A
:10EAC8001989891AADF844105989891AADF8461080
:10EAD8009989DB89891A9A1AADF84810ADF84A2045
:10EAE8000023002225F813200133082BF9D1864A88
:10EAF800864B12680392864A1B78126885490492ED
:10EB0800854E072202FB031B594572D00B7833B19F
:10EB180003F1150201239340039A134065D011F8BD
:10EB280006CC049B11F805AC11F8034C11F8018CC4
:10EB3800CCEBCC0E03EB4E0E6420BEF90020BEF9E0
:10EB480002309B1A9BB211F9022C4FEA53095A431F
:10EB58004FEA4A0792FBF0F214A8C9EB020292B2FC
:10EB6800074414B937F81C0C0CE0B6F9000037F963
:10EB78001C7CB84208DA0444844203DBA7423846C6
:10EB8800A8BF2046308008E007DD041BBC4203DB39
:10EB98008442A8BF044627463780DEF80A4011F9A8
:10EBA800047C012000FA0AF02042308812B217FBD8
:10EBB80000F014BF4FF0FF340124642790FBF7F0F6
:10EBC80090420ADB4FFA88F25A4392FBF7F2C9EBFC
:10EBD800020212B28242A8BF0246504B33F81C9080
:10EBE80002FB049423F81C4000E03380023607310E
:10EBF8008AE7474B4A4FD3F8008000260E2202FBD3
:10EC0800068237F8023F92F90640F0B214FB03F38C
:10EC1800642493FBF4F43C80FBF7B6FC01362044F3
:10EC2800082E3880EAD1344E394C336813F0200F5F
:10EC380032D00020FBF7A8FC288080460120FBF793
:10EC4800A3FC314B354F1B686880190624D52B4B24
:10EC5800D4F800C0D3F87832294A1B78012B1FD189
:10EC680013889CF91410B2F9022011FB03F34FF03A
:10EC7800320E93FBFEF399B29CF906305B42534384
:10EC88006FF0310293FBF2F20A44424493FBFEF325
:10EC98000B443A8018447880D4F800E0002318E048
:10ECA8009CF9061053884FF0320E11FB03F393FBC7
:10ECB800FEF308EB0301398011889CF9142012FB3C
:10ECC80001F292FBFEF21044E5E70133082BEA5308
:10ECD80028D00E2101FB03E135F91300B1F900201A
:10ECE800B1F9021090424FEA4307EEDB0AB28242C2
:10ECF800A8BF0246E9E700BF082200201804002048
:10ED08009A1A0020E0170020740B0020F818002041
:10ED1800F80E0020FF1800206E060020F6030020E1
:10ED2800F4030020544FD7F88CA19AF90830A3B9FE
:10ED380097F8548208F1FF33182B72D8DFE803F0F4
:10ED48003571714F7171714871717171715971714A
:10ED58007171714F657171593500DFF82C914FF061
:10ED68000008464B39F9021FBAF90620882000FB33
:10ED78000830FBF745FA22680E2380B203FB08220D
:10ED8800A9F80000B2F90030B2F9022000B29842A6
:10ED980003DB13B28342A8BF034608F10108B8F1A8
:10EDA800080FA9F80030DCD1C2E79AF8043013B193
:10EDB8000020698908E0324B1B7803F0040303F054
:10EDC800FF00002BF4D10146FBF75CFE012429E08B
:10EDD8000020E988FBF756FE0120298905E000207C
:10EDE8002989FBF74FFE69890120FBF74BFE0224B6
:10EDF80018E00224A01E35F81410C0B20134FBF745
:10EE080041FE082CF6D106240CE00324E01E35F858
:10EE18001410C0B20134FBF735FE072CF6D10424D8
:10EE280000E0002433689A0602D4B8F1050F0AD12D
:10EE380020462988FBF726FE601CC0B26988FBF7CC
:10EE480021FE0234E4B23368DB0208D497F8C036F6
:10EE5800002B3EF482ACFBF7DFFAFEF77EBC094ECE
:10EE680000256019C0B236F8021FFBF70BFE0D2D06
:10EE7800ECD00135F5E700BF180400209806002003
:10EE8800ED220020EE0C0020F403002010B5431EF4
:10EE98000A44914204D011F8014B03F8014FF8E7F6
:10EEA80010BD02440346934202D003F8011BFAE75F
:10EEB800704700000D4B30B51D6810F8013BEA188B
:10EEC800527802F00302012A11F8012B05EB020423
:10EED80008BF2033647804F00304012C08BF2032F3
:10EEE8009B1A01D1002AE8D1184630BD0401002040
:10EEF80010B50246134601321C78002CFAD1013BAA
:10EF080011F8012B03F8012F002AF9D110BDC9B25D
:10EF1800034610F8012B1AB18A42F9D118467047F6
:10EF280000290CBF184600207047034613F8012B30
:10EF3800002AFBD1181A013870470000104B70B531
:10EF48001E680A44914217D010F8013BF4186478FF
:10EF580004F00304012C11F8014B06EB040508BF6B
:10EF680020336D7805F00305012D08BF20341B1BE5
:10EF780003D1002CE6D100E00023184670BD00BF85
:10EF88000401002010B5034632B111F8014B03F813
:10EF9800014B013A002CF7D11A44934203D00021C7
:10EFA80003F8011BF9E710BD30B5037823B90B78D6
:10EFB800002B18BF002030BD034601301A783AB143
:10EFC80000228C5C34B19D5CA542F5D10132F8E792
:10EFD800104630BD184630BD00210A2200F0E6B8C0
:10EFE800174B2DE9F0411D68AC6D06460F46FCB97C
:10EFF800502000F0E9F8A8658460AB6D04604460B7
:10F008001C61DC60AB6D9C615C61AB6DDC629C6219
:10F01800AB6D5C631C63AB6DDC639C63AB6D5C6464
:10F028001C64AB6DDC649C64AB6D1C77AB6D5C627F
:10F0380030463946AA6D0123BDE8F04100F002B818
:10F0480068010020F0B548B9106838B9F0BD17F864
:10F05800016B5EB1B542FAD12BB1204604460F468A
:10F0680014F8015BF3E714600370F0BD4DB9156047
:10F078002846F0BD17F8016BAE4207D0002EF9D133
:10F088001C4623460F4613F8015BF3E715B1002130
:10F09800217000E02B461360F0BD0123FFF7D2BFBB
:10F0A8002DE9F047404CD4F800900F463D4615F83E
:10F0B80001EB09EB0E04667806F0080404F0FF067D
:10F0C8000CB12F46F2E774462D2C03D1BD1C7C7879
:10F0D800012603E02B2C04BF7C78BD1C13B1102B38
:10F0E8000AD15AE0302C56D12C7804F0DF04582C81
:10F0F8004CD16C7810230235002E14BF4FF0004815
:10F108006FF000480027B8FBF3FABE4603FB1A88E5
:10F1180009EB040C9CF801C01CF0040F01D0303C32
:10F128000BE01CF0030C1BD0BCF1010F0CBF4FF01F
:10F13800370C4FF0570CCCEB04049C4210DAB7F1B3
:10F14800FF3F0AD0D64506D801D1444503DC03FB6E
:10F158000E4E012701E04FF0FF3715F8014BD7E7B6
:10F168007C1C73460AD1002E4FF0220114BF4FF0C9
:10F1780000436FF0004301602AB911E00EB1CEF1EF
:10F1880000036AB107B1691E116009E03024002B41
:10F19800B2D10823B0E70A23AEE7302CACD1A3E7FD
:10F1A8001846BDE8F08700BF0401002030B51346BB
:10F1B800044A05460C46106829462246BDE83040F8
:10F1C800FFF76EBF68010020024B0146186800F087
:10F1D80003B800BF6801002070B5CC1C24F00304FC
:10F1E80008340C2C38BF0C24002C064603DA0C23F8
:10F1F8003360002070BD8C42F9D3204A1368104652
:10F208001946A1B10A68121B0ED40B2A03D90A6049
:10F218008B188C501FE08B420DBF5A684A685A60A1
:10F22800026018BF0B4616E00B464968E9E7144D23
:10F238002B681BB9304600F025F828603046214677
:10F2480000F020F8421C0346D1D0C51C25F0030568
:10F2580085420AD11C6003F10B001A1D20F007003B
:10F26800821A0AD05142995070BD3046E91A00F00E
:10F2780009F80130BBD02B46ECE770BDE022002036
:10F28800DC22002038B5064C0023054608462360DA
:10F2980000F008F8431C02D1236803B12B6038BD85
:10F2A800F4220020044A05491368002B08BF0B46C6
:10F2B8001844106018467047E4220020F822002005
:10F2C80084B08DED010A019BC3F3C750A0F17F0103
:10F2D8001E2927DC4A1C22DB16294FEAD3720ADDD5
:10F2E800C3F3160343F40003963883405042434067
:10F2F800981804B07047144BDDED017A03EB8203D4
:10F3080093ED007A77EE277ACDED037ADDED037A77
:10F3180077EEC77A17EE901A21F0004353B9002010
:10F3280004B07047DDED017AFDEEE77A17EE900A3A
:10F3380004B07047C1F31603C1F3C75143F4000387
:10F34800C1F19601CB40D1E76037010800B510EE56
:10F35800103A134A23F00043934283B018DDB3F107
:10F36800FF4F04DB30EE400A03B05DF804FB68464B
:10F3780000F0AEFA00F001004000C0F101009DED80
:10F38800000ADDED010A00F02FFF03B05DF804FB71
:10F39800DFED040A012000F027FF03B05DF804FB4D
:10F3A800DA0F493F0000000010B52DED028B2A4C02
:10F3B8008AB0F0EE408A00F0B3F894F900300133D7
:10F3C800B0EE408A04D0B0EE680A01F02DF928B9F1
:10F3D800B0EE480A0AB0BDEC028B10BDB0EE680A68
:10F3E80001F0D2F8F7EE007AB4EEE70AF1EE10FA7F
:10F3F800EEDD0123194A009318EE900A00230192CA
:10F408000893FDF715FC02460B461548CDE9042381
:10F41800CDE9022300F0D4FF94F90030022B8DEDE2
:10F42800060B0FD0684600F0C7FF58B1089B73B9A8
:10F43800DDE90601FEF706F900EE100A0AB0BDEC98
:10F44800028B10BD01F080F921230360EEE701F083
:10F458007BF9089B0360EBE76C0100206837010823
:10F468007037010800F07EB910B52DED028B2A4CDB
:10F478008AB0F0EE408A00F073FB94F90030013353
:10F48800B0EE408A09D0B0EE680A01F0CDF820B19C
:10F49800F5EEC08AF1EE10FA05D4B0EE480A0AB0CB
:10F4A800BDEC028B10BD01231C4A009318EE900A94
:10F4B800002301920893FDF7BBFB2478CDE90401F2
:10F4C800CDE902019CB900220023CDE90623684654
:10F4D80000F072FFA8B1089BC3B9DDE90601FEF789
:10F4E800B1F800EE100A0AB0BDEC028B10BD002086
:10F4F800002102460B46FDF719FD022CCDE9060155
:10F50800E5D101F021F921230360E4E701F01CF9BA
:10F51800089B0360E1E700BF6C0100207437010815
:10F5280008B510EE102A22F00043B3F17E5F2DEDEE
:10F53800028B12D00ADCB3F17C5F19DAB3F10C5FED
:10F548006ADCBDEC028B9FED760A08BD30EE400AFE
:10F5580080EE000ABDEC028B08BDBDEC028BDFED2E
:10F56800717A9FED710A002AC8BFB0EE670A08BD1C
:10F57800002AC0F28C80F7EE008A38EEC00AB6EE98
:10F58800008A20EE088AB0EE480A00F0E9FADFEDBA
:10F59800677A9FED673A9FED674ADFED672ADFEDEF
:10F5A800673A9FED675ADFED674ADFED676ADFED7F
:10F5B800675A9FED677AA8EE273AE8EE223AA3EE5B
:10F5C800084AE3EE884AA4EE085A10EE103AE5EE2F
:10F5D800086A23F47F6323F00F03E4EE885A07EEEA
:10F5E800903AA6EE887AF0EE486AE5EE888AE7EE69
:10F5F800E76AB0EE406A27EE088A30EE270A88EEFE
:10F60800288A86EE800AA8EE060ABDEC028B37EE41
:10F61800800A30EE000A08BD60EE007ADFED431A7A
:10F628009FED433A9FED434A9FED432ADFED433A6E
:10F638009FED436ADFED434A9FED435ADFED435A9E
:10F648009FED437ADFED436ADFED432AA7EEA13A47
:10F65800BDEC028BA3EE274AE7EE823AA4EE276AB6
:10F66800E3EEA74AA6EE275AE4EEA75AA5EE277AB4
:10F67800B7EE006AA5EEA76A67EE277AC7EE867A24
:10F68800E0EE676A30EE660A32EEC00A08BDB7EEF1
:10F69800008A30EE080AF6EE007A60EE277ADFED8F
:10F6A800232ADFED233A9FED243ADFED224A9FED2E
:10F6B800234ADFED235A9FED235ADFED236A9FED9E
:10F6C800236A9FED237AE7EEA23AA7EE834AE3EE98
:10F6D800A74AA4EE275AE4EEA75AA5EE276AE5EE54
:10F6E800A76AA6EE278AA6EEA77AF0EE488A27EE42
:10F6F800278AB0EE670A00F033FAC8EE287ADFED01
:10F70800176A9FED177AE7EE806AF0EE667A37EEB1
:10F71800800AF0EE006AA0EE667AB0EE470A19E7B2
:10F72800DB0FC93F00000000DB0F494008EF11382C
:10F73800047F4F3A461124BD2EC69D3D613330BF2C
:10F74800A80A4E3E2D57014090B0A6BE39D119C027
:10F75800ABAA2A3E6821A233DA0FC93F6821A2B3B7
:10F76800DA0F494010B582B0CDED010A019B23F0B4
:10F778000042B2F1FF4FF0EE407A19DC10EE100AA9
:10F7880020F00041B1F1FF4F12DCB3F17E5F49D0A8
:10F798009C1704F0020444EAD07479B9022C3ED0D4
:10F7A8009FED400A032C18BFB0EE670A02B010BDE7
:10F7B8009DED017A37EE270A02B010BD12B3B2F1FF
:10F7C800FF4F34D0B1F1FF4F1CD08A1AD2153C2A12
:10F7D80022DC002B4BDB9DED017A87EE870A00F0D7
:10F7E800D3FE00F0F5FD012C3AD0022C2FD0002CCE
:10F7F800E2D09FED2D7ADFED2D7A30EE070A30EE5C
:10F80800670AD9E7DFED2A7A9FED2A0A0028A8BF00
:10F81800B0EE670A02B010BD9FED250AE3E79FED41
:10F82800230AC9E702B0BDE8104000F0D1BDB1F12C
:10F83800FF4F21D0022CF2D0032C2AD0DFED1E7A04
:10F848009FED1E0A012C08BFB0EE670AB4E79FEDD2
:10F85800167ADFED167A30EE070A37EEC00AABE704
:10F8680010EE103A03F1004300EE103AA4E73C32E0
:10F87800B1DA9FED120AB6E7022C10D0032C0BD098
:10F88800DFED0F7A9FED0F0A012C08BFB0EE670A73
:10F8980092E79FED040A8FE79FED0B0A8CE79FED37
:10F8A8000B0A89E7DB0F49C02EBDBB33DB0F49408C
:10F8B800DB0FC93FDB0FC9BF00000080000000005C
:10F8C800DB0F49BFDB0F493FE4CB16C0E4CB164042
:10F8D80070B510EE103A944A23F00044944286B072
:10F8E80010EE106A054666DD904A94421ADC002B39
:10F8F800DFED8F7A8F4A24F00F0440F3DD809442C5
:10F9080070EE677A66D09FED8C7A77EEC76A012031
:10F9180077EEE67AC5ED006A77EEC77AC5ED017A2B
:10F9280006B070BD854A944266DDB4F1FF4F49DAEE
:10F93800E215863AA4EBC25307EE103AFDEEC76A09
:10F94800DFED7F7AF8EEE66A37EE667ACDED036A88
:10F9580027EE277AFDEEC76AF8EEE66A37EE667A92
:10F96800CDED046A67EE277AF5EE407AF1EE10FAEB
:10F97800CDED057A40F0B380F5EE406AF1EE10FA6D
:10F9880014BF022301236F4902208DE8030003A856
:10F99800294600F037F9002E12DA95ED007AD5EDF8
:10F9A800017AB1EE477AF1EE677A404285ED007A46
:10F9B800C5ED017A04E0002285ED000A42600020CE
:10F9C80006B070BD70EE407A0020C5ED017AC5ED35
:10F9D800007AF5E7DFED5C6A9FED5C7A77EEE67A10
:10F9E800012077EEC76A77EEE67AC5ED006A77EE12
:10F9F800C77AC5ED017AE3E700F0C6FDDFED546A8A
:10FA0800DFED4B5A9FED4C7AF6EE007AE0EE267A5F
:10FA1800FDEEE77A17EE900AF8EEE76A1F28B1EED6
:10FA2800666AA6EE250A66EE877A1DDC494A411EFB
:10FA380024F0FF0352F82120934215D030EE677A64
:10FA480085ED007A30EE470A002E30EE670A85ED24
:10FA5800010AB5DAB1EE477AB1EE400A85ED007ACF
:10FA680085ED010A4042ABE730EE677AE41517EE00
:10FA7800103AC3F3C753E31A082BE1DDDFED327AFE
:10FA88009FED327AF0EE405AE6EE275A30EE650ADC
:10FA9800A6EE270AF0EE407AD6EE877A35EEE77AB8
:10FAA80017EE103AC3F3C753E41A192C2CDC85ED72
:10FAB800007AB0EE650AC5E7944270EE277A10D056
:10FAC8009FED1D7A77EE876A4FF0FF3077EEE67A82
:10FAD800C5ED006A77EE877AC5ED017A70E70323F2
:10FAE80051E7DFED196A9FED197A77EEA67A4FF0A4
:10FAF800FF3077EE876A77EEE67AC5ED006A77EE33
:10FB0800877AC5ED017A5BE79FED137A9FED135A6B
:10FB1800B0EE650AA6EE070A75EEC07AE6EE077A39
:10FB2800D6EE857A8AE700BFD80F493FE3CB164067
:10FB3800800FC93FD00FC93F43443537800F494331
:10FB480000008043FC3701080044353708A3852EA0
:10FB580084F9223F7C37010800A3852E32318D2499
:10FB680010EE103A23F00042B2F1FF4F70B430D2D9
:10FB78006AB3002B3DDBB2F5000F4FEAE3512CD3FB
:10FB8800A1F17F02C3F31603D10743F4000348BF72
:10FB98005B00002456105B00254619214FF0807247
:10FBA800A818984202DC1B1A8518144401394FEA38
:10FBB80043034FEA5202F3D113B104F001031C448A
:10FBC800641004F17C5404EBC65300EE103A70BC88
:10FBD8007047A0EE000A70BC704713F400020DD104
:10FBE8005B00180202F10102FAD5C2F101021144C8
:10FBF800C6E730EE400A80EE000AE8E70122114429
:10FC0800BEE700BF2DE9F04F2DED048BD7B05F1E86
:10FC1800D74C649D0293D31E48BF131D54F825602A
:10FC28000191DB1023EAE3736FEA030BB91903931D
:10FC3800824602EBCB0BA3EB070314D41944659857
:10FC480001311AAA002BAABF50F82340DFEDCC7A65
:10FC580007EE904A03F10103A8BFF8EEE77A8B425A
:10FC6800E2EC017AEED1002E1ADB029B1AA9741C71
:10FC780001EB840442A89D00002FC0F2BA81DFED99
:10FC8800C07A52464B1933ED017AF2EC016A994277
:10FC9800E6EE877AF7D10431A142E0EC017AEBD1A4
:10FCA800029ADFEDB48A9FEDB48A06F18043013BE6
:10FCB8009B00C2EB827906AA03F10408134490441E
:10FCC80004934FEA89093446A50056AB2B44002C0F
:10FCD80013ED140A18DD42A94B1905AA60EE287A1B
:10FCE800B0EE407AFDEEE77A73ED016AF8EEE77A56
:10FCF8008B42A7EEC87A37EEA60ABDEEC77A17EE92
:10FD0800100A42F8040FE9D1584600F0A9FCB0EEF9
:10FD1800409AB4EE000A29EE000A00F03DFCF2EE2B
:10FD2800007AA0EE679ABBF1000FFDEEC99AF8EED3
:10FD3800E97A39EE679A40F34181601E06AACBF151
:10FD4800080352F8201041FA03F202FA03F30DF106
:10FD5800180EC91A4EF8201019EE900A1044CBF16B
:10FD6800070309EE900A1941002939DD19EE903A86
:10FD7800002C03F1010309EE903A40F3CB810022F5
:10FD880010460DF1140E08E0C3F5807C13B1CEF8CF
:10FD980000C00120013294420CDD5EF8043F0028C7
:10FDA800F2D00132C3F1FF039442CEF800304FF095
:10FDB8000100F2DCBBF1000F10DDBBF1010F00F018
:10FDC8000481BBF1020F09D1621E06AB0DF1180EBA
:10FDD80053F8223003F03F034EF82230022959D05D
:10FDE800B5EE409AF1EE10FA66D1631E9E420BDC26
:10FDF80006AA1544002255F8040D454542EA0002BA
:10FE0800F9D1002A40F07081731E06AA52F82330F7
:10FE1800002B40F07C81049B4FF0010E53F8042D19
:10FE28000EF1010E002AF9D0A644631C73452FDC9D
:10FE3800039A9D18029A05F18045A0180EEB020C52
:10FE4800659A013D02EB85051AAA02EB800002EBD8
:10FE58008C0C42AA02EB830455F8043F07EE903A53
:10FE6800F8EEE77A002FE0EC017ADFED457A0BDB5C
:10FE7800524600EB0901034633ED017AF2EC016AC0
:10FE88008B42E6EE877AF7D16045E4EC017AE3D15C
:10FE9800744619E7B7EE000A30EE499A00289FD059
:10FEA8005846059100F0DCFB39EE409A0599B5EE0D
:10FEB800409AF1EE10FA98D0B0EE490ACBF1000062
:10FEC800029100F0CDFB9FED2C7A0299B4EEC70A9F
:10FED800F1EE10FAC0F27E81DFED267A60EE277A25
:10FEE80006A8FDEEE77A631CF8EEE77A0BF1080B3B
:10FEF800A7EEC70AFDEEE77ABDEEC00A10EE102A9B
:10FF080040F8242017EE902A40F823205846B7EEF0
:10FF1800000A0393029100F0A3FB039B0299002BB4
:10FF2800C0F2C78003F1010E4FEA8E0242AC06A868
:10FF38009FED107A1044A71870ED017AF8EEE77A71
:10FF480067EE807A20EE070A67ED017AA742F3D1BF
:10FF5800043A17440025002EC0F2A880002DC0F2F4
:10FF6800A580064CDFED067A384600220CE000BF7B
:10FF7800143B01080000803B00008043203B01083F
:10FF880000000000AA4208DCF4EC016AB0EC017A37
:10FF980001329642E6EE877AF4DA56AA02EB850237
:10FFA80001357545A7F1040742ED287AD3D1649A43
:10FFB800032A5FD8DFE802F0673737B010D1631E35
:10FFC80006AA52F823100912CEE6621E06AB0DF1FE
:10FFD800180E53F8223003F07F034EF82230FDE666
:10FFE800F6EE007AB4EEE79AF1EE10FA0ADA00219A
:08FFF800F6E65FED1D7A04310D
:020000040801F1
:10000000A142E0EC017A7FF43BAE4DE619EE903A66
:10001000002C03F1010309EE903AC8BF02213FF71B
:10002000B2AEF7EE007A37EEC99A0221DCE62EAACC
:100030005FED2B7A02EB8E0E3EED017A964577EE60
:10004000877AF9D1002943D0DDED2E6A019AB1EE0D
:10005000677A002B76EEE77A82ED007A09DD2FA829
:100060000122B0EC017A0132934277EE877AF8DA16
:1000700009B1F1EE677A019BC3ED017A19EE903A6E
:1000800003F0070057B0BDEC048BBDE8F08F2EAA3B
:100090005FED437A02EB8E0E3EED017A013B5A1C76
:1000A00077EE877AF8D109B1F1EE677A019BC3ED5B
:1000B000007AE3E75FED4C7A73E7649A032ADDD8B0
:1000C000DFE802F0130202805FED517A0029BBD114
:1000D0009DED2E7A019A002BC2ED007A77EE677AB9
:1000E000BDDC019BC3ED017AC8E75FED597ADAE721
:1000F00006AAABF1080B52F82320002A7FF40AAFBE
:1001000006AA02EB830252F8040D013BABF1080B87
:100110000028F8D0FEE64FF0010E89E600204DE6FB
:10012000002B4FDD9A0056A810442EAD141D10ED83
:10013000287A2C44A81870ED017A77EE276AA84235
:1001400077EEE67A77EE277AB0EE667A64ED017A9A
:10015000C0ED006AEFD1012B34DD131D56AC144401
:10016000034414ED287A02442FAC184672ED017A4C
:1001700077EE876AA24277EEE67A77EE877AB0EE7C
:10018000667A60ED017AC2ED006AEFD15FED827AA6
:1001900030AA33ED017A934277EE877AF9D1A9B18B
:1001A000DDED2E6A9DED2F7A019AF1EE677AF1EE80
:1001B000666AB1EE477AC2ED027AC2ED006A82ED5C
:1001C000017A5BE75FED907A0029E9D101982E9AD8
:1001D0002F9BC0ED027A026043604FE7BDEEC00A7C
:1001E00006A810EE102A234640F8242092E600BF0D
:1001F00008B510EE103A23F00042B2F1465F2DED43
:10020000028BB0EE407A12DAFDEEC07A17EE901A49
:1002100019BB431C134300F0AA80012800F084801E
:10022000BDEC028BBFEE000A80EE070A08BD534901
:100230008A4212DD002BB8BFB1EE407ADFED507A72
:100240009FED500AB8BFF1EE600A77EEE07A30EE2B
:10025000477ADFED4D0A37EE277A67EE076A9FEDA2
:100260004B8A9FED4B2ADFED4B8ADFED4B1A9FED5A
:100270004B3ADFED4B2A9FED4B4ADFED4B3A9FEDBA
:100280004B5ADFED4B4A9FED4B6ADFED4B5A9FED2A
:100290004B0A3A4966EEA67A26EE871AA7EE882A16
:1002A0008A42E7EEA81AA2EE273AE1EEA72AA3EEC9
:1002B000274AE2EEA73AA4EE275AE3EEA74AA5EEB4
:1002C000276AE4EEA75AF0EE467AE5EEA67AB0EE9B
:1002D000606AA7EE816AE6EE260AE1EE000A37EED2
:1002E000200A24DC01281FD0FFEE006AC6EE806AD7
:1002F00010EE103A16EE902A23F47F6322F47F6208
:1003000023F00F0322F00F0200EE102A06EE103A3F
:10031000F7EE007AE6EE007A36EE477A70EEC70A1C
:10032000E0EE807AA7EEA60ABDEC028B08BD07EED0
:10033000900AB8EEE76A60EE006A70EE067A9B17E4
:10034000C6EEA77A03F00203C3F10103BDEC028BF2
:10035000F0EE005A77EEE00A00EE103A37EE607ADF
:10036000F8EEC06AA7EE656A26EE860A08BD00F0C0
:100370000FF9B7EE007A87EE000AD5E73FA12C3FD0
:1003800068212233DA0F493F000000005FAE9BB7BF
:1003900045F4A3388453D9377AC09538C8261A3A19
:1003A000B937813916696B3B48DEBE3AA427B33CA6
:1003B0001F37113C8988083ED10D5D3DABAAAA3E8E
:1003C00000207047000000009FED010B704700BF48
:1003D000000000000000F87F38B510EE105A25F03C
:1003E0000044B4F1A14FF0EE407A0BDBB4F1FF4FC3
:1003F00058DCDFED547A9FED540A002DC8BFB0EEF3
:10040000670A38BD514B9C425DDCB4F1445F4CDB64
:100410004FF0FF3367EEA75A9FED4D1A9FED4D2A1F
:100420009FED4D3ADFED4D1ADFED4D2A9FED4D4A20
:10043000DFED4D3A9FED4D5ADFED4D4A9FED4D6A90
:10044000DFED4D6A25EEA57A5A1CA7EE012AE7EEEC
:10045000212AA2EE073AE2EE873AA3EE074AE3EE3C
:10046000874AA4EE075AE4EE876AA5EE076A26EEED
:10047000877A66EE256A3ED0404A41499B001A447D
:1004800076EE876A92ED007A96EEA77A0B44002DFD
:1004900093ED000A77EE677A70EE677A28DBB0EEAC
:1004A000670A38BD30EE000A38BD9FED367A30EE6F
:1004B000077AF7EE006AB4EEE67AF1EE10FAA7DDFD
:1004C000B0EE670A38BD00F063F82F4B9C4219DC90
:1004D000A3F5D0039C422ADCF0EE007ABFEE007A4E
:1004E000A0EE277A002370EE277AC7EE277A91E7ED
:1004F000B1EE670A38BD76EE876AB0EE670AA6EEFF
:10050000E70A38BD214B9C420BDCF7EE087AB7EEC8
:10051000007AA0EE277A022370EE677AC7EE877A18
:1005200078E7FFEE007AC7EE807A032372E7F7EEF2
:10053000007A30EE677A70EE277A0123C7EE277AC9
:1005400068E700BFDB0FC93FDB0FC9BFFFFFDF3E1E
:10055000D769853C59DA4B3D356B883D21A215BDE5
:100560006BF16EBD6E2EBA3D95879DBD2549123E3D
:10057000388EE3BDABAAAA3ECDCC4CBE4C3B0108A5
:100580005C3B0108CAF24971FFFF973FFFFF1B4028
:1005900010EE103A23F0004300EE103A704700BF0F
:1005A00010EE102A22F00041CB0D7F3B162B17DCFA
:1005B000002B10EE100A19DB1A491941114222D002
:1005C000DFED197A70EE277AF5EEC07AF1EE10FAC7
:1005D00019DD002A18DB20EA010300EE103A70470B
:1005E000B1F1FF4F0FD330EE000A7047DFED0E7A06
:1005F00070EE277AF5EEC07AF1EE10FA03DD002AEC
:1006000008DB9FED0A0A70474FF4000242FA03F339
:100610001844E0E70029FFEE007A18BFB0EE670A41
:10062000704700BFFFFF7F00CAF249710000000061
:1006300010EE103A33F0004001D102207047A0F5CF
:100640000003B3F1FE4F01D204207047054B421E58
:100650009A4201D803207047A0F1FF40B0FA80F021
:1006600040097047FEFF7F0008B510EE103A33F0E6
:1006700000422DED028B11D0B2F1FF4F11D2B2F535
:10068000000F13D3D20D0244FE2A2EDC002A1ADDFD
:1006900023F0FF4343EAC25300EE103ABDEC028B55
:1006A00008BDBDEC028B30EE000A08BD1D4BDFED2E
:1006B0001E7A984220EE270A22DB10EE103AC3F38E
:1006C000C752193ADFE712F1160F1EDA4CF2503317
:1006D00098420ADC9FED158AF0EE400AB0EE480A17
:1006E00000F02AF820EE080AD8E79FED118AF0EE14
:1006F000400AB0EE480A00F01FF820EE080ACDE7E5
:10070000DFED0A0A20EE200AC8E7193223F0FF4382
:1007100043EAC253DFED077A00EE103A20EE270AD3
:10072000BCE700BFB03CFFFF0000004C6042A20DE0
:10073000CAF249710000003310EE103A23F0004273
:1007400010EE903A03F00043134300EE103A704766
:10075000014B1868704700BF680100200004004882
:1007600010000102000400482000010200100402F1
:1007700008001102A0070108880701088607010880
:1007800084070108FFFFFFFF0A01000301030203C2
:100790000303040305030603070308030903FFFF1C
:1007A0000003010302030303040305030603070315
:1007B00008030903FFFF0000524F4C4C3B504954C3
:1007C00043483B5941573B414C543B506F733B505E
:1007D0006F73523B4E6176523B4C4556454C3B4DF8
:1007E00041473B56454C3B0000000000A221010858
:1007F0000000000001000000A72101080100000026
:1008000002000000AE210108020000000300000009
:10081000B72101080300000004000000BD21010809
:100820000500000005000000C221010806000000CC
:1008300006000000CC2101080700000007000000AE
:10084000D52101080800000008000000DE21010891
:100850000900000009000000E72101080A0000006B
:100860000A000000F12101080B0000000B0000004D
:10087000FB2101080C0000000C000000052201080B
:100880000D0000000D0000000D2201080E00000008
:100890000E000000152201080F0000000F000000EC
:1008A0001D2201081000000010000000262201088F
:1008B00011000000110000002D22010812000000AC
:1008C000120000003722010813000000130000008E
:1008D0003F22010814000000140000004A22010811
:1008E0001500000015000000542201081600000049
:1008F000160000005B22010817000000170000002E
:100900006322010818000000180000006B22010893
:100910001900000019000000732201081A000000ED
:100920001A0000007D2201081B0000001B000000CF
:1009300000000000FF0000000100010200010300B0
:100940000104000105000106000107000108000183
:100950000900010A00010B00010C01030D00010E4A
:1009600000010F000110000111000112000113002D
:100970000114000160270108692701080000000038
:10098000A5710008852701088927010800000000DB
:10099000A7700008382D0108992701080000000001
:1009A0007DC30008B6270108BB270108CE27010830
:1009B000D5670008DF2701080000000000000000E4
:1009C00031650008E4270108EC270108FF2701082A
:1009D0003564000812280108162801080B280108B0
:1009E00031C10008292801080000000000000000B3
:1009F000A96200082E280108322801084D280108A4
:100A0000916300085F28010855280108652801083E
:100A1000ED62000873280108782801080000000032
:100A20003D6E0008932801088B28010899280108C9
:100A3000E1BC0008AB28010800000000B62801084E
:100A400041BC0008C9280108C2280108D1280108B2
:100A500001BC0008DB280108E7280108D1280108AB
:100A6000B9BB0008FB2801080329010800000000A9
:100A7000E96600081F290108262901080000000076
:100A800009730008442901084929010800000000F1
:100A900099C30008592901086029010800000000D5
:100AA000ED7600085F320108772901080000000098
:100AB000A56500086924010888290108972901080B
:100AC00089C10008A8290108AD290108B929010830
:100AD000216B00082D2A0108282A010800000000C7
:100AE00045C00008392A0108342A01080000000026
:100AF00085BB0008FE2A0108412A0108472A01088F
:100B00004D2A0108502A0108572A01085A2A0108CB
:100B10005F2A01086B2A01086E2A0108742A01085D
:100B20007B2A0108852A0108EF2A01088F2A01087B
:100B30009D2A0108A92A0108B02A0108B62A01083D
:100B4000C32A0108CE2A0108DB2A0108E22A01088B
:100B5000E92A0108F82A010800000000912601088E
:100B6000982601089D260108AE260108B82601082E
:100B7000C3260108CE260108D9260108DD26010872
:100B8000E6260108EC260108F626010804270108DC
:100B900007270108172701081E2701082727010832
:100BA0003127010839270108442701084D2701088A
:100BB0000000000000000000000000000100000034
:100BC000FA11010800000000000000000000000011
:100BD0000000000004000000DE1101080200000017
:100BE000D01101080000000000000000000000001B
:100BF0000000000005000000AD1101080000000029
:100C000000000000000000000000000000000000E4
:100C100000000000000000000000000000000000D4
:100C200000000000050000008A110108000000001B
:100C300000000000000000000000000000000000B4
:100C400000000000000000000000000000000000A4
:100C500000000000020000007C11010808000000F4
:100C60004411010800000000000000000000000026
:100C70000000000000000000000000000000000074
:100C8000000000000000803F000000000000803FE6
:100C90000000803F0000803F000080BF000080BF58
:100CA000000000000000803F000000000000803FC6
:100CB000000080BF0000803F0000803F000080BF38
:100CC000000000800000803F0000000000000000E5
:100CD000000080BF0000803F000000000000000016
:100CE0000000803F0000803F000080BF0000803F88
:100CF000000080BF0000803F000080BF000080BF78
:100D00000000803F0000803F0000803F0000803FE7
:100D10000000803F0000803F0000803F000080BF57
:100D2000000080BF0000803F0000000000000000C5
:100D3000000000000000803F0000000000000000F4
:100D4000000000000000803FE17A14BFE17A143F08
:100D50000000803F0000803F1F85EBBE14AEC7BE81
:100D6000000000BF0000803FE17A143FE17A143FA9
:100D7000000080BF0000803F1F85EB3E14AEC7BE61
:100D80000000003F0000803F0000803F240FD4BEE1
:100D90000000803F0000803F240FD4BE000080BFD1
:100DA0000000803F0000803F000080BF240FD43E41
:100DB0000000803F0000803F240FD43E0000803FB1
:100DC0000000803F0000803F240FD43E000080BF21
:100DD000000080BF0000803F000080BF240FD4BE11
:100DE000000080BF0000803F240FD4BE0000803F81
:100DF000000080BF0000803F0000803F240FD43EF1
:100E0000000080BF0000803FF704353FF70435BF86
:100E10000000803F0000803FF70435BFF70435BF76
:100E20000000803F0000803FF70435BFF704353FE6
:100E30000000803F0000803FF704353FF704353F56
:100E40000000803F0000803F00000000000080BFE5
:100E5000000080BF0000803F000080BF0000000055
:100E6000000080BF0000803F000000000000803FC5
:100E7000000080BF0000803F0000803F00000000B5
:100E8000000080BF0000803F000080BF0000803F66
:100E9000000080BF0000803F000080BF000080BFD6
:100EA0000000803F0000803F0000803F0000803F46
:100EB0000000803F0000803F0000803F000080BFB6
:100EC000000080BF0000803F000080BF0000803F26
:100ED0000000803F0000803F000080BF000080BF16
:100EE000000080BF0000803F0000803F0000803F86
:100EF000000080BF0000803F0000803F000080BFF6
:100F00000000803F0000803F000000BFD0B35D3F85
:100F10000000803F0000803F000000BFD0B35DBFF5
:100F20000000803F0000803F0000003FD0B35D3FE5
:100F3000000080BF0000803F0000003FD0B35DBFD5
:100F4000000080BF0000803F000080BF0000000064
:100F5000000080BF0000803F0000803F00000000D4
:100F60000000803F0000803F000000000000803F44
:100F7000000080BF0000803F000080BF000080BFF5
:100F8000000000000000803F000000000000803FE3
:100F90000000803F0000803F0000803F000080BFD5
:100FA000000000000000803F000000000000000082
:100FB000000000000000803FD0B35DBF0000003F94
:100FC0000000803F0000803FD0B35DBF000000BF45
:100FD000000080BF0000803FD0B35D3F0000003FB5
:100FE0000000803F0000803FD0B35D3F000000BFA5
:100FF000000080BF0000803F00000000000080BFB4
:101000000000803F0000803F000000000000803FA3
:10101000000080BF0000803F00000000A8AAAA3F97
:101020000000803F0000803F000080BFB0AA2ABFC0
:10103000000080BF0000803F0000803FB0AA2ABFB0
:10104000000080BF0000803F00000000A8AAAA3F67
:10105000000080BF0000803F000080BFB0AA2ABF10
:101060000000803F0000803F0000803FB0AA2ABF00
:101070000000803F0000803F0000803F0000000033
:10108000000000000000803F000080BF0000000062
:10109000000000000000803F000080BF0000803F93
:1010A000000080BF0000803F000080BF000080BFC4
:1010B0000000803F0000803F0000803F0000803F34
:1010C0000000803F0000803F0000803F000080BFA4
:1010D000000080BF0000803F000000000000803F53
:1010E000000080BF0000803F000080BF00000000C3
:1010F0000000803F0000803F0000803F00000000B3
:101100000000803F0000803F00000000000080BF22
:10111000000080BF0000803F00000000A8AAAA3F96
:10112000000000000000803F000080BFB0AA2ABF7E
:10113000000000000000803F0000803FB0AA2ABFEE
:10114000000000000302640000640003016400006A
:101150006400040264000064000401640000640090
:1011600005026400006400050064000064000602DB
:101170006400006400060064000064000401640070
:101180000064000500640000640003006400006463
:1011900000040064000064000502640000640006AE
:1011A000016400006400070364000064000300643D
:1011B000000064000301640000640004009C00005F
:1011C000640004016400006400070364000064001C
:1011D000000C7D00006400010D7D0000640004022D
:1011E00064000064000401640000640005026400FF
:1011F00000640005016400006400050264000064EE
:101200000000000061687300000103030102000098
:10121000117B00089D7B0008CD7B0008AF7B000898
:10122000A97B0008AD7B00080000000080250000BD
:10123000004B00000096000000E1000000C2010029
:101240000084030090D00300C9940008779400083C
:1012500031940008FB94000861940008F59400089C
:10126000000100006DAD00086DAD000805C5000867
:101270006DAD00086DAD00086DAD00086DAD0008E6
:1012800051C500086DAD00086DAD00086DAD0008DA
:101290006DAD00086DAD00086DAD000804010000E3
:1012A0000001000001000000B01F0108482D0108E6
:1012B000020100009D1F0108582D010803020000D3
:1012C0009A1F0108682D010804030000951F0108FA
:1012D000702D010805040000901F0108732D0108FE
:1012E00006050000871F01087A2D01080706000087
:1012F000841F0108892D010808070000811F0108CB
:10130000962D010809080000662200200000000058
:101310000A0900007E1F01089E2D01080C0A00002A
:10132000791F0108A52D01080D0B0000741F01088D
:10133000B52D01080E0C0000651F0108CA2D01081B
:101340000F0D000066220020000000000B0E0000C0
:10135000611F0108D52D0108100F00005C1F010856
:10136000E32D01089E350108A1350108A9350108C2
:10137000B2350108373601083C360108403601080D
:1013800049360108E6260108D92601084536010834
:10139000000000004C210108BE350108C3350108DA
:1013A000CB350108D4350108DC350108E3350108E7
:1013B000EB350108F33501080000000000000000D3
:1013C0004C210108BE350108F8350108C335010874
:1013D00000360108083601080F360108E335010818
:1013E000EB350108F3350108000000004C2101082D
:1013F000BE3501081A360108213601080000000038
:1014000000000000000000000000000000000000DC
:1014100000000000000000004C210108BE3501085A
:1014200028360108303601080000000000000000E6
:1014300000000000000000000000000000000000AC
:1014400000000000E92D010844000000D81A002027
:1014500000000000A00F0000F22D01084100000074
:10146000DB1A00200000000001000000042E01082B
:1014700041000000DA1A0020000000000100000016
:10148000122E010841000000DC1A002000000000BC
:10149000010000001F2E010844000000641C002011
:1014A000B0040000A4060000262E0108440000003D
:1014B000661C002000000000D0070000302E01084C
:1014C00044000000681C002000000000D00700005D
:1014D0003A2E010842000000601C002000000000BD
:1014E00012000000472E010841000000611C00208E
:1014F00001000000FF000000522E01084200000021
:10150000621C00200000000001000000622E0108A3
:1015100042000000A21C00200000000001000000AA
:101520001832010844000000101C002000000000D8
:10153000D0070000772E010844000000121C002094
:1015400000000000D0070000842E010844000000C5
:10155000141C002000000000D0070000902E01089D
:1015600044000000161C002000000000D00700000E
:10157000A32E010844000000181C002000000000F9
:10158000D0070000B32E0108440000001A1C002000
:1015900000000000D0070000C42E01084400000035
:1015A0001C1C002000000000D0070000CF2E010806
:1015B000440000001E1C002000000000D0070000B6
:1015C000E42E010844000000201C0020320000002E
:1015D000007D0000F32E010844000000221C0020C2
:1015E00032000000F2010000022F0108410000005B
:1015F000AC1C002000000000010000000F2F0108BB
:1016000041000000AD1C00200000000001000000AF
:10161000222F010841000000AE1C00200000000045
:101620003C000000342F010841000000AF1C0020E6
:1016300000000000B4000000402F0108420000003C
:10164000BA1C0020FFFFFFFF01000000562F010819
:1016500041000000BC1C0020300000007E000000A3
:10166000672F0108410000005E1C00200000000000
:1016700006000000792F0108410000005F1C0020D7
:10168000000000000A0000008B2F0108410000004C
:10169000E01C002000000000010000009C2F010859
:1016A00041000000E11C00200000000001000000DB
:1016B000B02F010860000000E41C0020A6FFFFFF1F
:1016C0005A000000C82F010860000000E81C00203C
:1016D0004CFFFFFFB4000000E02F010841000000B4
:1016E000EC1C00200000000001000000F92F0108A0
:1016F00041000000ED1C002000000000010000007F
:101700000430010841000000EE1C00200000000031
:10171000010000001930010841000000EF1C00200A
:101720000000000078000000333001084400000091
:10173000541C002000000000204E0000443001082E
:1017400041000000481C002000000000FF000000D5
:101750004F300108410000004B1C00200A0000002F
:101760003200000065300108410000004C1C0020E0
:101770000A000000320000007B3001084100000038
:101780004D1C00200A0000003200000095300108C6
:10179000480000004E1C0020F0D8FFFF102700007A
:1017A000A930010844000000501C00200000000087
:1017B000E40C0000BE30010841000000531C002072
:1017C0000000000001000000DC30010841000000C2
:1017D000521C00200000000002000000EF30010851
:1017E00041000000241C0020000000000800000050
:1017F000FA30010841000000251C00200000000014
:10180000080000000431010841000000261C0020EF
:1018100000000000080000000E3101084800000030
:10182000281C00204CFFFFFF680100001F31010849
:10183000480000002A1C00204CFFFFFF6801000048
:1018400031310108480000002C1C00204CFFFFFF34
:101850006801000041310108440000003A1C0020EA
:1018600064000000840300005731010844000000B8
:10187000301C002000000000000100006031010861
:1018800041000000361C0020000000008000000025
:101890007031010844000000321C00206400000088
:1018A000E80300008131010844000000341C0020DE
:1018B00064000000E803000093310108810000008B
:1018C000031E002001000000FA000000A5310108FD
:1018D00081000000041E0020000000000100000044
:1018E0009C31010881000000011E00200000000062
:1018F00020000000BA31010881000000021E002013
:101900000000000064000000C731010881000000F1
:10191000081E00200000000096000000E1310108D0
:1019200084000000061E0020010000008403000067
:10193000FB310108420000002E1C0020FFFFFFFFCA
:10194000010000001132010841000000B01C00201D
:1019500000000000010000002532010842000000E4
:10196000B11C0020FFFFFFFF010000003932010819
:1019700044000000B21C002050000000F4010000F0
:101980005332010842000000B41C00200000000097
:10199000010000006532010848000000B61C00206C
:1019A0000A000000900100007832010842000000A7
:1019B000B81C002000000000010000008D3201086A
:1019C00081000000441D0020000000000200000013
:1019D000A232010801010000962100200000000051
:1019E000FA000000AA32010801010000972100203E
:1019F0000000000064000000B23201080101000094
:101A00009E2100200000000064000000BE3201089A
:101A10000101000098210020000000006400000087
:101A2000C6320108010100009921002000000000D9
:101A300064000000CF320108010100009A2100205B
:101A40000000000064000000D9320108010100001C
:101A50009B2100200000000064000000E432010827
:101A6000010100009C21002000000000FF00000098
:101A7000ED320108010100009D210020000000005E
:101A800064000000F632010804010000A0210020DB
:101A9000E8030000D0070000053301084100000002
:101AA000A41C002000000000C8000000143301083E
:101AB00041000000A51C002000000000C80000003C
:101AC0002733010844000000A61C0020E8030000A2
:101AD000D00700003933010841000000A81C002095
:101AE00000000000010000004E3301084400000027
:101AF000AA1C0020000000002C0100006A3301082D
:101B0000440000006A1C0020EE020000CA08000029
:101B100076330108440000006C1C0020EE02000037
:101B2000CA0800008233010881000000791E0020ED
:101B300000000000010000008E3301084100000099
:101B40002F1C002000000000090000009B3301084A
:101B5000810000004C1D002000000000FA00000081
:101B6000AA33010881000000541D0020000000007D
:101B700064000000B933010881000000551D0020F9
:101B80000000000064000000C7330108A00000004E
:101B9000501D00200100000014000000D733010890
:101BA00081000000681D002000000000010000000E
:101BB000E6330108880000004A1D0020D4FEFFFF24
:101BC0002C010000F533010888000000481D0020AA
:101BD000D4FEFFFF2C010000033401088100000047
:101BE000581D0020000000003000000011340108E2
:101BF000A00000005C1D00200000000001000000AB
